:020000041000EA
:1000000000B5324B212058609868022188439860DF
:10001000D860186158612E4B002199600221596106
:100020000121F02299502B49196001219960352056
:1000300000F044F80222904214D00621196600F024
:1000400034F8196E01211966002018661A6600F04E
:100050002CF8196E196E196E052000F02FF8012189
:100060000842F9D1002199601B49196000215960AB
:100070001A491B48016001219960EB211966A021F2
:10008000196600F012F800219960164914480160C1
:100090000121996001BC002800D000471248134993
:1000A000086003C880F30888084703B5996A0420EC
:1000B0000142FBD001200142F8D103BD02B5186610
:1000C0001866FFF7F2FF186E186E02BD00000240BE
:1000D000000000180000070000035F00212200005C
:1000E000F4000018222000A00001001008ED00E03C
:1000F00000000000000000000000000074B24E7A12
:1001000000200420F7010010C3010010C5010010F9
:10011000C1010010C1010010C1010010C101001097
:10012000C1010010C1010010C1010010C701001081
:10013000C1010010C1010010C9010010CB01001065
:10014000CD010010CD010010CD010010CD01001037
:10015000CD010010CD010010CD010010CD01001027
:10016000CD010010CD010010CD010010CD01001017
:10017000CD010010CD010010CD010010CD01001007
:10018000CD010010CD010010CD010010CD010010F7
:10019000CD010010CD010010CD010010CD010010E7
:1001A000CD010010CD010010CD010010CD010010D7
:1001B000CD010010CD010010CD010010CD010010C7
:1001C00000BE00BE00BE00BE00BE00BE00F04BF888
:1001D000103800BEF2EB8871D0D00010F8D00010BB
:1001E0003402001090A31AE700202149086006C8D5
:1001F00081F3088810471F48006800282FD10DA4FC
:100200000ECC002902D000F012F8F9E71A491B4A77
:10021000002000E001C19142FCD1194988471949E9
:1002200088471949884700BEFDE701C901C29A42C3
:10023000FBD37047F8D00010C0000020581D0020EC
:1002400090ED0010000004200000042090ED00104C
:1002500000100420001004200000000070470B482C
:1002600006F024F90047EFF30580C0B270470000A4
:1002700008ED00E0000000D0581D0020502D0020A7
:1002800049350010B50C00107536001057560000A7
:1002900006005250ABB36053B4CB0010060052506E
:1002A000861C0302C4CB0010060052505422A29DAB
:1002B000CCCB001005005250DE65F46890ED0010C4
:1002C000F8B5C0460448054B10B5834203D0044B33
:1002D000002B00D0984710BD581D0020581D00204D
:1002E0000000000006480749091A8910CB0F591869
:1002F00010B5491003D0044B002B00D0984710BD17
:10030000581D0020581D00200000000010B5074CAB
:100310002378002B09D1FFF7D5FF054B002B02D026
:10032000044800E000BF0123237010BD601E0020C0
:100330000000000018C60010054B10B5002B03D0BC
:100340000449054800E000BFFFF7CCFF10BDC046E0
:1003500000000000641E002018C6001010B50748F9
:1003600007F09AF8064C0748210007F071F92100C0
:1003700005480A3107F06CF910BDC046BCC7001033
:10038000B8130020CCC70010DCC70010F0B5D6466B
:100390004F4646462D48C0B507F07EF82C4C2D48F8
:1003A000216807F055F92C4E2C48316807F050F9B8
:1003B0002B4B2C4819689A4607F04AF92A4D2B48CE
:1003C000296807F045F92A4F2A48396807F040F9AB
:1003D000294B2A481968984607F03AF9284B2948CA
:1003E0001968994607F034F9274807F031F9216870
:1003F000264C20000AF032F9002803D1244807F0E7
:100400004BF8FEE75346200019680BF0D5FA4B462F
:10041000200019680BF02EF9434639681A6820004D
:100420000AF014FF316820000AF0CEFF296820008E
:100430000BF070FA20000BF007FB164807F02CF8C1
:100440001CBC90469946A246F0BDC046B8C60010F6
:100450000C140020C8C6001014140020E4C60010BC
:100460001014002000C70010081400201CC7001042
:100470001814002038C700100014002054C70010C2
:100480000414002070C700108CC70010B01E00209C
:10049000A0C70010B0C70010F0B5C646CA4D00B5E1
:1004A0008046FD222800002106F0CEFEC423023D36
:1004B0005B42C64E2B80C533AB703378002B00D126
:1004C000ADE1EB707378002B00D1B7E12B71B378FD
:1004D000002B00D1B6E16B71F378002B00D1B3E1B2
:1004E000AB713379002B00D18AE1EB717379002B6A
:1004F00000D1ABE12B72B379002B00D1A8E16B7274
:10050000F379002B00D1A5E1AB72337A002B00D137
:10051000A2E10C27EB727B1CBA1C1D0011003E24CB
:10052000AB48C455377D002F3FD0C754757D5A1C4A
:1005300092B2002D00D15DE18554B57D991C89B240
:10054000002D00D158E14554F57DDA1C92B2002D02
:1005500000D14FE18554357E191D89B2002D00D19F
:100560004AE14554757E5A1D92B2002D00D141E1F9
:100570008554B57E991D89B2002D00D13CE14554CA
:10058000F57EDA1D92B2002D00D133E119008554B9
:10059000327F083189B2002A00D12DE109339BB2A4
:1005A00042545A1C92B21D001100B77F002F51D047
:1005B0002C2343558754531C911CF77F9BB289B25F
:1005C0001D008C46002F00D11EE1C7542023F75C8C
:1005D000D31C9BB21D00002F00D126E147542121DE
:1005E000775C111D89B28C46002F00D10CE1C754F5
:1005F0002223F75C531D9BB21D00002F00D114E194
:1006000047542321775C911D89B28C46002F00D17D
:10061000FAE0C7542423F75CD31D9BB21D00002FC2
:1006200000D102E147542521775C1100083189B2DD
:100630008C46002F00D1E7E0C7542623F75C130057
:1006400009339BB21D00002F00D1EEE00A3292B2B6
:10065000475411002827F75D002F4DD02C23292166
:1006600043558754531C775C911C9BB289B21D0083
:100670008C46002F40D0C7542A23F75CD31C9BB272
:100680001D00002F00D1D5E047542B21775C111DB0
:1006900089B28C46002F2FD0C7542C23F75C531DF2
:1006A0009BB21D00002F00D1C4E047542D21775C80
:1006B000911D89B28C46002F1ED0C7542E23F75CA3
:1006C000D31D9BB21D00002F00D1B3E047542F2152
:1006D000775C1100083189B28C46002F0CD0C754CA
:1006E0003023F75C130009339BB21D00002F00D1AB
:1006F000A0E00A32475491B23A2242554254B57AA8
:100700009F1CBFB2002D00D180E03C3AD31A00E01C
:1007100017007A1C92B2D11889B2C5557518AD7AF6
:10072000002DF5D108293BD8202585544A1CBB1C37
:1007300092B29BB2092A00D182E00231033789B21A
:10074000BAB2C55409292BD020234E1C551CB6B271
:10075000ADB28354092E51D043558D1C961CADB2B9
:10076000B6B2092D4ED08355CE1CD51CB6B2ADB253
:10077000092E43D043550D1D161DADB2B6B2092D3D
:1007800040D083554E1D551DB6B2ADB2092E35D0A1
:10079000961DB6B24355032934D0073292B2835521
:1007A0003A23835443461978561CB6B2002919D00F
:1007B000FE2E17D8451CAD198319FD264446B21AE2
:1007C00092B20134AA1809E072290020B81300205F
:1007D0007029002001330134934203D0197021782D
:1007E0000029F7D101221D4B1A7006F055FE04BCFA
:1007F0009046F0BD1300D4E60B00D2E62A00CFE706
:10080000072788E63200CBE70A0023E720211A1DDC
:1008100003339BB2C15592B2C1541E3994E70521EE
:10082000052204250423032779E61A000D00190088
:1008300063460FE70D00190063465DE704276AE68B
:100840001A00ADE7052766E6062764E6082762E694
:10085000092760E60A275EE60B275CE6812A00206E
:10086000F0B5DE46454657464E46E0B59C4C0A225A
:10087000A54404AC0021200020AD06F0E5FCFF22D9
:100880000021280006F0E0FCFF22002160A806F00D
:10089000DBFCFF220021A0A806F0D6FC6422002188
:1008A00007A806F0D1FCFF220021E0A806F0CCFC4E
:1008B0008C4B1A78002A41D022703E2A00D1EAE0FF
:1008C0005A78002A3AD062703E2A00D1E6E09A783F
:1008D000002A33D0A2703E2A3DD0DA78002A2DD0EB
:1008E000E2703E2A00D1D0E01A79002A26D0227187
:1008F0003E2A00D1CCE05A79002A1FD062713E2AEC
:1009000000D1CEE09A79002A18D0A2713E2A00D1F7
:10091000D9E0DA79002A11D0E2713E2A00D1D5E07F
:100920001A7A002A0AD022723E2A00D1D1E05A7ADD
:10093000002A03D062723E2A00D1CDE06A4806F058
:1009400087FE00252800694B9D443CBC9046994693
:10095000A246AB46F0BD032102220020A0545A5CFF
:10096000002AEBD02A703A2A00D18FE1012201310E
:10097000585C17000028E1D0A85401323A28F6D17B
:100980000022EA555A185078002200280DD0013272
:10099000561EC027B4466E467F00F6196746F055CE
:1009A0008818181840780028F1D1C0206946002323
:1009B000400009188B542978002900D15DE10022FC
:1009C0000020002798469946431C9C46434607AEA4
:1009D000B2469B185B005344561C1954B2462C294E
:1009E00062D060460137E95D0029EDD107AB9C4636
:1009F00042445200624411543D482278817A8A422E
:100A00000BD1002A10D0002301E0002A0CD00133C2
:100A1000C118E25C897A8A42F7D0002A00D139E114
:100A2000002908D0914206D1C0226B4652009B1883
:100A30001B783A2B64D00025002760AB03933A2340
:100A40006B4402930CAB019326236B4400935246F4
:100A500007AB2100274806F0FBFDA0226B46920061
:100A60009B181B78002B00D16CE72A00A0A9224814
:100A700006F0EEFD002F00D164E7E0A8FFF70CFDC3
:100A8000E0A91E4806F0E4FD5CE70421032264E7C8
:100A90000521042261E7012100225EE702210122F3
:100AA0005BE70621052258E76146092999DC49469A
:100AB0001954092E00DDC2E0931C9A46B30032009F
:100AC000002098468EE70721062246E708210722E4
:100AD00043E70921082240E70A21353A3DE7C046AD
:100AE0007CFBFFFF5028002070C800108404000029
:100AF000B8130020F0C700102CC8001054C8001014
:100B00006B460A329B181B783A2B94D10378002B42
:100B10005AD082216A46FF31521812789A428AD1FD
:100B20004378002B50D06A460131521812789A420D
:100B300000D080E78378002B46D084216A46FF31BD
:100B4000521812789A4200D075E7C378002B3BD038
:100B50006A460131521812789A4200D06BE7037945
:100B6000002B31D086216A46FF31521812789A4202
:100B700000D060E74379002B26D06A460131521835
:100B800012789A4200D056E78379002B1CD0882136
:100B90006A46FF31521812789A4200D04BE7C37967
:100BA000002B11D06A460131521812789A4200D0B7
:100BB00041E7037A002B07D08A216A46FF31521899
:100BC00012789A4200D036E78C226B46FF329B188F
:100BD0001A78002A0FD00B23A02519006846AD0013
:100BE0000B3940194254C0216A464900013352185A
:100BF000D25C002AF0D16121A0226B4689460231E5
:100C00009200884608319B1800250027002000220A
:100C10008C461B78002B33D0A0266946B6000132E3
:100C20008919895C7B2B13D0002F31D1AE00B346DC
:100C30005D44303B6D00ED18ADB20B00EAE707AA4A
:100C400090466246B30053445B004344995475E6B2
:100C50006B460136FF369B194E461F181E544346FD
:100C60007B70C31C6046B870E0276E46BF00F61963
:100C7000581CF15401270B00CCE701239A46BBE630
:100C8000E0216A46890052181354D6E6002777E619
:100C90000300E9E7002900D0CDE6C5E6034A044B8E
:100CA0001168596092881A817047C046B0C600101A
:100CB000DC1E0020F0B5DE4657464E464546E0B500
:100CC00095B006F0D1FCFF220021914806F0BCFA55
:100CD000904FFF220021380006F0B6FA062001F0FE
:100CE00075FA052001F072FA042001F06FFA022073
:100CF00001F06CFA032001F069FAD0231B069B4631
:100D000040212022596258465A62042610230824A2
:100D1000002543624662446281617F490D708261B1
:100D20007D4A557043617C4B9D704661FA2001F00D
:100D3000BFFE5B469E619C610024774B7748DD7067
:100D400001F0B6FEFFF70AFBFFF720FB744B26000D
:100D50009946744B9846744B9A460021484609F0D0
:100D6000EFFF051E0ED143461B78002BF5D0002E59
:100D700003D16E4B9B6A9B059E0D012E21D0013E37
:100D8000B6B2EAE748460AF06BF90100684806F097
:100D90005FFC0024484609F0E1FA01345C4A631E16
:100DA000D054AC42F6D1130000225A551B783C2B8C
:100DB00003D1574B5B78FF2B20D05E4806F06CFBCD
:100DC000D1E70021484609F007FE3978002908D00C
:100DD000002401344846A4B209F046FA395D0029DE
:100DE000F7D10021484609F003FF002148460AF0E8
:100DF00075F90023424600261370AEE7444B9B78FA
:100E0000012BDAD1032D04DDEA1E4B4940480BF0DB
:100E1000FBFB3F4B9C4600236544033D60462B7023
:100E200006F03AFBFFF71CFD0500041E9BD02528A9
:100E300001D901F0AAF9414A8300D3589F464023C3
:100E40005A4693610022344B1A7043461B78002B9C
:100E50008DD182E75B460824FA205C6101F028FE10
:100E60005B469C6101232C4AD37043461B78002BC0
:100E700000D07CE771E710235A469361264A0F3B66
:100E8000937043461B78002B00D070E765E7202362
:100E90005A465361204A1F3B537043461B78002B30
:100EA00000D064E759E720235A46936100221A4B89
:100EB0005A7043461B78002B00D058E74DE71023AB
:100EC0005A4653610022144B9A7043461B78002BFC
:100ED00000D04CE741E75B460424FA205C6101F056
:100EE000E7FD5B4600229C610B4BDA7043461B78A2
:100EF000002B00D03BE730E740235A465361064AB7
:100F00003F3B137043461B78002B00D02FE724E7AC
:100F10005028002070290020DC1E002088130000CB
:100F2000B01E0020812A0020B81300200040054098
:100F30008CC80010ACC800105328002018C6001040
:100F4000D84B00211B78D8485A1E9341D54A3033DC
:100F5000137253785A1E9341D24A3033D371937827
:100F60005A1E9341CF4A30339371D3785A1E93411E
:100F7000CC4A30335371FD2206F066F9C422CA4BC5
:100F80005242023B1A80C5329A7052461278002AA9
:100F900001D100F015FCDA7052465278002A01D1D6
:100FA00000F0ABFC1A7152469278002A01D100F091
:100FB0001EFD5A715246D278002A01D100F046FD3A
:100FC0009A7152461279002A01D100F0E1FDDA71DE
:100FD00052465279002A01D100F03EFE1A72524662
:100FE0009279002A01D100F0D2FE5A725246D2798B
:100FF000002A01D100F060FF9A725246127A002A4C
:1010000001D100F0E7FFDA7218230E210F240D2220
:101010000A930C93013B0993013B0793013313930C
:10102000023B069301330893023B0593013312936D
:10103000023B049301331093023B0393013311935A
:10104000023B029301330D93023B019301330E9354
:10105000023B009301330B93023B0F93023B9C46F0
:1010600001333E2560463D545046057D002D3DD060
:10107000BD54437D002B01D100F074FC7B54837D73
:10108000002B01D100F076FC009ABB54C37D002BED
:1010900001D100F03FFD019ABB54037E002B01D12A
:1010A00000F040FD029ABB54437E002B01D100F0BA
:1010B00002FE039ABB54837E002B01D100F0A5FEF3
:1010C000049ABB54C37E002B01D100F0B6FE059AF2
:1010D000BB54037F002B01D100F074FF069A0999DD
:1010E000BB540A9B0C9C0093079A089B5046857F33
:1010F000002D63D02C20B85452467D54D27F002A54
:1011000001D100F0F9FD0098D91C3A542022504634
:10111000845C89B20A00002C01D100F06EFE7C5480
:1011200021225146181D8C5C80B20200002C01D196
:1011300000F0F9FE3C5422225046591D845C89B2CD
:101140000A00002C01D100F084FF7C542322514678
:10115000981D8C5C80B20200002C01D100F0A4FF2D
:101160003C5424225046D91D805C89B20A001C00E0
:10117000002801D100F0A1FF7854252251460834FF
:10118000885CA4B22200002801D100F0D1FF3855BC
:101190002622190050460931805C89B20A000028D5
:1011A00001D100F0CEFF1A001C000A320B3392B2BC
:1011B000785499B213000C34A4B2009428255046F8
:1011C000405D002863D00435BD547854292251462F
:1011D0008A5C002A01D100F099FD0098D91C3A548C
:1011E0002A225046845C89B20A00002C01D100F00A
:1011F00097FD7C542B225146181D8C5C80B2020056
:10120000002C01D100F09FFE52463C54591D545D04
:1012100089B20A00002C01D100F09DFE7C542D22E1
:101220005146981D8C5C80B20200002C01D100F068
:1012300029FF3C542E225046D91D805C89B20A00F9
:101240001C00002801D100F049FF78542F2251469C
:101250000834885CA4B22200002801D100F05FFFAE
:1012600038553022190050460931805C89B20A0095
:10127000002801D100F080FF1A001C000A320B3355
:1012800092B2785499B213000C34A4B200943A2567
:10129000BD5452467D54917A002900D17CE2002051
:1012A00006E0C046DC1E0020722900201400180051
:1012B00039555146431C9BB2C918897A621C92B2B7
:1012C0000029F3D11100082B42D82021A51CADB272
:1012D0008C46B9542900072800D15BE26146E01C26
:1012E00080B279550100072B00D153E26146251DDC
:1012F000ADB239542900062B00D14BE26146601D86
:1013000080B279550100052B00D143E261460634D5
:101310003954A1B2042B00D13CE22024901D80B2AC
:101320007C540100032B00D134E2D51DADB23C54F6
:101330002900022B00D12DE21000083080B27C552C
:101340000100002B00D025E2093292B211003C547A
:101350003A237B54D74B501C197980B2002911D005
:10136000FE280FD8FD239A1A92B2013200233818B2
:1013700002E001339A4205D0C154CE49C9184979D7
:101380000029F6D1012342463800137006F084F894
:1013900043461B78002B00D0E9E4DEE4FD22002167
:1013A000C54805F051FFC422C34B5242023B1A808C
:1013B000C5329A7052461278002A00D141E2DA70A2
:1013C00052465278002A00D169E21A715246927848
:1013D000002A00D1DDE25A715246D278002A00D1AB
:1013E0006AE39A7152461279002A00D1A2E3DA71B7
:1013F00052465279002A01D100F000FC1A7252467E
:101400009279002A01D100F093FC5A725246D279A7
:10141000002A01D100F021FD9A725246127A002A68
:1014200001D100F0A0FDDA7218230E220C210E204B
:101430000C930B93013B0893013B079301331393E8
:10144000023B069301330993023B05930133129348
:10145000023B049301331093023B03930133119336
:10146000023B029301330D93023B019301330E9330
:10147000023B009301330A930F928C46013B013AE1
:1014800001313E2564463D555446257D002D39D019
:10149000BD54627D002A00D15DE23A54A27D002A4B
:1014A00000D16FE2009BFA54E37D002B00D1FCE2F7
:1014B000019ABB54237E002B00D198E3029ABB54BF
:1014C000637E002B01D100F0FEFB039ABB54A37E88
:1014D000002B01D100F0A1FC049ABB54E37E002B49
:1014E00001D100F018FD059ABB54237F002B01D1D8
:1014F00000F0A7FD069A0898BB540C9B079A00932E
:1015000009990B9B5446A57F002D62D02C24BC5416
:1015100052463D54D27F002A00D1DBE30098CB1C19
:101520003A5420225046845C9BB21A00002C01D110
:1015300000F07BFCFC5452462123081DD45C80B291
:101540000200002C01D100F080FC3C5422225046C5
:101550004B1D845C9BB21A00002C01D100F069FD88
:10156000FC5452462323881DD45C80B20200002C18
:1015700001D100F090FD3C5424225046CB1D805CEC
:101580009BB21A00002801D100F0B0FDF854524679
:1015900025230C00D05C0834A4B222000B000028E4
:1015A00001D100F0B4FD3855262250460933805C45
:1015B0009BB21A00002801D100F0D5FD0A00F854B2
:1015C0000B000A320B3192B288B211000C339BB27D
:1015D000009328255446645D002C61D00435BD5429
:1015E0003C5429225046825C002A00D17BE30098BB
:1015F000CB1C3A542A225046845C9BB21A00002C21
:1016000000D1F3E3FC5452462B23081DD45C80B276
:101610000200002C01D100F08EFC52463C544B1DC0
:10162000545D9BB21A00002C01D100F01AFDFC544D
:1016300052462D23881DD45C80B20200002C01D1BB
:1016400000F017FD3C542E225046CB1D805C9BB20F
:101650001A00002801D100F038FDF85452462F231B
:101660000C00D05C0834A4B222000B00002801D189
:1016700000F045FD3855302250460933805C9BB25E
:101680001A00002801D100F065FD0A00F8540B0093
:101690000A320B3192B288B211000C339BB2009324
:1016A0003A25BD5452463D54907A002800D1B4E00A
:1016B000002505E0DC1E0020722900202300150013
:1016C00051466A1C92B28918F854887A5C1CA4B2FC
:1016D0000028F3D12100082A3AD82021981C80B292
:1016E0008C4639550100072D52D06146DD1CADB244
:1016F00039542900072A4BD06146181D80B279550C
:101700000100062A44D061465D1DADB2395429005E
:10171000052A3DD061460633795599B2042A37D05F
:101720002020A31D9BB278541900032A30D0E51D58
:10173000ADB2F8542900022A2AD0230008339BB204
:1017400078551900002A23D10934A4B22100F85495
:101750003A2352467B54083BD25C601C80B2002A7C
:1017600000D10FE6FE2800D90CE6FD21091B89B245
:1017700001310023381803E001338B4200D101E628
:10178000C2541A0054463332A25C002AF4D1F9E55F
:101790000C00DDE70A00DBE52022009903339BB251
:1017A0007A54FA54A31C9BB2FA54E31C9BB2FA5429
:1017B000231D9BB2611DFA5489B222000023ACE5BF
:1017C0000F230A930C93013B0993013B07930133C9
:1017D0001393023B069301330893023B05930133B5
:1017E0001293023B049301331093023B03930133A2
:1017F0001193023B029301330D93023B019301339A
:101800000E93023B009301330B93023B0F93023B79
:101810009C4605210422013323E420220098033151
:1018200089B23A547A54991C89B27A54D91C89B233
:101830007A54191D89B27A54591D89B21C000022AC
:101840006EE70F23052203210C930B93013B0893B2
:10185000013B079301331393023B06930133099332
:10186000023B059301331293023B0493013310931F
:10187000023B039301331193023B029301330D9317
:10188000023B019301330E93023B009301330A9311
:101890000F928C460520013B013A0131F1E51023FE
:1018A000062204210C930B93013B0893013B079301
:1018B00001331393023B069301330993023B0593D3
:1018C00001331293023B049301331093023B0393C1
:1018D00001331193023B029301330D93023B0193B9
:1018E00001330E93023B009301330A930F928C460F
:1018F0000620013B013A0131C3E510230A930C9302
:10190000013B0993013B079301331393023B069379
:1019100001330893023B059301331293023B049376
:1019200001331093023B039301331193023B029363
:1019300001330D93023B019301330E93023B00935D
:1019400001330B93043B9C460F9506210724052287
:101950000133FFF786FB019902000A9B0098009172
:101960000F99CFE5019B0A000B9C009900930F9BF8
:10197000FFF7BCFB029B009A0199009323000E9C89
:10198000FFF7B4FB0299009A0198009119000E9B91
:10199000B8E51123072205210C930B93013B089313
:1019A000013B079301331393023B069301330993E1
:1019B000023B059301331293023B049301331093CE
:1019C000023B039301331193023B029301330D93C6
:1019D000023B019301330E93023B009301330A93C0
:1019E0000F928C460720013B013A013149E5112253
:1019F00005200A920C92013A0992013A07920132AB
:101A00001392023A069201320892023A059201328A
:101A10001292023A049201321092023A0392013277
:101A20001192023A029201320D92023A019201326F
:101A30000E92023A009201320B92023A0F922B0060
:101A400007210824013A8446FFF70BFB12230A936F
:101A50000C93013B0993013B079301331393023B22
:101A6000069301330893023B059301331293023B23
:101A7000049301331093023B039301331193023B10
:101A8000029301330D93023B019301330E93023B0A
:101A9000009301330B93023B0F93023B9C460821BA
:101AA000092407220133FFF7DCFA039B0298009315
:101AB000019A0D9B0A9925E51223082206210C9311
:101AC0000B93013B0893013B079301331393023BB4
:101AD000069301330993023B059301331293023BB2
:101AE000049301331093023B039301331193023BA0
:101AF000029301330D93023B019301330E93023B9A
:101B0000009301330A930F928C460820013B013A5F
:101B10000131B6E4039B029900930D9C019A0B9B43
:101B2000FFF7E4FA049B03990093119C029A0E9B21
:101B3000FFF7DCFA1323092207210C930B93013BD7
:101B40000893013B079301331393023B0693013340
:101B50000993023B059301331293023B0493013333
:101B60001093023B039301331193023B0293013321
:101B70000D93023B019301330E93023B009301331B
:101B80000A930F928C460920013B013A013178E417
:101B900013230A930C93013B0993013B07930133F1
:101BA0001393023B069301330893023B05930133E1
:101BB0001293023B049301331093023B03930133CE
:101BC0001193023B029301330D93023B01930133C6
:101BD0000E93023B009301330B93023B0F93023BA6
:101BE0009C4609210A2408220133FFF73AFA049B94
:101BF00003980093029A119B0E9983E414230A22FE
:101C000008210C930B93013B0893013B079301338D
:101C10001393023B069301330993023B059301336F
:101C20001293023B049301331093023B039301335D
:101C30001193023B029301330D93023B0193013355
:101C40000E93023B009301330A930F928C460A20B5
:101C5000013B013A013114E414230A930C93013B34
:101C60000993013B079301331393023B069301331E
:101C70000893023B059301331293023B0493013313
:101C80001093023B039301331193023B0293013300
:101C90000D93023B019301330E93023B00930133FA
:101CA0000B93023B0F93023B9C460A210B24092213
:101CB0000133FFF7D6F9059B04990093109C039A12
:101CC0000D9BFFF713FA059B04980093039A109B52
:101CD0000D9917E49D1C581CACB2009A190080B2F3
:101CE0000094230075E49D1C581CACB2009A1900A6
:101CF00080B200942300D3E4A51C611CA8B2009A12
:101D0000230089B200900400FFF758FAA51C611C5B
:101D1000A8B2009A230089B200900400FFF7B7FA36
:101D20005C1DA4B2043399B200941300FFF7AFFA1C
:101D300015230B2209210C930B93013B0893013BC4
:101D4000079301331393023B069301330993023B3C
:101D5000059301331293023B049301331093023B2A
:101D6000039301331193023B029301330D93023B22
:101D7000019301330E93023B009301330A930F92B8
:101D80008C460B20013B013A0131FFF77AFB15230A
:101D90000A930C93013B0993013B0793013313937F
:101DA000023B069301330893023B059301331293E0
:101DB000023B049301331093023B039301331193CD
:101DC000023B029301330D93023B019301330E93C7
:101DD000023B009301330B93023B0F93023B9C4663
:101DE0000B210C240A220133FFF73BF94B1D9BB258
:101DF000043188B20093110052E45C1DA4B2043394
:101E000099B200941300FFF7D9F9069B0599009346
:101E1000129C049A119BFFF769F9069B05980093A1
:101E2000049A129B1199FFF76DFB4B1D9BB2043175
:101E300088B200931100FFF7CCFB079B0699009333
:101E4000089C059A109BFFF751F98B1D9BB2053139
:101E500088B200931100FFF7BCFB16230C220A2165
:101E60000C930B93013B0893013B079301331393AE
:101E7000023B069301330993023B0593013312930E
:101E8000023B049301331093023B039301331193FC
:101E9000023B029301330D93023B019301330E93F6
:101EA000023B009301330A930F928C460C20013BB6
:101EB000013A0131FFF7E5FA16230A930C93013B2F
:101EC0000993013B079301331393023B06930133BC
:101ED0000893023B059301331293023B04930133B1
:101EE0001093023B039301331193023B029301339E
:101EF0000D93023B019301330E93023B0093013398
:101F00000B93023B0F93023B9C460C210D240B22AA
:101F10000133FFF7A6F8079B06980093059A099BE3
:101F20001099FFF7EFFA9C1DA4B2053399B2009403
:101F30000300FFF743F98B1D9BB2053188B2009374
:101F40001100FFF7ADFB9C1DA4B2053399B20094BC
:101F50000300FFF79CF9DC1DA4B2063399B200948C
:101F60001300FFF794F917230D220B210C930B9309
:101F7000013B0893013B079301331393023B069304
:101F800001330993023B059301331293023B0493FF
:101F900001331093023B039301331193023B0293ED
:101FA00001330D93023B019301330E93023B0093E7
:101FB00001330A930F928C460D20013B013A013107
:101FC000FFF75FFA099B07990093139C069A129BEF
:101FD000FFF78CF817230A930C93013B0993013BFD
:101FE000079301331393023B069301330893023B9B
:101FF000059301331293023B049301331093023B88
:10200000039301331193023B029301330D93023B7F
:10201000019301330E93023B009301330B93023B78
:102020000F93023B9C460D210E240C220133FFF737
:1020300018F8CB1D9BB2063188B200931100FFF750
:10204000C8FA089B07980093069A139B1299FFF70A
:1020500059FADC1DA4B2063399B200941300FFF7BD
:10206000ADF8CB1D9BB2063188B200931100FFF78B
:1020700017FB0B00083307319BB288B200931100A5
:10208000FFF70EFB1C0008340733A4B299B200948A
:102090000300FFF7FCF80B00083307319BB288B24E
:1020A00000931100FFF795FA1C0008340733A4B21F
:1020B00099B200940300FFF781F809340833A4B201
:1020C00099B200941300FFF779F80B000933083137
:1020D0009BB288B200931100FFF7E2FA093408338B
:1020E000A4B299B200941300FFF7D1F80B000933A2
:1020F00008319BB288B200931100FFF76AFA0A33E5
:1021000009319BB288B200932100FFF7C9FA0A3364
:1021100009319BB288B200932100FFF75AFA1C00E4
:102120000A340933A4B299B200941300FFF7AFF850
:102130001C000A340933A4B299B200941300FFF7CB
:102140003DF81C000B340A33A4B299B2009413007A
:10215000FFF734F80B000B330A319BB288B20093BF
:102160001100FFF79DFA0B000B330A319BB288B2C6
:1021700000931100FFF72DFA1C000B340A33A4B2B0
:1021800099B200941300FFF782F8434619780029AA
:1021900001D1FEF7E3FDFEF7EAFDC046094A8300E0
:1021A00094464022634410B51C68C0006240C024BD
:1021B00014408022520113431C60034B9C46604430
:1021C000416010BD04C00140004001400123D02205
:1021D0008340120693629361094A83009446402229
:1021E00063441968C0004A40C02111408022520156
:1021F00013431960034B9C460523604443607047BA
:1022000004C0014000400140F8B5EFF3108772B6FA
:102210000D4E3368002BFCD0BFF35F8F0725CB0832
:10222000C01801230D40AB401D000478254007D1A4
:1022300023430370BFF35F8F356087F31088F8BDC9
:10224000100001F019FAC0462C0100D0F8B5CE46B6
:1022500047468C4680B5EFF3108972B6214D2C6845
:10226000002CFCD0BFF35F8F9A422CD807210125A8
:1022700011408D40D4080419267835421FD007211B
:102280008846063909E045460F001540AF40D4089E
:10229000041926783D00374211D001329342F2D220
:1022A00001204042BFF35F8F00220E4B1A6089F37A
:1022B000108800280FDB0CBC90469946F8BD3543CA
:1022C00025701000EEE7BFF35F8F00232B6089F3CA
:1022D0001088012040426346002BECD0089801F0A2
:1022E000CBF9C0462C0100D0024B18688007C00F04
:1022F0007047C04600C006400021044B044ABFF3AB
:102300005F8F02C39342FAD17047C046000100D0EC
:10231000800100D0044A1078431CDBB2172B00D98F
:10232000102313707047C0461C14002000B5054BE5
:1023300083B00100009318221F230348FFF786FF94
:1023400003B000BDD0C800108C23002083680B4868
:1023500010B5844661446244090112019A18591863
:1023600054684B6801209C4201D802D00020C0B2C2
:1023700010BD12680B689A42F9D8F7E7FFFFFF0F0C
:102380000A4B1968EFF3108072B60A68002AFCD075
:10239000BFF35F8F1B68BFF35F8F00221A6080F36B
:1023A000108840BF002000217047C04654290020FB
:1023B000F8B557464E464546DE46E0B51F000CAB25
:1023C0001D780DAB1B7881469A4603681600984627
:1023D000002D3BD1987B002832D042464546440030
:1023E00012682418033C121951780300A9730029BC
:1023F00000D1E9730021050091705170117029E03E
:10240000D31814199D702278002A00D05A705B46A8
:10241000237043465D734B463200187D3B0000F04D
:1024200003FD041E07D05346002B04D14B46290060
:10243000186800F0E9FE0E9B002B44D028001C70A9
:102440003CBC90469946A246AB46F8BD2B006C00BA
:102450006419033C1D4A94464A4692686344944674
:102460001B010A9A63449A600B9A1E605F60DA60EF
:10247000434600221B681B199A705A701A70434613
:102480005B7B9B46002BC4D043462A009868594684
:102490005B6898475B4642465B005B44033B1268BF
:1024A0000028ADD0D31814195A46A2701A78002A01
:1024B00007D11D705A46434628005A73AB45BFD119
:1024C000A9E76270F5E72800BAE7C046FFFFFF0FF3
:1024D000F0B5DE46454657464E46724B8200E0B5A3
:1024E000D55800238DB00B909B4627E0069A079B9A
:1024F0001100194303D02B69002B00D093E02B6807
:10250000DA7B002A07D051008A1819688C464946A0
:102510006244033A51704A46DA73EA684B4694467D
:10252000013B63441A7801321A705B462B616B6879
:10253000BFF35F8F5A461A6084F3108800F012FCD4
:102540006A68EFF3108472B61368002BFCD0BFF3F7
:102550005F8F2B689C465B7B9946002B5BD0AA68FB
:10256000514B90464B441B01984443461A685B68A4
:1025700016001F00361A8F41002F6EDD0B9800F0F9
:1025800053FC0022002300270026089209936B6861
:10259000BFF35F8F5A461A6084F31088002E76D0FE
:1025A000534618024B4639001843B0476A680690F4
:1025B0000791EFF3108472B61368002BFCD0BFF3C1
:1025C0005F8F079B002B91DA2B69002B97D0069821
:1025D0000799089A099B121A8B4108980999069243
:1025E0000793079A914203D807D1069A904204D9DB
:1025F00001225242D317069207935B4601210493AE
:102600004B460391029301970096069A079B280078
:10261000FFF7CEFE89E700220023002708920993E6
:1026200000260020B3E700F09DFB069A079B1218D6
:102630004B41994202D804D1904202D90122524220
:10264000D3175946049101210391494601970291FC
:1026500000962800FFF7ACFE67E7002F01D1002E9F
:102660008CD10021604600F023FD43461A685B6868
:102670000892099343469E68DF68EB684B44013B30
:102680001B789A461B021843286100207FE7002828
:1026900000D053E70DB03CBC90469946A246AB46ED
:1026A000F0BDC04638280020FFFFFF0F10B5124CC8
:1026B0006368002B04D00A21104800F041FC10BDD3
:1026C00023000F4A1021206800F0D4FC032000F002
:1026D0003DFB032000F014FC0A49032000F05EFBE0
:1026E000FFF718FE084B9C46032360442375074BF5
:1026F00080006060DC60DEE72014002054290020A8
:102700004D230010D1240010400000343828002050
:102710000048704720140020F0B54546DE46574675
:102720004E46E0B585B00092019310AB1B780500D2
:102730009B4600239A4698466A68EFF3108972B662
:102740001368002BFCD0BFF35F8F2E68B47B002C86
:1027500050D067003F193368033FDB195A78B273D2
:10276000002A00D1F27342469A705A701A70AA6811
:10277000534B94460099019AE3181B016344196076
:102780005A600E9A9A600F9ADA6042463368DB19F3
:102790009A705A701A70737B0393002B40D0190003
:1027A000736822009C46B068E047039932688C4603
:1027B0004B006344033B00282BD0D719D318B970C2
:1027C0001A78002A00D073E01C70039B73739C423C
:1027D00027D0EB681B19013B18786B68BFF35F8F3C
:1027E00042461A6089F310885346002B26D1000216
:1027F000204307E06B68BFF35F8F1C6089F310888C
:102800000120404205B03CBC90469946A246AB46EA
:10281000F0BDD318D7199C703A78002A44D139708A
:102820007473287D009A019B00F0FEFA824600280E
:10283000CFD02100286800F0E7FCCAE75B46002BF8
:1028400030D00E9B0F990020984703000B4329D0EE
:1028500006000F1E15DA0098019902000B00921B6A
:10286000BB41994202D808D1904206D901235B426C
:10287000DC1700930194DA465EE700920193DA4692
:102880005AE700F06FFA36184F4100960197B942A7
:10289000ECD8F0D1B042EED901235B42DC170093B3
:1028A0000194E8E70020ADE75A70039B3B70B7E75F
:1028B0007A701C70039B73739C4200D089E7B0E769
:1028C000FFFFFF0FF0B557464E464546DE46040073
:1028D000E0B50D0006267642F71736196F4185B030
:1028E0008F4200D987E000D182E000F03BFA32004D
:1028F0003B00121A8B41002B00DC87E0674B9946A6
:102900005A68EFF3108B72B61368002BFCD0BFF33C
:102910005F8F4B461B6898469B7B9A46002B7BD06B
:102920005B0053444246033B9C4641461268009379
:10293000624453788B73002B00D1CB73002349463C
:102940009370537013708968554A8C4652445549A8
:1029500012016244166057609160D360009942464C
:102960008C461268624493705370137043465B7BCD
:102970000393002B00D16FE01900404643465246B6
:102980005B6880689847039B9C465A006244033A00
:10299000002854D0009940468C46036803999A1841
:1029A000634499701178002900D059705346137010
:1029B0004246039B53739A4551D04B465B68BFF325
:1029C0005F8F00221A608BF31088BC46B0460094DB
:1029D000019500266546344F344A7B6A9D424CD8A7
:1029E000B96A414501D29D4247D0009C019D1BE040
:1029F000864200D879E70026002700F0B3F93200BC
:102A00003B00121A8B41002B00DD77E7002B0BD126
:102A1000002A00D072E707E04B465B68BFF35F8F88
:102A200052461A608BF310882000290000F0A6F9A6
:102A300005B03CBC90469946A246AB46F0BD434625
:102A40001968009B8A18CB18514691701978002993
:102A500000D05170039A1A70434652465A734B463F
:102A60003200187D3B0000F0DFF90028A5D04B466E
:102A70005146186800F0C8FB9FE71168EFF310801B
:102A800072B60B68002BFCD0BFF35F8F1368BFF3E7
:102A90005F8F1E6080F3108820BF9EE72014002007
:102AA000FFFFFF0F81230010004005405429002044
:102AB00070B5060000F056F9FA2204000D009200ED
:102AC00000233000002104F053FB001969418D42BE
:102AD00005D901204042C117FFF7F4FE70BD8D42B9
:102AE000FAD18442F5D8F7E7F8B557464E46DE46A8
:102AF0004546664CE0B581460F006268EFF31088EA
:102B000072B61368002BFCD0BFF35F8F2668B57BCD
:102B1000002D00D19FE06B005B19033B9A463368A0
:102B200053441A005B78B373002B00D1F373002376
:102B3000937053701370A168554A8C464946AA1881
:102B40001201624411605349D3605760916032684A
:102B50005244937053701370737B9B46002B6DD05F
:102B60002A001900B068736898475B465A005A44B7
:102B7000033A002857D0594633689A18534499703D
:102B80001178002900D059705B46157073735D454C
:102B900055D00026E36862685B19013B1B78BFF3E0
:102BA0005F8F0021116088F31088002E59D11B021D
:102BB0001D4320BF6268EFF3108872B61368002BC4
:102BC000FCD0BFF35F8FFF232068E9B2427B2B402C
:102BD0008A4250D05A00924602689A44944652461D
:102BE0006244033A9278002A45D123699D4200D17C
:102BF00022616368BFF35F8F00221A6088F3108838
:102C0000254A536A9F4207D8926A01264A4503D251
:102C1000FF1A7B1E9F41FEB230003CBC9046994695
:102C2000A246AB46F8BD534631688A18CB1895705A
:102C30001978002900D051705A461A707573207D9A
:102C40004A463B0000F0F0F8061EA2D0290020689A
:102C500000F0DAFA9EE76368BFF35F8F1D6088F3C8
:102C600010880D4A0026536A9F42D5D8926A0136D1
:102C70004A45CDD3D0E7E2682D0A94466344013B30
:102C80001B78AB42B5D100F0BFFAB2E720140020A8
:102C9000FFFFFF0F8123001000400540F0B5C6463E
:102CA00000B5EFF305833F22134018001038EFF30F
:102CB000108772B61F4D2A68002AFCD0BFF35F8FC1
:102CC000012211008140884644461B494C631B4C3D
:102CD0002678A4463400C440224007D1BFF35F8F5A
:102CE0002A6087F3108804BC9046F0BD4C6A1449F2
:102CF000820051588C420FD3124BD25843469E4308
:102D000063461E70BFF35F8F00232B6087F310882C
:102D1000002AE8D09047E6E70B4A9B0094466344BC
:102D20001A681A60BFF35F8F00232B6087F3108847
:102D3000D9E7C046280100D000400540882A00207D
:102D4000602900207C220020D03F054010B5010002
:102D5000024A0348FFF758FA10BDC046ECC80010FD
:102D6000852A0020044A516A00E01900906A536ADB
:102D70009942FAD17047C04600400540064A536A5E
:102D80009942FCD807D1044B02E05A6A914202D121
:102D90009A6A8242F9D370470040054070B504003A
:102DA0000D00EFF3108672B61A4A1368002BFCD0A0
:102DB000BFF35F8F002D1BD0200000F0FFFD1649F0
:102DC00088420AD0200000F001FE0121200000F01E
:102DD000DBFD0123A340114A1360114BA400E55011
:102DE000BFF35F8F00220B4B1A6086F3108870BD13
:102DF0000B4BA200D5500122A2400A4920000B78BB
:102E000093430B70044900F00BFE0021200000F0FA
:102E1000BBFDE5E7280100D09D2C0010386005407F
:102E20007C220020882A0020F0B5D6464F46464630
:102E30002E4CC0B5656A00E00D00A66A616AA94221
:102E4000FAD1AB4248D9EFF3108972B6284C216809
:102E50000029FCD0BFF35F8F264901268C460978F4
:102E600086400F00884661463743FFB20F70041D4D
:102E70001E49A400204D4E636250840063510D6AC8
:102E8000002435421BD04D6A00E025008C6AA24622
:102E90004C6AAC42F9D1AB4224D801D1524521D879
:102EA000474521D0114B154A1E625E631F2318400F
:102EB0001E3B834013606346424601241A70BFF3F1
:102EC0005F8F00220A4B1A6089F3108820001CBC17
:102ED00090469946A246F0BDAB4201D1B242B2D86B
:102EE0000124F3E70024EAE70124E8E70040054075
:102EF000280100D0882A00206029002080E200E01C
:102F000010B5EFF3108472B60A490B68002BFCD0A1
:102F1000BFF35F8F01238340074A0848136202789A
:102F20009A430270BFF35F8F00230B6084F3108815
:102F300010BDC046280100D000400540882A00206E
:102F4000024B9C4661448900016070474000003498
:102F500010B50400FFF7DEF901002000FFF7F0FFD5
:102F6000FF232371BFF35F8F10BDC04610B504006F
:102F7000FFF7D0F901002000FFF7E2FFFF23A38055
:102F8000BFF35F8F10BDC04610B504000120FFF7EE
:102F9000CDF9044B9C46604480002060BFF35F8FF6
:102FA00010BDC04640000034F8B54746CE4680B557
:102FB0004C0003686418033C1A19567807000D008A
:102FC000002E04D128000CBC90469946F8BD710033
:102FD0008919033988464344597889460021597034
:102FE0005170002D11D07B6832002900806898470D
:102FF0003B68002832D01A1943449D70117800298B
:1030000000D059701670A04600E035004B46002BEA
:10301000D8D049463800FFF7C7FF041ED2D00200BF
:103020007B682900B868984763001B19033B3A681E
:10303000002809D1D318424494701978002900D08F
:1030400051701D702500BDE74146D31851189D7081
:103050000A78002A00D05A700C70B3E742461C1957
:103060009A18A6701378002B00D063701570350085
:10307000CCE7C04610B583600023CCB24373013364
:10308000047342608373C4730068012C06D9421C28
:103090000133DBB2137003329C42F9D8FF2319408D
:1030A0004B005918002340180338437010BDC04628
:1030B000F0B54E4657464546DE46E0B5467B0368CA
:1030C0007400A419033C1A19177883B005008946C7
:1030D000002F1ED1002911D0C07B00282AD041002A
:1030E0000918591803394E70EE73002F06D0790075
:1030F000C9190339884600214344997000233000E0
:1031000053706F7303B03CBC90469946A246AB46E1
:10311000F0BD7900C91903398846591848788246A4
:10312000002809D149460029E5D0E87B0028D6D1FE
:10313000EE73DCE7EE73E1E742005244033A934654
:103140005B445A78019200225A704A706B68020000
:103150003900A86898472B68002830D1414650466E
:103160005A4659189A1888701078002800D048706C
:103170001770D8465746019A002A2DD01100280012
:10318000FFF712FF8246002825D0020039006B6845
:10319000A868984753465900514403392B680028C2
:1031A0001CD04246591898188F70027894461A1904
:1031B0006446002C00D04C7051460170B2E759466D
:1031C000424659189A188F701078002800D048701D
:1031D00051461170CFE72B681A19A3E75A18984483
:1031E00093465046424690705A461278944660463E
:1031F0001A19002802D04046644644705846884652
:10320000077057468EE7C046F0B54546DE4657463E
:103210004E46E0B50C0083B005000023002927D0FE
:103220006600477B01683619033E8819A74233D0F0
:103230008278002A1CD053009B18033BCB181A78C5
:10324000A2421FD142781A70002302788370437023
:103250009146002A33D1EA7B002A66D053009B189E
:10326000C91803394C70EC730023437001236F734A
:10327000180003B03CBC90469946A246AB46F0BD50
:10328000002AE1D053009B18033BCB185A78A24286
:10329000F6D142785A70D7E702780192002A46D1D7
:1032A000EA7B002A3FD053009B18C91803394F709E
:1032B000EF7300234370019B6B730123D8E7520027
:1032C0004A44033A90468A185778002F42D1EB7B44
:1032D000002B00D029E14F466E7BEC7300239370E6
:1032E0004370002EC2D03A006B683100A86898473E
:1032F00073009B19033B2A68002808D0D318424466
:103300009670197800290CD11F703700AEE741463E
:10331000D31851189F700A78002A00D05A700E7086
:10332000A4E75170F0E7EF73C3E7EC739CE7140078
:10333000A44652006244033A90468A185478A14643
:10334000002C58D1EB7B002B00D0F7E0EF7300236B
:103350009370AEE77800C01903388246514448782C
:103360004B7053706B6883463A004946A86898478B
:103370002B68002800D1A2E04246981852469918BE
:103380004A468A70019002000078002801D0019A14
:10339000487017704F465A46002A28D059462800D0
:1033A000FFF702FE8146002820D002006B6839003A
:1033B000A86898474B465B004B44033B9C4600285B
:1033C0006DD042462B689818624699188F7001900C
:1033D0000078002800D083E04A4601980270E97B1B
:1033E00098196E7B002951D1019A76E72B684246E5
:1033F0009A180192F3E7600048440338824651442A
:1034000048784B7053706146220083466B68A86809
:10341000644698472968002878D0524643468A185F
:10342000CB1894701878002800D050704A46C246D5
:103430001A705B46002B50D059462800FFF7B4FDA8
:103440008046002848D0019C020021006B68A868D3
:10345000984743465A004244D31E2968002844D066
:103460005246CB188A189C701078002800D05870EB
:1034700043461370EB7B8819002B00D166E75E0092
:10348000F318C91803394F70EF7360E74A00944688
:1034900061445B18033B5C70019AEC731EE729687A
:1034A0004846CA184346CB18987010788046881949
:1034B0004646002E00D05E701770E04607E7414692
:1034C000524659189A188F701078002800D048700A
:1034D0004946D04611705EE729685346CA18C9E7C5
:1034E0004A46487001990A7079E7CA18534640461F
:1034F000CB1898701078844664468819002C00D048
:103500005C70019B1370434601931BE75346CA1836
:1035100043464846CB1898701078002800D0587061
:10352000019B13704B46019383E703267343C9182D
:1035300003394C706E7BEC734F46CFE60326734322
:10354000C91803394F7001E72D4B2E4A70B51A6028
:103550002D4A2E4B2E491A6010008B689843FBD1E0
:103560002C4C2D4DAC4209D20322231D0335ED1AFC
:103570009543ED1808CC9847AC42FBD100F09AF87F
:10358000264A224B1A60224A9368DB018033FBD122
:103590004022234B2348244D9A675A671A67DA66FC
:1035A000A84205D30EE0FFF7E1FC2000AC4209D2AF
:1035B000040003680834002BF5D1FFF7C9FC200094
:1035C000AC42F5D3194D1A4CC022A168280003F073
:1035D00041FEA560FEF790FE00F05CFBFFF766F889
:1035E000144C154DAC4209D20322231D0335ED1AAC
:1035F0009543ED1808CC9847A542FBD170BDC04655
:1036000000E00040BFCDFBFEFE7F3C0000F000402C
:1036100000C00040381D0020481D0020FFFFFF01B2
:1036200000F00140301D0020381D00200000002067
:1036300000ED00E0481D0020581D002000BEFDE701
:10364000094A1368002B06D008491818884208D880
:10365000106018007047064B044918181360884220
:10366000F6D901235B42F4E728240020000004205F
:10367000502D002000BEFDE70FB400B5084883B010
:1036800003F00AFF049B002B07D005A91800019145
:1036900002F0ECFE034803F0FFFE00BEFDE7C0466B
:1036A0001CC9001050C8001010B50148FFF7E4FF16
:1036B00010C9001030B50C2083B000F04FFBFEF7AE
:1036C00013FE00280ED0964B964A1A605A609A60F4
:1036D000DA601A615A619A61DA611A62924A5A6230
:1036E00003B030BD914CA06700F08CFB0122904BE1
:1036F0001A60636C012BFCD103228E4B1A608B4A3B
:10370000936B012BFCD1022405338B4A01218B489A
:10371000009400F0D1FA0523894A009401218948D8
:1037200000F0CAFA884B5A68FF2A02D88022520059
:103730005A6080227A4C7F4B21691201824D1A60B7
:10374000002900D0E5E0E0217F4B02201A681140FB
:10375000802252012A431160196848400321014028
:10376000116004219A681142FCD0802280219201CC
:103770002A4309011160802252005A60734B236171
:10378000734B5968FF2900D8C1E00322684B704889
:103790001A60012103009A681142FCD0E0251A68E2
:1037A000154080225201024315601B684B400321E3
:1037B000194011600221664A93681942FCD08023A7
:1037C00080219B010343090119608021614B49005D
:1037D00051606361604B5A68FF2A00D859608022AB
:1037E0005E4BE16912015C4D1A60002905D06069E9
:1037F00002F0B2FE01300138FDD1E02256490B68DB
:103800001A4080235B012B431A60802380229B0196
:103810002B4312011A608022424B52004A60E3613E
:103820004F4B5968FF2900D85A6080224D4B216ABE
:1038300012014B4D1A60002905D0606902F08CFE20
:1038400001300138FDD1E02245490B681A40802340
:103850005B012B431A60802380229B012B431201C2
:103860001A6080235B004B602E4B3F4A23623F4B24
:103870005968914201D801325A6080223C4B616AFA
:1038800012013A4D1A60002905D0606902F064FE09
:1038900001300138FDD1E02234490B681A40802301
:1038A0005B012B431A60802380229B012B43120172
:1038B0001A608023DB024B601B4B63622D4B5A68FE
:1038C000FF2A02D8802252005A6080222A4BA16926
:1038D0001201284D1A60002905D0606902F03CFEF3
:1038E00001300138FDD1E02222490B681A408023C3
:1038F0005B012B431A60802380229B012B43120122
:103900001A6080235B004B60124BA361E8E65A60AB
:103910003BE7606902F020FE01300138FDD112E77B
:1039200090230020006CDC021BB7000000800040E8
:103930003CB0004030B00040002F68590080024089
:1039400000389C1C00C0024030800040001BB700C3
:103950003C800040405973075480004054B0004000
:103960006080004060B00040FFFF03006C800040BA
:103970006CB000404880004048B00040014B8000DF
:10398000C05870479023002001238340002902D1B2
:10399000034A13607047034A1360034A1360F9E750
:1039A00080E100E080E200E000E100E001238340EC
:1039B000014A13607047C04600E200E0024B10303D
:1039C0009B688000C058704700ED00E070B50D00A6
:1039D000EFF3108672B60F4A1368002BFCD0BFF3CA
:1039E0005F8F0D4B10309B6884001B590B4A93422C
:1039F00003D09D4201D0FFF757FE074B9B681D5136
:103A0000BFF35F8FBFF35F8F0022024B1A6086F314
:103A1000108870BD240100D000ED00E0CD01001041
:103A2000F0B54546DE4657464E46E0B50D0083B03C
:103A3000EFF3108A72B65D4A1368002BFCD0BFF317
:103A40005F8F1022914681444A46594B96009B68ED
:103A50009C59584B98469C4205D0AC4251D0564F89
:103A6000E31B2F2B12D9524B9B689C51BFF35F8FE6
:103A7000BFF35F8F00224D4B1A608AF3108803B0AA
:103A80003CBC90469946A246AB46F0BD012383401C
:103A90009B465A46494B1B681A4000925A46484B6F
:103AA0001A60BFF35F8FFCF7DEFB0190002803D0A4
:103AB000814501D0FFF7F8FD012322009A43414BD5
:103AC00006209C4613006146DB1B5B415943090DF0
:103AD00093688C4610569D420AD151E043001B1852
:103AE00006209B00FB1899681856A94211D01A00AD
:103AF0000028F3DA009B002B05D15A46304B1A60A0
:103B0000B1E71C00AFE75A462F4B1A602B4B1A60E7
:103B1000A9E7002825DB4200111889007D18884696
:103B2000A9689960E979D971062169569971A979CD
:103B30007F2913D8AD88F91A6D052D15454449190B
:103B4000E0250905490D2D022943998012181F4BC4
:103B50009200BF181A781870BA71CBE7BD2109021C
:103B6000F3E70199002913D1002A0FD0FF209071AB
:103B700017489080154A1078987163461370B9E71A
:103B800013000028C7DA019A002A01D14446F1E760
:103B9000104A1149D21A083A5002400D0143998047
:103BA0000E4952080A43DA80A4E7C046240100D037
:103BB00000ED00E0CD0100104814002000E100E01D
:103BC00080E100E0AAAA000080E200E0862A00204E
:103BD00000BDFFFF8214002000F0FFFF00F8FFFF90
:103BE000F8B5012504000543FCF73DFBEFF3108613
:103BF00072B6214A1368002BFCD0BFF35F8F1F4BB6
:103C00001F4A2100C91A49414A43120D1D4980002B
:103C10008F6852B23F58AF421CD00621595691428C
:103C200026D012215956914224D01E215956914234
:103C300014D02A2159560320914210D0124B1978E2
:103C40001A70A171BFF35F8F00220B4B1A6086F3CD
:103C50001088F8BD8B680D491950EFE7022041002C
:103C6000091889005B18FF21997109499980E5E7D6
:103C70000020F4E70120F2E7240100D048140020DE
:103C8000AAAA000000ED00E0862A0020CD01001065
:103C900000BDFFFF054B064A1360064A13605360E0
:103CA0009360D3601361536193617047808080801B
:103CB00000E400E004E400E0F8B504000C201E007D
:103CC00017000D0002F048FC4201121A9101891AF6
:103CD000C90009188901380002F03EFC069B360431
:103CE0001B031E432368002B21DB184BE2185342B1
:103CF0005A4180235B019C4652421A40144B624455
:103D00001A60144B1A60144B170099688F43FBD14B
:103D1000C023221D9B01134321222560A0601A604D
:103D20002268002AFCDA0822E6601A60F8BD3F2308
:103D300022681340AB42D8D1A3681B051B0D8342F8
:103D4000D3D1E368002ED0D1F0E7C0460040FDBFDC
:103D500000E0004000F0004000C0004080239B00D5
:103D60001843014BD86270470080054010B580248D
:103D70001B4BE4051C6000281AD00123194C184382
:103D8000194BDC61194C44401C62596298628021D5
:103D9000134BC9051960164816490860E021C9048B
:103DA0001960002A07D18022134B12061A6010BD39
:103DB0000D4BD861EBE753019B1A9B009A180F4BF0
:103DC00012019A4208D80E4B1A60074B5A608022A3
:103DD000094BD2051A60EAE7094A13601A00F4E7B2
:103DE00000B00540D3C007B0008005402D3FF84F1C
:103DF000FCFF01000820014000A00540FFFFFF007C
:103E000030280020AA23064A1B0113602F230549EE
:103E1000D360054B19605368002BFCDA7047C0462D
:103E20000040024000B0FA00006002407047C04607
:103E300010B5002803D04A680B681100984710BDE0
:103E400010B5002801D003F0D7FA10BDF0B55746E1
:103E50004546DE464E46E0B585B0984610AB1D7827
:103E6000139B93469A460223149A0F0013400600B0
:103E70000F9C12990193002B2DD1013313409C46C6
:103E80005346002B66D18C420DD21F2C00D912E173
:103E90000E9B30201B1902E00133202C03D001348B
:103EA0001870A142F8D86346002B14D0A24512D94D
:103EB0000E9B30201B191F2C21D8AC4615005246F2
:103EC00002E00133202C17D0013418709442F8D14D
:103ED00092462A006546D3062ED5530519D4002CE8
:103EE00011D1119B102B00D1D9E0022B1FD10E99BB
:103EF00060330B7001241AE092462A006546D3060F
:103F00003ED5530505D4A14200D19FE0544500D1D0
:103F10009CE0119B102B65D0022B06D11F2C65D87D
:103F200062210E9B1B19197001341F2C5ED83021A1
:103F30000E9B1B19197001341F2C57D8002D1BD153
:103F4000530700D570E0130750D520230E990B5569
:103F5000013415E06346002B6BD0002D00D070E0DB
:103F60000C2313426DD18C42A0D21F2C90D9534602
:103F70002024202BC3D8AEE72D230E990B550134F6
:103F8000930736D05B4603931A000E9B0294994622
:103F90004B46013C551C185D39004346B0472A008A
:103FA000002CF5D1039A029B944663441D00019BAB
:103FB000002B0FD05B46EB1A53450BD22A005D460F
:103FC000541C434639002020B0472200631B534550
:103FD000F6D32500280005B03CBC90469946A24681
:103FE000AB46F0BD930641D51F2C52D95D469307D1
:103FF00012D1544538D25B4653441B1B0F941C000E
:104000000F9B5A469946551C434639002020B0471D
:104010002A00A542F7D14C46002CC8D00E9B039530
:1040200002942A009946B3E72B230E990B550134CD
:10403000A6E78C4200D34EE71F2C00D828E72024A7
:1040400049E701235B429946CA448CE7631E002B73
:1040500015D1119B102B19D0022B00D147E730232B
:104060000E9901240B7069E75D46D5E71F2C00D936
:1040700086E778210E9B1B191970013455E71199B9
:10408000023C1029AED01C000B0045E793060DD56D
:10409000002458210E9B1B191970013445E7930623
:1040A00004D558230E9901240B7040E778230E990C
:1040B00001240B703BE72024F5E6C046F0B54546E9
:1040C000DE4657464E46E0B59BB09846259B249C5D
:1040D0001D00089009910A920C93002200232000F1
:1040E00029000B9402F0EEFC002800D0A7E10B9A07
:1040F0000C9B92469B468023289ADB001A400E9226
:1041000001D1062326938023289A1B011A40564684
:104110005B460D92334300D161E15B465800CC4BC6
:10412000400D9C46604402F0FBFCCA4ACA4B02F0B8
:1041300086FCCA4ACA4B02F05BFC5B46C94A1B03B9
:104140001B0B1A4304000D00C74B11005046002200
:1041500002F045FCC54AC64B02F071FC02000B00A0
:104160002000290002F044FC02F0F2FC814602F03B
:10417000D7FCC04AC04B04000D0002F060FC0022D6
:10418000BE4B02F035FC02F0E3FCBD4A0600BD4B1D
:104190002000290002F053FC040030000D000F96AF
:1041A00002F0BEFCB84AB94B02F049FC02000B0019
:1041B0002000290002F013FC02000B0006000F0093
:1041C00002F03DFC320004000D003B0030003900DD
:1041D00002F00EFC002210901191AD4B200029003E
:1041E00002F00FFC0022AB4B02F002FC02000B00BD
:1041F0002000290002F005FC0022A74B02F0F8FB8A
:1042000002000B002000290002F0FBFB0D008021C2
:10421000040032003B000020C90502F0E0FB020070
:104220000B002000290002F0E3FB02000B001098B5
:10423000119902F0E6FB00228A4B02F0D9FB974A63
:104240000F9B9446634400221B0502F0F8FB050017
:104250000C0002000B005046594602F033FC0028C7
:104260000BD001235B429C46280021000022894B91
:10427000E14402F0C6FB05000C004B46C626633342
:104280009E42B6410D9B76420436002B00D0BCE026
:10429000279B00279E4200D29F1B0223289A1A4088
:1042A0000D9203D0734273415B421F404B46002B7B
:1042B00007D0504659462A00230002F0A2FB82464E
:1042C0008B46002200230B980C9902F0FBFB002880
:1042D00003D08021090659448B4652465B4650461E
:1042E000594602F00AFC002800D044E101226C4B40
:1042F00052425046594602F0E5FB002800D0D7E074
:10430000289A684B039713400493269B52460293C6
:104310005B4609990092019308980A9A434600F077
:10432000FFFC0200002E52D02020289B089C034056
:1043300059424B415B421840531C45309A460999FB
:104340004346A0474B46DA179D18DB0F9946731E6C
:1043500055409B46002412AE02E03C00202F0DD0B9
:1043600028000A2102F0F8F8671C30313419217056
:1043700028000A2102F0F0F8051EEED1052306936D
:104380005B460593002304930A3303934B4601973E
:104390000096099F089E029352464346390030001A
:1043A000FFF754FD0D9B0200002B10D00A99431A11
:1043B000279898420BD989460500434639002020AA
:1043C000541CB0474B462200E31A9D42F5D810001A
:1043D0001BB03CBC90469946A246AB46F0BD0D9B37
:1043E00055465C46002B27D000239946269B4B451B
:1043F00000DDB1E0002326938023289ADB001A43D6
:10440000002328920026994642E723002B43EDD053
:10441000254A264B5046594602F062FB002800D040
:104420009FE0269B002B00D132E70E9B5A1E934142
:10443000269AD31A26932BE70426994628E780224A
:10444000120694460C9BA24663449B4653E6C04624
:1044500001FCFFFFFB799F501344D33FB3C8608B2F
:10446000288AC63F0000F03F0000F83F61436F63B9
:10447000A787D23F71A379094F930A400000E03F1C
:104480001655B5BBB16B0240EF39FAFE422EE63F3E
:1044900000002C400000244000001840FF030000F2
:1044A000FFFFEFFFFFF7FFFF2D431CEBE2361A3F44
:1044B0000A9A289B14009B0715D1042F13D9B246E2
:1044C0004646151FED19BB46099F0B953300390071
:1044D0002020089D541CA8470B9B22009C42F5D12C
:1044E000B0465F4656464D4B49469A464346B94606
:1044F00022000425A346B0461F000B915346013D00
:10450000541C585D09993B00089EB0472200002DBD
:10451000F4D13B005C460B9A464698460D9B4F46AD
:104520009146221D002B00D1FCE60A9BD31A9F4224
:1045300000D8F7E6B3464646BA46099F330039002D
:104540002020089D541CA8470A9B2200E31A9A4584
:10455000F4D8B0465E46E5E64A469B1A013B2693F0
:104560004AE700222E4B5046594602F0ABFA00288B
:1045700000D03BE755E70A9B289A9A46920717D145
:10458000032F15D9B2461A004646DC1EE419BB4675
:10459000099F0B94330039002020089C551CA0472C
:1045A0000B9B2A009D42F5D1B0465F465646AA466F
:1045B0001C4B49469B464346B94652460324B046E7
:1045C0001F000B915B46013C551C185D09993B008F
:1045D000089EB0472A00002CF4D13B000B9A4F46AE
:1045E00091465246464698460D9B0332002B00D119
:1045F00098E60A9BD31A9F4200D893E6B3464646F4
:10460000BA46099F330039002020089D541CA84752
:104610000A9B2200E31A9A45F4D89AE710CB0010BF
:1046200080842E410CCB0010F0B5DE4657464E4636
:104630004546E0B597B005000E0093461F00209A4E
:10464000219B1000190002F058FA002800D0AEE2B9
:10465000209821990122C54B524202F033FA0028DA
:1046600000D034E1209821990122C14B524202F03E
:104670003FFA002800D0C1E0209821990022BD4BCC
:1046800002F036FA002800D008E120982199002293
:10469000B94B02F017FA002800D0FFE020982199CA
:1046A0000022002302F00EFA002800D074E200235A
:1046B0000D938023249ADB001A40904600D0BAE183
:1046C0000023AE4C069307940EAB06249A4620981E
:1046D000219902F03DFA099002F022FA02000B0043
:1046E0002098219902F07BF9069A079B02F0A7F91E
:1046F0000A900B9102F050FA81460C9002F00CFAED
:1047000002000B000A980B9902F069F900229C4BF9
:104710000A900B9102F0ECF9002800D1E5E14B463C
:10472000013318000C9302F0F7F9069A079B02F088
:10473000D7F9002800D0FBE1002C00D09CE1099CB7
:10474000200002F0EDF902000B002098219902F000
:1047500046F900228A4B0690079102F0B3F900282F
:1047600000D1D5E14346202B00D112E15C1C099B0E
:104770000A211800994601F0C7FE424653463031DF
:10478000995448460A2101F0BFFEA0468146002800
:104790001ED05346A846BA464D461F00B14600E01B
:1047A0003400202C00D162E228000A2101F0ACFE86
:1047B000661C30313C19217028000A2101F0A4FE4A
:1047C000051EEDD13B0045465746B0469A464E463B
:1047D0000323249A1340012B00D1B1E14246202447
:1047E000202A00D1DCE00D9A002A00D135E24246B1
:1047F0005146541C40462D220A54D1E0249B5B07AD
:1048000000D5ADE05F4B9A46032398465B4606937E
:10481000249B9B0718D1239B434500D84EE25B4461
:104820001C004346E41AB9465A4637002E002500BC
:10483000541C4B4639002020B0472200AC42F7D12F
:1048400035003E004F460694B14644465646BA46A9
:104850002F00069A013C551C305D53464946B84727
:104860002A00002CF6D1069B3D0043441A00249BED
:104870009B0724D55B462399D31A99421FD92E0052
:10488000D0464F460D00434639002020541CB04707
:104890005B462200E31A9D42F5D810E0249B5A465D
:1048A0000493239B31000393229B28000293209BB7
:1048B000219C009301943B00FFF700FC02001000D4
:1048C00017B03CBC90469946A246AB46F0BD249B2F
:1048D000D8469B0718D1239B042B15D95B461C1F78
:1048E000239BB8469C46644437005A462E00250058
:1048F000541C434639002020B0472200AC42F7D177
:1049000035003E004746A0461F4BB9464246370099
:1049100004249A462E005346013C551C185D39006C
:104920004B46B0472A00002CF5D14246249B350067
:1049300004323E009B07C2D55B462399D31A9942A5
:10494000BDD93700C8462E000D004346390020204F
:10495000541CB0475B462200E31A9D42F5D8AEE7EF
:104960000A4B9A460423984650E7C046FFFFEFFFE4
:10497000FFFFEF7F65CDCD4165CDCDC180842E4158
:104980000000E03F20CB001010CB001018CB00102F
:10499000A2460323249A1340012B00D1CEE0202409
:1049A000D846002B17D1239B9C4214D25B441B1B7F
:1049B000B8465A463700A1462E001D00541C4346F7
:1049C00039002020B0472200AC42F7D135003E002C
:1049D0004746A0464C4643464246A146B8463700A5
:1049E0002E0006935346013C551C185D3900434682
:1049F000B0472A00002CF5D106994B468C466344FB
:104A00001A00249B35003E009B0700D457E75B4605
:104A10002399D31A994200D851E737002E000D0090
:104A2000434639002020541CB0475B462200E31A5D
:104A30009D42F5D843E7229B092B00D85BE10EABE2
:104A40009A4630235246137001229046229B2F3201
:104A50005C1E4146203B504605E0013C425401317A
:104A60009C4200D1EEE0092CF7D10022A84B8846E9
:104A70008246069207932AE64346202B89D0631E7E
:104A8000069301230C9C434420000A21994601F01F
:104A900063FD534642463031995420000A2101F00B
:104AA0005BFD041E00D122E1A84625004C46B94614
:104AB0005746B24612E0069B2800013B0A210693A6
:104AC00001F04AFD661C30313C19217028000A2192
:104AD00001F042FD051E00D1CFE03400202CEAD1C8
:104AE00056464546BA464F4653E700220A980B9968
:104AF000884B01F0E7FF002800D01DE60C9B002B3F
:104B000002D0DB0700D417E60C9B01330C9313E6AD
:104B10000022069807997F4B01F0EAFF002800D099
:104B200020E60123A44623409C446346099319E6EA
:104B3000099B0133099300230C93FDE5202398463C
:104B4000239B002B00D1BFE00D9B002B03D1249AA7
:104B50000C33134202D0239B013B2393239B4345F9
:104B600000D8B1E042463023202A00D1B1E04246CD
:104B700050462399541C83548C4200D1A1E022005A
:104B8000202CF7D1202399465B46B8468246370051
:104B900006935A462E0025E7209A219B00200021EB
:104BA00001F01DFF0123209021910D9381E5249BAD
:104BB000D8469B0718D1239B032B15D95B46DC1ED7
:104BC000239BB8469C46644437005A462E00250075
:104BD000541C434639002020B0472200AC42F7D194
:104BE00035003E004746A0464B4BB946424637008B
:104BF00003249A462E005346013C551C185D39008B
:104C00004B46B0472A00002CF5D14246249B350084
:104C100003323E009B0700D451E65B462399D31A2A
:104C2000994200D84BE63700C8462E000D00434697
:104C300039002020541CB0475B462200E31A9D42F5
:104C4000F5D83CE6354BE2009B181A685B68069283
:104C5000079320238246984639E5249A52073BD58C
:104C600042465146541C40462B220A5498E63B00CB
:104C7000454657464E469A468BE64546B04656460A
:104C8000BA464F464346202B00D182E6069B40465B
:104C90001A004244110054463022002B29D0431CF4
:104CA0002254202B00D173E618008B42F7D1A24684
:104CB0005A1C904651462E22CA5453E55B46069331
:104CC000C2E5239B8246984642460123202A00D013
:104CD00089E52024D8467EE6249A4446120700D46B
:104CE0005EE620225146404601340A5458E6C84642
:104CF000C8E74346DCE7DA00084B9B185C681B6892
:104D000006930794002398460EAB229C9A46DEE455
:104D100065CDCD410000E03F0CCB001028CB00104A
:104D2000F0B557464E464546DE46E0B597B0079289
:104D3000012206000F002098219998465242CF4B3D
:104D400001F0D6FE00284DD0249B5B0700D541E141
:104D5000CB4B9A4603239B46079A249B14009B0740
:104D600011D1239B9B450ED2190013008C4663443E
:104D70001D005B46ED1A541C434639002020B04705
:104D80002200AC42F7D1B946220037005D465646B4
:104D9000A246013D541C705D43464946B847220077
:104DA000002DF6D15246249B3E005A444F469B07A5
:104DB00010D507992398531A98420BD989460500B4
:104DC000434639002020541CB0474B462200E31ACA
:104DD0009D42F5D8100017B03CBC90469946A246BB
:104DE000AB46F0BD002220982199A64B01F080FE31
:104DF000002800D0F3E0209821990022A24B01F076
:104E000061FE002800D0EAE02098219900220023CA
:104E100001F058FE002800D092E100230D93802578
:104E2000249BED001D4000D017E10023974C089310
:104E300009940EAB06249B462098219901F088FE28
:104E400081460C9001F06CFE02000B002098219925
:104E500001F0C5FD089A099B01F0F1FD0A900B9144
:104E600001F09AFE824601F057FE02000B000A98FC
:104E70000B9901F0B4FD0022854B0A900B9101F0D3
:104E800037FE002800D148E101239C46E244504609
:104E900001F042FE089A099B01F022FE002800D092
:104EA0009CE1002C00D006E10C9C200001F038FEB3
:104EB00002000B002098219901F091FD0022744B13
:104EC0000890099101F0FEFD002800D176E1202D27
:104ED00000D1BAE00C9B0A211800994601F014FB9E
:104EE0005B463031595548460A2101F00DFB6C1CD8
:104EF0008146250000281AD04D46BA46B1465F4685
:104F000000E03400202C00D103E128000A2101F048
:104F1000FBFA661C30313C19217028000A2101F08F
:104F2000F3FA051EEDD13500BB464E465746032326
:104F3000249A1340012B00D10EE12024202D0BD008
:104F40000D9A002A00D034E1249A520700D46FE170
:104F50002B2259466C1C4A55079A1500002B12D17A
:104F6000239B9C420FD2190013008C4663441B1BE9
:104F7000A1461C00551C434639002020B0472A009A
:104F8000A542F7D14C46A246A9462A005B46013C01
:104F9000551C185D39004346B0472A00002CF5D156
:104FA0004B4653441A00249B9B0700D412E70799F1
:104FB0002398531A834200D30CE7894605004346E1
:104FC00039002020541CB0474B462200E31A9D4272
:104FD000F5D8FFE62F4B9A4604239B46BCE6209A61
:104FE000219B1000190001F088FD00281AD120989B
:104FF00021990122284B524201F064FD002811D171
:10500000249B079A0493239B39000393229B30002F
:105010000293209B219C009301944346FFF74EF896
:105020000200D7E6249B079A0493239B390003933D
:10503000229B30000293209B219C009301944346C5
:10504000FFF7F2FA0200C5E683460323249A1340D1
:10505000012B00D17FE020247EE7229B092B00D882
:10506000F2E00EAB9B4630235A461370229B01257B
:105070005C1E3022203B594615E0C046FFFFEF7F03
:1050800020CB001065CDCD4165CDCDC180842E41B2
:105090000000E03F18CB0010FFFFEFFF013C4A5536
:1050A00001359C427BD0092CF8D100226C4B8B46F9
:1050B00008920993C0E6202DC7D06B1C50460A21E8
:1050C000994601F049FA5B463031595550460A215C
:1050D00001F042FA013C8246002800D1B2E04B4682
:1050E0005546B146BA465F4611E09B4628000A2164
:1050F0005E1CBB4401F030FA5B4630311970280069
:105100000A2101F029FA013C051E76D03300202B3C
:10511000EBD1BB464E46574697E700220A980B99BB
:10512000504B01F0CFFC002800D0BAE65346002BCC
:1051300002D0DB0700D4B4E601239C46E244B0E68B
:10514000209A219B0020002101F049FC012320909E
:1051500021910D9363E62025239B002B46D00D9BC8
:10516000002B03D1249A0C33134202D0239B013B22
:105170002393239BAB4239D93023202D3AD0594673
:10518000239A6C1C4B5594422ED02500202CF8D12C
:105190002023079D8B469A46A9462A00F6E6324B05
:1051A000E2009B181A685B688B46089209932025D9
:1051B00042E62D2259466C1C4A55CDE6002208983D
:1051C0000999284B01F094FC002800D07FE60123C8
:1051D000A44623409C4463460C9378E64B46013337
:1051E0000C9300239A465CE68B46239D0123202DD9
:1051F00000D0A5E62024079DC5E63500BB464E46F7
:105200005746202D00D120E7611930222B00002CB9
:1052100009D058466B1C4255202B00D114E71D00C5
:105220008B42F7D183462E2259465D1CCA544EE666
:10523000249A2C00120700D48EE62022594601340D
:105240004A5589E64D46DCE7DA00074B00259B18F6
:105250005C681B68089309940EAB229C9B46EBE5A7
:1052600065CDCD410000E03F28CB0010F0B5DE4613
:1052700057464E464546E0B5A9B01E00329B9046C3
:105280000A93BF4ABF4B83468A461A60002968D0FA
:10529000D1460025DA46307800280BD00136252883
:1052A0001BD02A0043464946D04730786C1C250065
:1052B0000028F3D1D3462A00CA46454501D34346C8
:1052C0005A1E434651460020D847280029B03CBC0E
:1052D00090469946A246AB46F0BD102330789B46D7
:1052E0000E3B9C460300203B721CDBB20027A64C01
:1052F0001100102B0DD89B00E3589F460123160088
:105300001F433078721C0300203BDBB21100102BCE
:10531000F1D90300303B092B00D8AEE100239B46B6
:105320002A2800D1CFE100242E2800D1BDE10300BE
:10533000683BDBB2122B00D9D3E3944A9B00D358CD
:105340009F46042316001F43DBE7634616001F43F6
:10535000D7E75B4616001F43D3E7082316001F4319
:10536000CFE78B4B9B4693E780235B0070781F430E
:105370004E1C0300253BDBB2532B92D8854A9B0081
:10538000D3589F4670786C2801D100F0C0FC802370
:105390005B001F434E1CECE780239B0070781F438B
:1053A0004E1CE6E77078682801D100F019FD8023D3
:1053B0004E1C1F43DDE7462801D100F058FC0722B0
:1053C0000A9B049707339343013294469C446246F8
:1053D0000A925A46029403925C681B682A00009362
:1053E0000194494643465046FFF71EF9050052E72F
:1053F0002A006C1C434649462520D04725004AE731
:105400000A9B1A1D1B680C920A931878002C00D076
:10541000ABE3002801D100F0A2FF02211A004942AB
:1054200001239C46434608900B9307E00A98634685
:1054300080469B1A43445B18002B03D0013213783B
:10544000002BF3D10B9B089898460A9BD31A08931C
:105450008023DB003B400B9303D0089BA34200D981
:10546000089402231F4001D100F0DBFC002801D189
:1054700000F0BCFC0B9B002B01D000F062FE0A9BED
:105480002A005C1B23005446B2464E46B9464746A6
:1054900098463B003100551CA0474346585D2A0002
:1054A0000028F6D1B8464F46B1465646A246002FD0
:1054B00001D000F09BFC0C9B0A93ECE60A9B1A1DA2
:1054C0001B689346002B00D142E3212217430A9721
:1054D0000F2020A90B940022089184460C0002E0C2
:1054E00020290CD00A0061461940CFB2380037306D
:1054F000092900D80738511CA0541B09F0D10B9C76
:105500000A9B019106930823059308330393002314
:105510000293089B2A000093049443464946504650
:10552000FEF794FC5B4605000A93B4E60A9B6C1CEC
:1055300004330B940893BB0700D478E30A9B2A003A
:10554000187849464346D0475B465D44012B01D855
:1055500000F07EFE2B0057464D46B1464646984623
:105560000B9A541C330029002020B84722004445E0
:10557000F7D1B046BA464E46A946250073E3C04669
:105580006D5200102C2800202CC9001070C900108A
:105590002D3E0010BCC90010782800D1ECE258283C
:1055A00001D100F067FC6F2801D100F051FD6228A5
:1055B00001D100F04FFE10233A009A430B92692864
:1055C00001D000F039FF7B0501D500F02BFD8023D1
:1055D0009B001F40F73BFF3B0C93002F01D000F0D6
:1055E000C3FC80230B9A5B001A40130094460A9A6E
:1055F00004320D92002B01D000F0CAFD0B9B5B061C
:1056000001D400F0BCFD0A9B1B78DA1798185040B3
:10561000DA0F0A92002B08D10B9A1033110099432C
:105620000B91520501D500F0A2FE0B9B61279B0652
:1056300000D541275A4620ABFFB20E950F94B346D2
:1056400008930A3F644610920C9D1E000CE0303314
:10565000DBB2621C3355002801D100F017FC202A70
:1056600001D100F013FC1400290000F075FFCBB24B
:105670000929ECD9DB19DBB2EBE70023010001E0DB
:10568000160001329800C01840004018117803003D
:1056900008003038303B0928F2D908009B46B11C7D
:1056A000002416002E2800D041E680237078DB000D
:1056B0001F430300303B092B15D92A2800D1DAE219
:1056C0000E00013133E60A990B1D09688B4600294B
:1056D00004DA02210F43594649428B467078B11CC7
:1056E0000A9316001FE6030000E03100A000001935
:1056F0004000C0184B7830381A00303A4E1C040075
:10570000092AF2D91800023111E6202302009A4337
:10571000472A02D180231B011F43022398434528B7
:1057200001D11E331F4307220A9B073393430132E3
:1057300094469C44624619685868089109900A92F8
:1057400003000A000B910C900898099901F0D5F913
:10575000002800D09BE20122E34B52420B980C99A7
:1057600001F0C6F90122E14B5242002800D0D5E2F7
:105770000B980C9901F0A6F9002800D0A2E30022B2
:1057800000230B980C9901F09DF9002801D000F03E
:1057900055FD0B9A0C9B08920D938023DB003B4038
:1057A000179300D1062480230D9A1B013B400E93D2
:1057B000130008990F910B4301D100F0B6FCCC4BBC
:1057C00050009C46400D604401F0AAF9C94ACA4BFA
:1057D00001F035F9C94ACA4B01F00AF90D9A109047
:1057E00011911303C74A0F991B0B1A431B921A916D
:1057F00000221A981B99C44B01F0F1F8C34AC44B1C
:1058000001F01DF902000B001098119901F0F0F859
:1058100001F09EF90F9001F083F9BE4ABE4B109043
:10582000119101F00CF90022BC4B01F0E1F801F0FC
:105830008FF9BB4ABB4B16901098119901F0FFF8F5
:1058400010901191169801F06BF9B74AB74B01F01F
:10585000F6F802000B001098119901F0C0F8020050
:105860000B001090119101F0EAF814901591109826
:10587000119902000B0001F0BBF800221E901F914D
:1058800014981599AA4B01F0BCF80022A94B01F01D
:10589000AFF802000B001498159901F0B2F800223D
:1058A000A54B01F0A5F802000B001498159901F022
:1058B000A8F8109A119B1490159180210020C90519
:1058C00001F08DF802000B001498159901F090F882
:1058D00002000B001E981F9901F093F80022894BDB
:1058E00001F086F8169B1A00944B9C4662441305FF
:1058F0001D9300231C931C9A1D9B01F0A0F814908B
:10590000020016910B0008980D9901F0DBF80028B1
:105910000AD00F9B1498013B0F9316990022854BD8
:1059200001F06FF814901691C6230F9A63329342D8
:105930009B415B42043310930E9B002B1DD0169BA2
:10594000149A134301D100F0C1FC7D4A7D4B0898A5
:105950000D9901F0C5F8002809D000227A4B08986B
:105960000D9901F0AFF8002801D000F0AFFC002C39
:1059700003D0179B5A1E9341E41A00230E93109BE9
:105980009B4502D95A46D31A0E9302233B401793E4
:1059900006D0109B5A4253410E9A5B421A400E9217
:1059A0000F9B002B07D008980D99149A169B01F0B5
:1059B00028F808900D91002200230B980C9901F013
:1059C00081F8002805D08020000684460D996144A6
:1059D0000D910D99089A0B00089801F08EF8002897
:1059E00001D000F0E2FC0122404B524208980D9990
:1059F00001F068F8002801D000F075FC534B089ABC
:105A00003B4004930E9B029403930D9B49460092E6
:105A1000019350462A004346FFF782F90200109B8B
:105A2000002B00D170E1202007403B0059424B4140
:105A300000275B42511C18400B91434649464530B4
:105A4000D0470F9A109BD117013B54180D93D20FDA
:105A500020AB0E954C403D000C9208930F961F0012
:105A600002E03500202E0DD020000A2100F074FD48
:105A70006E1C30317D19297020000A2100F06CFD68
:105A8000041EEED1052306930D9B320005930023DF
:105A900004930A3303930C9B01920293089B0B9A85
:105AA00000934946434650460E9D0F9EFEF7CEF9A1
:105AB000179B0200002B00D126E1431B9B4500D819
:105AC00022E15C465746531C9A46494643462020ED
:105AD000B8475246531B9C42F5D8BA461500FFF70B
:105AE000DAFB0E0045E4C046FFFFEF7FFFFFEFFF4C
:105AF00001FCFFFFFB799F501344D33FB3C8608B79
:105B0000288AC63F0000F03F0000F83F61436F6302
:105B1000A787D23F71A379094F930A400000E03F65
:105B20001655B5BBB16B0240EF39FAFE422EE63F87
:105B300000002C400000244000001840FF0300003B
:105B40002D431CEBE2361A3F80842E41FFF7FFFF06
:105B5000102239009143113211430A917A0500D481
:105B6000B6E420AB00210893CAE4002801D100F07C
:105B7000F6FB611E1A0053E480231022DB003B4039
:105B80000C920C2297430B973A00002B02D0012372
:105B90009A430B9280270B9BBF001F40692800D1BE
:105BA0001BE5642800D118E5002F00D07CE280239B
:105BB0000B9A5B001A40130094460A9A04320D9225
:105BC000002B00D050E30B9B5B0600D445E30A9BFF
:105BD0001878002807D10B9A1023110099430B91D4
:105BE000520500D5BFE30B9B61279B0600D54127DB
:105BF00020ABFFB20A950E940F9608930A3F6546B4
:105C00000C9C1E000AE03033DBB26A1C735500287E
:105C100000D111E2202A00D10EE21500210000F08F
:105C20009BFCCBB20929EED9DB19DBB2EDE75B4671
:105C3000012B00D8A7E36B1E9B4433005E469B46B6
:105C400001E02500013443462A0049462020270070
:105C5000D047B442F5D15E4602350A9B3A00187827
:105C600049464346D047089B0A93FFF714FB20237D
:105C70001F43FFF7A4FB0A9AB0781468F11CE343B2
:105C8000DB171C40131D0A930236FFF750FB2C0054
:105C9000BB0710D15B46032B0DD9EC1E23002A0055
:105CA0005B440893434649462020541CD047089B38
:105CB00022009C42F6D103230893DC4B22000B9375
:105CC0002B003D001F00089B0B98511C013B0C91C1
:105CD0000893C05C49464346D047089B0C9A002B6A
:105CE000F2D13B002F00E21C1D00BB070CD5531B5B
:105CF0009B4509D95F46541C434649462020D0475E
:105D00002200631B9F42F6D81500FFF7C4FAC02398
:105D10009B00B0781F430336FFF72BFB0B980C99C1
:105D200000F0D0FE002800D0CCE07B0700D46BE26E
:105D3000BF4B089304230C930B95BB071CD10C9B02
:105D40009B4500D82DE35A465419E41A33002A0023
:105D50004E46A94655469A460D97571C4346310074
:105D60002020A8473A00BC42F7D15346AA464D46E8
:105D7000B1461E000B970D9F330056469A460B9A6C
:105D80000C9C0D95089B013C551C185D49464346EB
:105D9000B0472A00002CF5D153460B99B2468C46E9
:105DA0001E000C9B0D9D63441A00BB07ACD5531B12
:105DB0009B45A9D933005C464E4657469946531C2D
:105DC0009A46310043462020B8475246531B9C4216
:105DD000F5D84B46BA46B14615001E00FFF75BFAF0
:105DE000C023B0781F430336FFF7C3FA089B9B45D7
:105DF00001D8FFF760FB5A465419E41A33002A0011
:105E00004E46574699460135434631002020B84753
:105E10002A00A542F7D14B46BA46B1461E00FFF70D
:105E20004AFB089A531C934500D8A8E25B465B19CD
:105E30009B1A08971F0033002A004E46A14654467D
:105E40009A460135434631002020A0472A00BD4232
:105E5000F7D15346A2464C46B1461E005B4601337D
:105E6000089F08930A9B1878002801D0FFF702FBCF
:105E7000FFF721FB0C233A009A4314331A430B9289
:105E80007B0500D4C7E010230C9380E6109B5E4690
:105E90009B460E9D0F9C0B9B049406935B460593BB
:105EA0000C9B03930A9B0293089B019200932A0088
:105EB000434649465046FDF7C9FF0D9B05000A932E
:105EC000FFF7E9F90B95BB071BD15B46042B00D804
:105ED000B0E233002C1F2A004E46A94655469A468A
:105EE0005C440897571C434631002020A8473A00DD
:105EF000A742F7D15346AA464D46B1461E000B971E
:105F0000089F4C4B0424089333004E46B94657462D
:105F10009A460B9A0C95089B013C551C185D310064
:105F20004346B8472A00002CF5D15346BA464F469F
:105F30000B9AB1460C9D1E000432BB0700D4E3E669
:105F4000531B9B4500D8DFE633005C464E46574660
:105F50009946531C9A46310043462020B847524682
:105F6000531B9C42F5D834E707220A9B073393431F
:105F7000013294469C4462465F680A921A68FB1795
:105F800018931993189819990300534012930B0012
:105F90007B4013939446129A139B121A8B411292D0
:105FA00013936246FB0F14933A4307D10B9A1023C5
:105FB000110099430B91520500D5E7E10B9A61233B
:105FC000920600D54123DBB220AA0A3B0E950F941E
:105FD00010960027129C139D08920D930C9E0CE0C6
:105FE0003032D2B2089C7B1CE255020004000D0046
:105FF0000A433FD0202B3DD01F0032000023200059
:10600000290000F0EBFAD2B2092AE9D90D9B9C468F
:106010006244D2B2E6E780239B001F40F13BFF3B86
:106020000C93C1E50A230C93B1E5C0460CCB0010DC
:1060300018CB001010CB00100A9D0E9C0F9E0B9BDE
:10604000049406935B4605930C9B039300232AE775
:1060500008230C938023DB003B40642800D090E5AC
:106060003A000B97002B00D091E58027BF00174026
:10607000FFF7B3FA12941395109E0F9C0E9D0B9A86
:10608000049406925A4605920C9A01930392149A2C
:106090000292089B2A000093494643465046FDF76A
:1060A000D5FE0500FFF7F7F807220A9B0733934355
:1060B000013294469C44624603CB03000A920B4390
:1060C00007D10B9A103317009F430B97520500D549
:1060D00063E10B9A6123920600D54123DBB220AA2B
:1060E0000A3B0E950F94002708920D930C9C109676
:1060F00015000CE03032D1B2E95518007A1C31009D
:10610000334300D185E0202A00D182E0170022002D
:10611000002300F063FAD2B203000E00092AE9D985
:106120000D998C466244D1B2E6E70E9B002B00D05D
:10613000C7E00D9B149116930423109300230F9333
:106140001BE40A9B64195B1B0A9333002A004E462A
:10615000B94657469A4608E043463100551CB847B1
:106160000A9B585D002862D02A00A242F4D153460F
:106170001500BA464F46B1461E00FFF798F90B9B33
:106180001B0600D4F7E00A9B00229B5EFFF73DFA56
:106190000A9B1B68DA1798185040DA0F0E92002BF2
:1061A00006D10B9A1033110099430B9152051FD45D
:1061B0000B9A6123920600D54123DBB220AA0A3B49
:1061C00008920A9309E03033DBB208997A1CCB5568
:1061D000002810D0202A0ED017000C9900F0BCF92E
:1061E000CBB20929EFD90A9A94466344DBB2ECE7B3
:1061F000002220AB08930B9B049406935B46059307
:106200000C9B03930E9B4EE68D4B089303230C933C
:1062100092E50E9D0F9C109E0B9B049406935B468B
:1062200005930C9B019203930023029331E753469D
:10623000BA464F46B1461E00FFF739F980221206D2
:1062400094460B9B08930C9B63440D93FFF7A5FAB0
:10625000250008E502230C93FCE60B9B1B0600D4EB
:1062600098E00A9B1888B4E40A9B1868002806D1B5
:106270000B9A1023110099430B91520573D40B9A7A
:106280006123920600D54123DBB220AA0A3B089283
:106290000A930BE03033DBB208997A1CCB55002807
:1062A00000D1CCE6202A00D1C9E617000C9900F0F5
:1062B00053F9CBB20929EDD90A9A94466344DBB26B
:1062C000EAE70D9B1491169300230F930F9B9C42BA
:1062D00057DDE41A013C8023DB001F4300231093A9
:1062E0000F93FFF74AFB0B95BB070FD10E9B042BB7
:1062F00059D99C462A002C1F6444531C0B934946D1
:1063000043462020D0470B9A9442F6D104244D4BAB
:106310000B9A08930C97089B013C571C185D494643
:106320004346D0473A00002CF5D10B9A179B0C9F9F
:106330000432002B01D1FFF772FB0E99531B8B42E5
:1063400001D3FFF76CFB434649462020541CD0473D
:106350000E992200631B8B42F5D3FFF760FB0023ED
:106360000893FFF775F820AB0022089367E620AB8F
:10637000002208938FE50A9B1B68FFF746F90893F4
:1063800072E50024A7E72F00250066E420AA002379
:10639000089274E60A9B18681BE420AB002208935D
:1063A0003AE70B95E8E40B95B0E72C00BB0710D15A
:1063B0000E9B032B0DD99C462A00EC1E64440894C6
:1063C000434649462020541CD047089B2200A34244
:1063D000F6D1032308931C4B22000B932B003D00A6
:1063E0001F00089B0B98511C013B0C910893C05C4B
:1063F00049464346D047089B0C9A002BF2D13B00FC
:106400002F001D00179BE21C002B01D1FFF707FB9B
:106410000E99531B8B4201D3FFF701FB43464946BC
:106420002020541CD0470E992200631B8B42F5D3C9
:10643000FFF7F5FA0B9564E5063B17000C9309E6A8
:1064400020CB001010CB00100CCB001000B585B095
:106450000391012102900093034813004A4202A9CC
:10646000FEF704FF05B000BD313E001010B5094A2B
:1064700084B01468002C09D001220091030052421C
:1064800003A90548A047012004B010BD01F004F89D
:106490000020F9E72C280020413E0010014804218B
:1064A000014B184790140020CD640010142310B540
:1064B0000100188804331B88984710BD162310B5B7
:1064C0000100188802331B88984710BDF0B5C646F6
:1064D00000B5002916D0142304000125984618277A
:1064E000890046184346216818883B88984701C4AC
:1064F000431E984140420540A642F3D1280004BC07
:106500009046F0BD0125F9E7124A936F9B0815D21A
:106510009066D166002905D0FFE7FFE7FFE7516FDE
:10652000106F704704B580210906C217514000283A
:1065300000D0C84306F038F8002104BDF0B5146E51
:10654000556E576F166FFFF7E3FF14665566576772
:106550001667F0BD000000D0114A936F9B0813D25C
:1065600010665166002905D0FFE7FFE7FFE7516F8E
:10657000106F704704B5002801D00020C04306F01A
:1065800013F8002104BDC046F0B5146E556E576F68
:10659000166FFFF7E5FF1466556657671667F0BD7F
:1065A000000000D094464E4A926F9208624601D293
:1065B00030E0C046F0B54A4EB56F6D08FCD3346E7E
:1065C000756E776F366F00F025F89446444A14666E
:1065D0005566576716676246F0BDC0469446404A06
:1065E000926F9208624601D258E0C046F0B53C4E28
:1065F000B56F6D08FCD3346E756E776F366F00F033
:106600004DF89446364A14665566576716676246D3
:10661000F0BDC046002B24DB11D000293EDA00B5C6
:10662000C943404200D1013100F038F8C94340422B
:1066300000D10131DB43524200D1013300BD002AB9
:10664000EBD1002801D1002905D00020C90FC907CE
:1066500001D1C043410800B505F09EFF0022002390
:1066600000BD00B500290ADBDB43524200D10133F3
:1066700000F014F8C943404200D1013100BDC943C4
:10668000404200D10131DB43524200D1013300F0DE
:1066900005F8DB43524200D1013300BD002923D16C
:1066A000002B18D1002A0CD0BC460D4F38667A66F4
:1066B00000210023FFE7FFE7FFE77A6F386F6746A7
:1066C0007047002801D00748010000B505F064FFBD
:1066D0000022002300BD02000B00002000217047B3
:1066E000000000D0FFFFFFFF002B00D0BFE0130C25
:1066F00028D1002AE7D080B4114F39667A66FFE7C7
:10670000FFE730B4040C7B6F396F1B0423433B66F7
:106710007A66FFE7FFE7FFE7C04684B27B6F3D6F15
:106720001B0423433B667A66FFE7FFE7C04600236E
:106730002C042D0C7A6F386F00196941B0BC70477A
:10674000000000D0F0B594460025140E01D11202CD
:106750000835140F01D112010435940F01D19200B4
:106760000235D40F01D152000135D40B0134254F2D
:106770007C66254C3C660E0C93B2FFE7FFE7FFE713
:106780003C6F6643360C7703BE467343DF0B5B04F6
:10679000C01AB941130C7343DB18C91ACE086643FB
:1067A000360CB64493B273431F0F1B01C01AB94194
:1067B000130C73431F0B1B05C01AB941860D8F02C2
:1067C0003E436643360C092D24DB520A7243801A7D
:1067D0007703460A6643360C16235B1BDE40DF4018
:1067E000BF1964466643821B7046043506330100B8
:1067F000D940A840C01900D30131A24206D20023DB
:10680000F0BD0000000000D0FFFFFFFF121B0130B1
:10681000F3D3F1E709277F1BFE406446A2B272431F
:10682000801A00D20139220C7243130C1204821A0E
:1068300099410B007046043513370100F940A84018
:10684000801900D30131002B02D1A2420AD2F0BD3F
:10685000013000D30131121BFAD2013BF8D1A24220
:1068600000D2F0BD013000D30131121BF7E7F0B5C3
:106870001C0C00D080E00CB400251C0A04D11B02C3
:10688000160E3343120208351C0B04D11B01160FE0
:106890003343120104359C0B04D19B00960F334304
:1068A00092000235DC0B02D192185B4101351C00CD
:1068B000971864410134464F7C66464C3C660E0C8A
:1068C000FFE7FFE7FFE7C0463C6F6643360C770300
:1068D000BE4697B27743C01B00D20139C01B00D21D
:1068E00001399FB27743C91BC91B170C77437E043C
:1068F000FF0B801BB941CE086643360C0C2D33DBF1
:10690000B644120B1F053A431B0B97B27743C01BCB
:1069100000D201399FB27743C91B170C77433E045D
:106920003F0C801BB941860D8F023E4366432927E9
:106930007F1BFE400C3D7746AF40BF1930BCA2B272
:10694000ABB272437343801A9941220C7243130C09
:106950001204801A994102000B000137001BA94163
:10696000F9D2781E0021F0BD0C277F1BFE40774630
:106970007F0BAF40FF19E0E700245D1C07D0144FE8
:106980007D663966FFE7FFE7FFE7FFE73C6F95B2FB
:106990009EB265436643401BB141150C1E0C654316
:1069A000664336042F0C3E432D04401BB1419942EF
:1069B00004D202000B0020000021F0BD01D1904262
:1069C000F7D3801A994101349942F2D3F6E70000D7
:1069D000000000D0FFFFFFFF48404140484018B48E
:1069E0001B4B5B68FC46019308BD04DF436C001041
:1069F00018B4174B1B68FC46019308BD00DF4D6CB3
:106A000000109446134A926F920809D2624618B455
:106A10000F4BDB68FC46019308BD0CDF056F0010CF
:106A20000C4AF0B5146E556E576F166F6246FFF73D
:106A3000EEFF084A1466556657671667F0BD18B42E
:106A4000034B9B68FC46019308BD08DFA96D00104D
:106A50008C2A0020000000D0FFB55040424050403A
:106A600059404B40594000E0FFB5154F4C00640DB4
:106A700003D0BC4204D10C0314D80020090D090531
:106A80005C00640D03D0BC4204D11C030AD8002270
:106A90001B0D1B0501264B4009D44B4003D58B42EF
:106AA00000D18242FFBD9942FCD19042FFBD0B4311
:106AB000DB1803431343F5D0C9434918FFBD000059
:106AC000FF07000000B5FFF7CFFF804100BDC046C3
:106AD00000B5FFF7C9FF01D9002000BD012000BDAE
:106AE00000B5FFF7B9FF01D9002000BD012000BDAE
:106AF00000B5FFF7B1FF804100BD012040054A000D
:106B0000121804D85A00121801D80020704701202A
:106B100070470020704700000021002805D1704711
:106B2000C1174840401AFAD0C90713B5064B1B6875
:106B300098470CBC441CA2401005120B0349091BCA
:106B400009051943114310BD502900201F040000FE
:106B500010B54C00620D8023D218DB00D21A5B0501
:106B60007E2A10DD9E3A13DACC170903490819432F
:106B70005242D140640001341532202A05DAD04057
:106B80000843604310BD002010BD0846604310BD9F
:106B9000C80FC018013810BD18B4044B5B6AFC461E
:106BA000019308BD24DFB570001000008C2A00207E
:106BB000132370B51C78012C11D01ADD0F48FFF794
:106BC0007DFC0F4D01008022280000F043FB022CC9
:106BD00010D00C48FFF76AFC0B4B186070BD084DD5
:106BE0000A4A29002B00803104C38B42FCD1AA64DD
:106BF000EFE7034D054AAA64EBE7C04653440000A3
:106C00008C2A00204C33000050290020116C001009
:106C100007B5604601880A0A0230DF2AFAD1C9B2F4
:106C2000820804D3028840880004104300E0006812
:106C3000014A5050039007BD8C2A00200FB403BCBA
:106C40000CBCF0B50124E407634000E0F0B50C0D86
:106C5000CF0F661E3605891B640503D3C943404226
:106C600000D30131640D03D0661CF60A07D0E41B83
:106C700000207F00791C89078912803C24031D0DA8
:106C8000DF0F6E1E36059B1B6D0503D3DB4352429F
:106C900000D301336D0D03D06E1CF60A07D0ED1B37
:106CA00000227F007B1C9B079B12803D2D032F1B26
:106CB000661B58D4A446202E46DA20371400BC4068
:106CC0001D00BD40F24033412A4380185941CB0F8B
:106CD00005D0C943C043002264425041514162463D
:106CE0004D0D28D10D0D07D100281FD0241940418A
:106CF0004941013A0D0DF9D0640006D3013000D3AB
:106D00000131002C01D140084000013A0BD4941C01
:106D1000E40A04D112051144DB071944F0BDD90778
:106D2000204B194300E0D9070020F0BD0029DDD138
:106D3000002CDBD1F0BD0132C6074008CD07284347
:106D40004908002EE1D0D9E73C2E29DA203E403711
:106D50001400BC4000D00124F24014431A00BB4090
:106D60001C43D317ACE7AC46202F08DA20360400CA
:106D7000B4400D00B540F84039412843A5E73C2F09
:106D80000CDA203F40360400B44000D00124F84023
:106D900004430800B1400C43C117EAE71000190092
:106DA000002494E70000F07FF0B50C0D661E360558
:106DB000891BE60A6405640D02D0651CED0A04D047
:106DC000002001210905803C2403A4461C0D671EF8
:106DD0003F05DB1BE70A6405640D02D0651CED0A64
:106DE00004D0002201231B05803C24037740644427
:106DF00097B484B296B27443070C7E43150C6F436C
:106E000080B26843361802D3012000043F183004D2
:106E1000350C00197D41844688B29AB250430C0C5F
:106E200062431F0C7C438EB27E43921902D301262B
:106E30003604A4191604170C3618674101BC81B238
:106E40009AB25143040C62431B0C5C4380B258431A
:106E5000121802D30120000424181004130C401847
:106E600063412D185E410020474106BC88B293B2B1
:106E700058430C0C6343120C544389B251435B18C2
:106E800002D301210904641819041A0C091862417B
:106E90006D1856410020474118BCF902720D11438C
:106EA000F0026A0D1043ED020A0D03D16D19404145
:106EB0004941013B124E9B1B7600B3420ED26D003E
:106EC00007D30130002671416646354301D14008A1
:106ED00040001B05C918E4072144F0BD0BDA01335B
:106EE00006D1013004D101314F0D01D04908F2E73C
:106EF000E1070020F0BD013631050020EBE700007E
:106F0000FF030000F0B51C0D671E3F05DB1BE70A01
:106F10006405640D02D0661CF60A04D00022012329
:106F20001B05803C2403D0252D060026F6432E6643
:106F30001E096E66CE0FF619B44649004F0D02D0F9
:106F40007E1CF60A03D000200021403F3F033E1B79
:106F5000B600B444013F7F05C91B49082E6F0136B6
:106F600076089C02950D25437543ED137543AD13CB
:106F700001356D10F603761B0CB4CC02450D2C4385
:106F8000A2B2B3B25A43270C7B43350C6F43A4B271
:106F90006C431B1902D3012424043F191C041D0C4B
:106FA000A4187D4124196D41009A91B2ACB261439D
:106FB000170C7C432B0C5F4392B25A43A41802D3A4
:106FC00001221204BF182204230C52187B41019C99
:106FD0006C431B19520ED9010A434401A01A81B215
:106FE000B2B2514303145A43360C734387B277430A
:106FF000D617D21900277E4136049B191704160CA8
:107000007F185E417316ED18F30100268033754139
:10701000A90F06D16400690AE8055B0A184309D282
:107020002FE00422944480337541A90AA8059B0AE5
:10703000184326D3404149412404009A019B0D0086
:107040005543641B4343E41A95B286B27543170C4B
:107050007E43030C5F4392B25A43B61802D3012217
:107060001204BF183204330C52197B4152429C4126
:10707000002C02D40022013051414008CA071043BD
:10708000490802B06246D7079210084BD218084B45
:107090009A4203D212058918C919F0BD0020002AAE
:1070A00001DC3900F0BD01331905F5E7FD030000EF
:1070B000FE070000002200B5203200F004F80800AE
:1070C00000BD000000220B150AD410B5944600F054
:1070D00031F81414013400DA0021CB17144C204786
:1070E0000020002170476244343A0CD40C2A07DA9D
:1070F00004009140904052422032D440214310BDC0
:10710000D843D94310BD203207D40C469440524294
:1071100020321141D040204310BD0800C917203251
:1071200003D452422032104110BD1800190010BD86
:10713000E77000100A0DCC0F531E1B05C91A52052B
:1071400003D3C943404200D30131520D03D0531C35
:10715000DB0A07D0121B00206400611C890789121A
:10716000803A1203014BD21A70470000FF0300005F
:1071700051434343C9188C46110C83B24B4310B49E
:10718000040C614392B280B2504362431C041B0C56
:10719000001910BC59411304120CC018514161442C
:1071A00070470000132310B51C781348FFF786F9C9
:1071B000012C0BD004DD01008022104800F04AF8B9
:1071C0000F48FFF773F90F4B186010BD0B4C01000F
:1071D0005422200000F03EF80B4B6365A365E36585
:1071E00023666366A366E36623676367A367E36753
:1071F0002362E361E4E7C046534600008C2B002085
:107200004C330000502900200D72001007B5604675
:1072100001880A0A0230DF2AFAD1C9B2820804D3EF
:10722000028840880004104300E00068014A505082
:10723000039007BD8C2B002001480421014B184707
:10724000A0140020CD640010014B1B6818470000FB
:10725000A0140020014B5B6818470000A014002018
:10726000F0B5C64600B5437C06000C001500002BA7
:1072700006D1036811002000984704BC9046F0BD79
:10728000002AFADD0A78037C00200A2A2CD001218A
:10729000012D1BD0184B984602E03900BD4215D095
:1072A0004B1EE25C635C4F1C0A2BF6D10D2AF4D016
:1072B0003368884203DA091A201898473368022194
:1072C0004046984738003900BD42E9D1854203DD88
:1072D000291A3368201898476419013C23780D3B1C
:1072E0005A4253413374C8E7002BD0D102480221DF
:1072F000336898470120CAE7D8CB0010F0B54F4655
:10730000D6464646314BC0B51C680700002C1BD042
:107310002F4B98462F4B9A4602E0E468002C13D07E
:107320002368002BF9D042461268002A01D0A242FD
:10733000F3D1627C3D1D3E68002A0CD1310028004B
:107340009847E468002CEBD100233B601CBC9046BE
:107350009946A246F0BD002EDFDD3979227C00205F
:107360000A292BD00121012E03D119E049464E45AF
:1073700016D04B1EEA5C4B1C99466B5C0A2BF5D170
:107380000D2AF3D02368814203DD091A2818984793
:107390002368022150469847484649464E45E8D161
:1073A000864203DD311A236828189847AD19013D3C
:1073B0002B780D3B5A4253412374AEE7002AD1D1BA
:1073C0000448083998470120CCE7C0462024002013
:1073D00024240020D8CB00100B6870B505000C00E9
:1073E000802B04D05A1C2260E418257170BD08005F
:1073F000FFF784FF2368F5E7F0B5CE46474680B532
:1074000083B06B46DD1CD02328701B061C681F4B05
:10741000804601A91800994605F0CEF8071E2DD127
:10742000019B64B29C4224D0484605F0E5F8184B15
:1074300001271C68002C25D0164E07E001222900E8
:107440002000FFF70DFFE468002C0AD02368002B12
:10745000F9D03368002BF1D0A342EFD0E468002CC0
:10746000F4D1002F0ED1404603B00CBC9046994693
:10747000F0BD074B1C68002CDED1F4E7044B1C6800
:10748000002CD9D1484605F07FF8ECE7301D0020EC
:107490002024002024240020F0B5DE4657464E4626
:1074A0004546E0B583B0070004F0E8FED02301AD07
:1074B0001B06060029002F481C6805F07DF882464F
:1074C000002849D1019B64B29C423FD0294805F075
:1074D00093F8294B9B461C6801239A46002C40D008
:1074E000264B98460A2399460EE0320039002000C8
:1074F000FFF7B6FE4B460122290020002B70FFF754
:10750000AFFEE468002C0BD02368002BF9D0434673
:107510001B68002BE9D0A342E7D0E468002CF3D12C
:107520005346002B1DD15B461C68002C06D06368B7
:10753000002B1AD09847E468002CF8D1300003B033
:107540003CBC90469946A246AB46F0BD0A4B1C682F
:107550009B46002CC4D1F1E7074B1C689B46002CCE
:10756000BED1044805F010F8DDE7E468002CDED158
:10757000E4E7C046301D0020202400202424002001
:107580000D4B1A68002A12D0824203D109E09842BA
:1075900007D01A00D368002BF9D1002900D0D060A1
:1075A00070470029FCD1C368D360C160F8E70029A7
:1075B000F6D01860F4E7C04620240020F0B5C64697
:1075C000D02300B51F4EA2B01B060700884630002E
:1075D00001A91C6804F0F0FF051E07D1019B64B2ED
:1075E0009C4203D0300005F007F8013584220021C9
:1075F00001A8FFF729FE43463A0001A91248FEF709
:1076000025FF019B0700002B18D1104B1C68002C94
:1076100006D06368002B0DD09847E468002CF8D1A1
:10762000002D02D0300004F0AFFF380022B004BCBF
:107630009046F0BDE468002CEBD1F1E701A8FFF71C
:107640005DFEE2E7301D0020D973001020240020E9
:107650000FB400B583B004A901C90191FFF7AEFFD3
:1076600003B008BC04B0184710B500F035F910BDE0
:107670007047C0460022014B1A707047872A0020CD
:10768000012070474B790020FF2B00D070478B7989
:10769000002BFBD1CB79012BF8D1082AF6D98A78B7
:1076A000014B09301A70F1E7872A002070B50029D4
:1076B00015D115495379107909781B02034300202D
:1076C000994200D070BD5378012B0AD0022BF9D11A
:1076D000002064220021FCF749FB0120F2E7012091
:1076E000F0E7D478917824020C430500E20502D536
:1076F000620A93401D000548FEF7D8FE7F21030073
:10770000214028009847C046872A002055420000A3
:107710000123037000487047DCCB00104A780B78D7
:1077200012021A438B7810B51B041A43CB781B0640
:1077300013439622D200934200D010BD0348FEF7B7
:10774000B5FE0021030008009847C04655420000DE
:1077500070B5184C82B005000E00200001A904F09D
:107760002BFF002808D1D0231B061B68019A9A42E0
:107770001CD0200004F040FF002001F049FE00284A
:1077800007D103256D42200004F0FEFE280002B060
:1077900070BD002001F054FE0028F2D02900320014
:1077A000002001F05BFE051EEBD0ECE703256D42E7
:1077B000ECE7C0465829002010B51F20FCF7F6F86A
:1077C000FA200021800010BD10B5064C00212000D9
:1077D00004F0F2FE002804D000F074FE200004F053
:1077E000D3FE10BD58290020F0B546464F46D64678
:1077F000C0B5364F82B080460E00380001A904F0B3
:10780000DBFE00280ED1D0231B061B68019A9A428A
:1078100005D102B01CBC90469946A246F0BD380086
:1078200004F0EAFE002001F0F3FD002832D000242D
:10783000002E34DD264B99469A4612E0002843D1AB
:1078400000F040FE002001F089FE002001F0E0FD84
:10785000002824D0002001F0BDFE002823D0A6423D
:107860001DDD0020351B01F0B5FE8542E6DC4346F8
:107870002A001919002001F029FE050000F022FE5F
:10788000002001F06BFEFBF76DFA4B46641918609F
:107890005960E4E7002000210D4B18605960380062
:1078A00004F072FEB5E7FBF75DFA53460D001A6867
:1078B0005B6800218446074812184B419D42EED870
:1078C000CDD19445CBD9EAE70500D0E7582900206F
:1078D000581E002020A1070010B51D4B84B01B7856
:1078E00002F08AF81B491F20FCF770F801211F20C5
:1078F000FCF74AF81848FBF72BFBFAF709FF0400DE
:10790000FBF730FAFA220023920012184B419942F9
:1079100018D901225242D31701210291002101916D
:107920000E4920000091FAF7F7FE0400631E9C4107
:10793000E4B2002803D001210948FFF721FE20000E
:1079400004B010BD9942E7D19042E2D8E4E7C046C6
:10795000F4D00010C977001058290020B977001022
:10796000B01400200048704794CC001000487047C5
:1079700040CC001070B5040016480378002B20D0CE
:10798000002C06D1C1241448144BA4004380048069
:1079900070BD052C1CD8124B0F48A400E558811C63
:1079A000002304E001330A800231132B0DD0EA5C7E
:1079B000DCB2002AF6D1C023013464009B001C43D2
:1079C000E5E7112102F0A0FADAE7CA24A400DEE715
:1079D0000020DDE7702A0020F823002009040000C1
:1079E000A8CC0010F0B55746DE464E4645469823D3
:1079F0008024E0B56B4A6402D75883B0274228D070
:107A000001222321684B00205A54DA70674901F0A3
:107A1000B3FA8022664B92021A65664B9A46FB06C1
:107A20001CD480235B011F424AD18023DB011F420B
:107A300000D08DE080231B021F4200D096E0BC42A4
:107A400000D0AAE003B03CBC90469946A246AB46A3
:107A5000F0BD102300249A46FB06E2D5514B9B6DE6
:107A60009846002B27D0524B00249B460123994671
:107A700043460126B8461F0004E001347600E4B214
:107A8000202C17D03E42F8D05B469E654B466508D9
:107A9000A3436D00ED18444B6D019C4665442800DE
:107AA00000F08CFB00286CD10134B743E4B27600BF
:107AB000002FE5D1474680235B0154461F42B4D0D6
:107AC0001C430023374A00211360384A3A48936028
:107AD000D3603A4A9360D360394A9360D360394A9D
:107AE0009360D360384A9360D360384A9360D36020
:107AF000374A9360D360374A9360D360364A9360C5
:107B0000D360364A9360D360354A9360D360354A78
:107B10009360D360344A9360D360344A9360D360F7
:107B2000334A9360D360F0229200FFF78DFB314B14
:107B3000314A00211A600020012201F0F1F980226F
:107B40001B4B12031A658023DB011F4200D171E732
:107B50000122042100201C4301F050F91022144B93
:107B60001A6580231B021F4200D168E7012205210C
:107B700000201C4301F042F980220D4B12011A65CE
:107B80005DE74B46AA8AA97800200093002301F004
:107B90001BFA280000F03AFA86E7210017487940DE
:107BA000FBF76AFD000011502C240020000010504B
:107BB00000301150100001006C240020080010500B
:107BC00010001050180010502000105028001050C5
:107BD0003000105038001050400010504800105035
:107BE00050001050580010506000105068001050A5
:107BF000700010503428002080011050C0CC0010BC
:107C000010B501210520FBF7BFFE10BD10B5002205
:107C10000021024800F02CFA10BDC0464C24002080
:107C20008022024B5202DA647047C0460020115095
:107C3000F0B5C64600B5070000F0C2F90C23354D7B
:107C40003549AB670520FBF7C1FE40239846334C0E
:107C5000402200212000FFF7F7FA43460126A383C4
:107C6000212100232E4A6670A260136063545F31A5
:107C700061844146A187023963542A4A2A496360D4
:107C8000E260A1620B60E262284A63629360D360A3
:107C9000274A20009360D360264A00219360D36076
:107CA000254A40309360D360244A9360D360244ACD
:107CB0009360D360234A9360D360234A9360D36078
:107CC000224A9360D360224A9360D360214A936032
:107CD000D360214A9360D360204A9360D360204AE6
:107CE0009360D3601F4A9360D360F0229200FFF745
:107CF000ABFA1D4B1D4A38001A6080239B052E6489
:107D0000EB6490231A4AEA50FFF78AFF04BC9046BE
:107D1000F0BDC04600001150E57900102C24002071
:107D200084001050000110508000105000001050CE
:107D30000800105010001050180010502000105073
:107D400028001050300010503800105040001050E3
:107D50004800105050001050580010506000105053
:107D6000680010507000105034280020800110501E
:107D700010D001000B785B0602D14B78052B00D0A8
:107D800070478A78014B1A60FAE7C046000011502C
:107D9000F0B5CE46474680B58B7848799C46072398
:107DA0000340C8780A798007800F1B021343C2B2D0
:107DB00091467F21624666461140D4094F00294D05
:107DC0003A195201AA1896700126B44666466640D2
:107DD000567000269383D6709077CA00012C27D066
:107DE0002148804688014244281882601660002994
:107DF00027D01E4AC9009446614441603F223F3368
:107E000093434A46022A00D15B0019493F190A6888
:107E10007F01D3180B60174BED19EA605A4080239D
:107E20001B0613434A4696061E436B681E600EE00F
:107E30001148804688014244281882621660002951
:107E40000AD1002364012D196B600C4BEB600120FB
:107E50000CBC90469946F0BD064AC9009446614460
:107E60004162CBE72C240020840010500400105005
:107E700034280020000010508000105000011050E5
:107E800000231C4A10B59360D3601B4A0021936005
:107E9000D3601A4A1A489360D3601A4A9360D36039
:107EA000194A9360D360194A9360D360184A93606B
:107EB000D360184A9360D360174A9360D360174A1F
:107EC0009360D360164A9360D360164A9360D36080
:107ED000154A9360D360154A9360D360144A936047
:107EE000D360F0229200FFF7AFF9124B124A1A60EA
:107EF00010BDC04600001050080010501000105077
:107F00006C24002018001050200010502800105041
:107F100030001050380010504000105048001050F1
:107F20005000105058001050600010506800105061
:107F30007000105034280020800110507F2020B5A0
:107F4000150008404000C909401804494001401884
:107F50001A00290000F08CF8012020BD2C240020FC
:107F60007F2310B50B40C909002B03D1022207481B
:107F7000521A8266802258004018054B4001C018F2
:107F80001201002100F048F810BDC0460020115039
:107F90002C2400207F2310B50B400BD0C9095800BA
:107FA0004018054B4001181800230022C3700349F4
:107FB00000F032F810BDC0462C240020FFF7FFFF70
:107FC00080220D4B520410B51A600C4B0C491A60FC
:107FD00010008B689843FBD10A4C9C2200212000A2
:107FE000FFF732F98022002152010748FFF72CF9F0
:107FF0000923636710BDC04600E0004000F0004068
:1080000000C0004000001150000010500023037415
:10801000438283828361704710B58368002901D051
:108020001C682140002A11D08024E4001143224220
:108030000CD01A6822420BD10A4A0A401A60FFE7A4
:10804000FFE7FFE7FFE7FFE7FFE78368196010BD81
:108050007F2281780448CB091140044A9B009A583A
:10806000FBF70AFBFFFBFFFFD4CC0010C414002079
:10807000F0B5C646002300B583820133037443681C
:1080800004001E68838B81611F1C934200D9171C5A
:108090008025BFB2D21BE37892B2ED0062823D43ED
:1080A000002B02D09025AD013D4301204340E370F9
:1080B0006378002B50D0002A1DD1A023DB011D4383
:1080C000384B1B6C384B33408026B6051E43636823
:1080D000A2681E6013685B0559D4344B2B401360B3
:1080E000FFE7FFE7FFE7FFE7FFE7FFE7A3681D60A4
:1080F00004BC9046F0BD80235B011D43294B1B6CE3
:108100009B0702D4A378DB09DCD0A38B191C934214
:1081100000D9111C80278BB2FF00D21A98461F434A
:10812000E37892B26282002B03D090274146BF01D0
:108130000F4301214B40E3706378002B19D0002AD4
:1081400002D18023DB011F43194B3F043340A0269B
:10815000F6053D431E43BAE73A00E068FFF77AF8B8
:10816000A369628A9C46802367441B02A7611D4362
:10817000A1E7E06842464030A169FFF76BF8A369C8
:10818000628A4344A36180231B021F43D7E77F22F7
:10819000A1780848CB091140074A9B009A58FBF781
:1081A0006BFAC04600001150FFFFFFAFFFFBFFFF5F
:1081B000FFFFFFDFD4CC0010C4140020F0B5C6468A
:1081C00000B5067C0400002E00D1D8E083681A6850
:1081D0001D684378AD05AD0D002B50D1838AEB1897
:1081E0009BB28382A18B62688D4206D20023638298
:1081F0001368300004BC9046F0BD1268520001D5EF
:108200008D4269D0638A002BF3D062681F1C166808
:108210008B425FD88025BFB2DB1BE2789BB2ED00BA
:1082200063823D43002A37D101214A40E2706278DF
:10823000002A3AD0002B47D0802252011543584AD9
:10824000126C920757D4A278D20954D1554B3340BF
:108250008026B6051E436368A2681E6013685B052E
:1082600000D593E0504B2B401360FFE7FFE7FFE79B
:10827000FFE7FFE7FFE7A36800261D60B9E72A00D4
:10828000C1688069FEF7E6FFA38AA269EB189BB27A
:108290005219A382A261A5E7012190254A40E2700C
:1082A0006278AD013D43002AC4D13A00A169E0687B
:1082B000FEF7D0FFA3699C4680231B021D43638AFF
:1082C0006744A761002BB7D1A023DB011D43344BCA
:1082D0001B6CBBE70F1C9DE7A26815686278AD01B7
:1082E000AD0D002A3DD1EB18A3828D4200D389E762
:1082F000002363827DE7A28B111C9A4221D880273C
:108300008AB2FF009B1A90461743E2789BB26382C1
:10831000002A03D090274146BF010F4301214A4064
:10832000E2706278002A0ED0002B02D18023DB019C
:108330001F431E4B3F043340A026F6053D431E431A
:1083400089E7191CDBE7E06842464030A169FEF787
:1083500081FFA3694344A36180231B021F43638AF7
:10836000E2E7E1682A004031A069FEF773FFA38AC3
:10837000A18BEB18A382A3695B19A361B5E77F23E7
:1083800081780B4A19400B48FBF776F97F22A178D8
:108390000948CB091140064A9B009A58FBF76CF933
:1083A00000001150FFFFFFAFFFFBFFFFFFFFFFDFEC
:1083B000C4140020F4CC0010D4CC0010024B587828
:1083C000431E9841C0B2704720220020024B18780B
:1083D0004007C00F7047C04620220020014B18788C
:1083E0007047C046832A0020F8B54746CE462B4D3D
:1083F00080B52B780700002B04D001200CBC9046E0
:108400009946F8BD532200212548FEF71DFF254C53
:108410002000FAF79DFD244B1C60244C20001C30EA
:10842000FAF7B2FD200001F023FD214B1C60214B27
:10843000002B2AD0204E00243000FFF769F91F4B93
:108440001F4A98461860914633780BE04246630015
:108450001B191268DB009B58984701343378E4B24B
:10846000A34209D39C42F1D315D14B46984701341E
:108470003378E4B2A342F5D23800FFF7D9FB3800D5
:10848000FFF7BEFB01232B70B7E701F0B1F80A4BF1
:108490001B78002BF0D000231B68FFDE832A00200E
:1084A00020220020D821002074220020CC1400209B
:1084B0007822002011770010822A0020E81E002078
:1084C000F1950010F0B5DE4657464E464546E0B5FC
:1084D0008BB001F097FA002800D18FE1CF4BD04E3E
:1084E0009B4607AC3568EA69EFF3108172B61368F2
:1084F000002BFCD0BFF35F8F29622800210001F020
:108500003DFBEA692B6ABFF35F8F0021116083F3A3
:108510001088002800D171E16378082BE2D85A4610
:108520009B00D3589F466368002BDBD0A068984718
:10853000D8E77F222179BB4B0A405500C8095B1957
:108540001B18180001273030C578BD43C570C578A9
:108550000337BD43C570002A00D199E1B24ADB7CE4
:10856000002A00D190E1B14A1278934200D389E108
:108570005A00D318AE4ADB001268D318002B00D182
:108580003CE11D6962792078A368A847AAE7012227
:10859000A44F01213B78042013433B703323FA5C42
:1085A0008A43FA54FA5C8243FA540133FA5C8A43F0
:1085B000FA54FA5C8243FA5423780020019300F0C5
:1085C00095FE602322791340602B00D151E1402BAE
:1085D00000D141E1D206D20E012A00D16AE1002A7F
:1085E00000D15BE1022A00D043E17F22217A0A40D8
:1085F0000F2A00D93DE1C80984465200B8188A4DB7
:108600006044C07C002D00D18FE1884D2D78A842B8
:1086100000D388E145002818854DC0002D682D182D
:10862000002B00D187E1002D00D122E1E86800F0A5
:108630005DFEEB6808AA00210198984716E1794B86
:108640001B78DB0700D44DE77A4B002B00D149E7BC
:1086500000E000BF46E7734B1A78D20700D441E729
:10866000754A002A00D13DE718780007C00F00E0E6
:1086700000BF37E76D4D6C4A2B78002A00D1B7E078
:1086800000276B491A0088469F4214D24146096868
:108690007B008C46DB19DB0063445B69002B0DD04B
:1086A0002078984701372A78FFB2974200D919E716
:1086B00013009F42EAD39F4200D09CE00137FFB2F3
:1086C000974200D90EE71300F3E72378574D564A37
:1086D000984600272B78002A00D1B3E0574A9246EB
:1086E000534A91462A00454690460FE04A46126892
:1086F0007B009446DB19DB0063445B6828009847E5
:10870000434601371B78FFB2BB420BD39F42EDD3E8
:108710006BD1534628009847434601371B78FFB278
:10872000BB42F3D23F4D532200212800FEF78CFDBF
:108730001022FF21E81CFEF787FD28002022FF21E0
:108740001330FEF781FD00F0C7FD3D4B002B00D13B
:10875000C8E600E000BFC5E62378344D324A9846AB
:1087600000272B78002A50D0344A9246304A91464E
:108770002A00454690460FE04A4612687B00944620
:10878000DB19DB0063445B682800984743460137E8
:108790001B78FFB2BB420BD39F42EDD325D153468A
:1087A00028009847434601371B78FFB2BB42F3D2FB
:1087B0001C4D532200212800FEF746FD1022FF2108
:1087C000E81CFEF741FD28002022FF211330FEF7B0
:1087D0003BFD00F081FD2379AB7083E6019800F04A
:1087E00045FF2B78002B00D192E200235B68FFDE6F
:1087F000002B00D176E600235B69FFDE0BB03CBCAA
:1088000090469946A246AB46F0BD404600F02EFF8A
:108810002B78002BCCD000235B68FFDE28CD001026
:10882000782200202022002011770010822A0020C8
:10883000E81E002000000000000000006D960010FF
:1088400000000000404600F011FF2B78002B00D103
:1088500068E700235B68FFDEC948002809D000F004
:1088600045FD08AA0021019800E000BF002800D0C3
:1088700038E620780021FFF773FB20788021FFF78E
:108880006FFB2FE69B1ADBB2002BB7D1BD4D79E60B
:1088900062792078A36800F03DFD23E6202B00D10B
:1088A00028E1002BE5D16379092BE2D8B64A9B0079
:1088B000D3589F46237A0F2BDBD8B44AFB18DB78BA
:1088C000002A2BD0B24A1278934225D2B14A5D00D9
:1088D000EB181568DB00ED18002DCAD0E86800F031
:1088E00005FDEB6808AA002101989847002800D0F0
:1088F000F8E5602523791D40BBD163790A3B012B44
:10890000B7D800F0F3FC63790A2B00D150E108A935
:10891000019800F06FFCE5E59B1ADBB2002BA8D1B3
:108920009D489E4DDBE7401BC0B2002800D1F8E017
:108930000025002B9DD163799946012B04D0002B93
:1089400000D1FAE0032B94D1E388002B1BD14B46D6
:10895000BA18012B00D1FAE013003022904663448C
:1089600098444346DB789B070DD40198FFF7F8FA4B
:1089700043460222DB7813434246D370D378012268
:1089800013434246D370002D00D1ABE5E86800F0F8
:10899000ADFCEB6808AA002101989847002000F080
:1089A000A5FC3423FB5CDB0700D59BE5AFE7A3798F
:1089B00003931A007B789A4207D07B78002B00D073
:1089C0007EE1039B002B00D0FBE0039B08A90198EC
:1089D0007B7000F00FFC85E57B7806AA02321370ED
:1089E00008A90123019800F01DFC7BE5E088030A3B
:1089F000C0B20F2B00D93CE769499A008A589746C4
:108A000008A800F079FCA1790198FFF7FFF802228D
:108A10003B7813433B7065E5E388012B00D028E7E2
:108A200008223B7808A9934301983B7000F0E2FBD1
:108A300058E50220397806AB9A1C8B068908DB0FB3
:108A400001400B43138008A90223019800F0EAFBC0
:108A500048E5E388012B00D00BE708223B7808A902
:108A6000134301983B7000F0C5FB3BE54D4B002BD9
:108A700000D1FEE600E000BFC37881781B0202004F
:108A80000B43019808A900F0CDFBEFE6464B002B05
:108A900000D1EEE600E000BF021E00D1E9E6137847
:108AA00008A9019800F0BEFBE0E62189FEF762FF0D
:108AB000021EF4D1DDE6022B00D176E13B4B002B08
:108AC00000D1D6E600E000BF002800D1D1E6C3788F
:108AD00082781B02134308A90200019800F0A2FB50
:108AE000C4E6FEF73FFF1223020008A9019800F038
:108AF00099FBBBE6237A0F2B00D9BAE6234AFB1871
:108B0000DB78002A13D0224A127893420DD2214AF0
:108B10005D00EB181568DB00ED18002D00D1A8E60C
:108B200084E5002B06D11D4D05E79B1ADBB2002B17
:108B300000D09EE61848194D79E5BA181300634431
:108B40003033DB7806AA9B07DB0F02327AE72F333C
:108B50009846624490444346DB789B0700D412E772
:108B60000198FFF717FA43460222DB789343424607
:108B7000D370D3784A4693434246D37003E7C04646
:108B800000000000619800104CCD0010117700101B
:108B9000822A0020E81E00207D970010B4CD00102E
:108BA00074CD001000000000000000000000000074
:108BB00006AB9A1C08A901230198157000F032FB3E
:108BC00090E4581EC0B2FEF7D1FE002800D150E656
:108BD0004378022B00D04CE60125C3795A112A4074
:108BE000120191463A789B119046102241469143DA
:108BF0000A0049460A4320212B408A435B01134364
:108C00003B7009239946C37882781B021343C3182B
:108C100081440493994500D3C0E04D4601226B780E
:108C200002920B2B04D1EB7802932B78ED186B7822
:108C3000042B00D01DE60022049B90465B1B9BB2D8
:108C40009A46674A674B1B78002A25D02A0045467A
:108C500090469D421AD2644A6B0012685B19914695
:108C6000DB0099444B469B68059252464146019869
:108C70009847082803D95346834200D3A7E0594BAD
:108C800001351B78EDB2AB42E3D2F2E59D4214D13F
:108C9000564A574B9146E8E752462900019800F0A2
:108CA000FBFCD0468246082802D94346834242D282
:108CB0004C4B1B78002B00D1DBE500239B68FFDECB
:108CC0000198FFF7DDF8BB78464D454A9A460021EA
:108CD0002B78002A00D181E5434A90462A000D00F6
:108CE00091460FE0424612686B0094465B19DB0028
:108CF00063445B68019898474B4601351B78EDB299
:108D0000AB4205D39D42EDD300D06EE5394BF1E780
:108D1000532200213800FEF797FA1022FF21F81C99
:108D2000FEF792FA380020221330FF21FEF78CFA6A
:108D30005346BB7045E62D4B9946294B9846029BFE
:108D4000012B35D0029B002B17D0A9787A18D27846
:108D50000B00FF2A00D08CE5002206E08B18DBB266
:108D6000F818C078FF2800D083E54046FB18D8707B
:108D70000132029BD2B29A42F0D338004346290016
:108D80001330524600F07EFE164B55441B78434587
:108D900000D26EE5049BAB4200D93FE7164B002B97
:108DA00000D112E600E000BF0FE6FEF7DFFD8BE624
:108DB00048468068A97884460D487B18DA7884454F
:108DC0000AD0FF2A00D054E54246DA70D5E7434680
:108DD0008246A8461D00B2E702230293B6E7C046CA
:108DE00011770010822A0020E81E0020B4CD001068
:108DF000999600106D9600100000000070B586B0C6
:108E00006B4605000C00981C0A220021FEF71CFA94
:108E10006B461D705C70032C4FD01BD9042C07D0FF
:108E2000052C40D13C4B1A78D20766D406B070BDF1
:108E3000394B1A78D207F9D504211A780A431A70E7
:108E4000364B1C68E269EFF3108172B61368002B91
:108E500019D1FBE7022C26D101212F4B1A788A4326
:108E60001A701A780331A2431A7000225A701A78C5
:108E70008A431A70294B1C68E269EFF3108172B6BD
:108E80001368002BFCD0BFF35F8F2162694620007E
:108E900000F03AFFE269236ABFF35F8F002111609F
:108EA00083F31088C2E71D4B1C68E269EFF3108161
:108EB00072B61368002BE6D1FBE7174B1A785207FE
:108EC000B4D504210E201A7868448A431A70002110
:108ED0000A22FEF7B9F9052303AE73700F4B357004
:108EE0001C68E269EFF3108172B61368002BFCD0A6
:108EF000BFF35F8F21623100C9E704211A788A43EA
:108F00001A70064B1C68E269EFF3108172B61368A1
:108F1000002BB8D1FBE7C046202200207822002099
:108F200070B584B06B4606000D000A220021981D22
:108F3000FEF78AF9012301AC63700E4B25711D68A1
:108F40002670EA69EFF3108372B611680029FCD02D
:108F5000BFF35F8F2B622100280000F0D5FEEA6985
:108F60002B6ABFF35F8F0021116083F3108804B078
:108F700070BDC04678220020002330B585B001AD19
:108F80006B8028700633082202A86B70FEF762F926
:108F90000C4B1C68E269EFF3108372B6116800296C
:108FA000FCD0BFF35F8F23622900200000F0ACFEED
:108FB000E269236ABFF35F8F0021116083F3108899
:108FC00005B030BD78220020F0B5C64600B584B0AB
:108FD0001D006B4680460F00160000210622981DDA
:108FE000FEF732F9434601AC2370072363700F4B41
:108FF00065711D682771A660EA69EFF3108372B688
:1090000011680029FCD0BFF35F8F2B62210028007C
:1090100000F07AFEEA692B6ABFF35F8F00211160CE
:1090200083F3108804B004BC9046F0BD7822002081
:10903000F0B5DE464F4646468346C0B50C00002AD2
:1090400043D04978052916D1E678B607B60FB34262
:1090500011D17F23A1780B400F2B0CD8531E9846BB
:109060001B4B002599467F274B462000997800F03E
:10907000CDFC002805D100201CBC90469946A34693
:10908000F0BD21005846FEF783FE0028F3D0A378F8
:10909000DA09012A13D0089A13702378E418454599
:1090A00013D06378052BE6D1E3789B079B0FB3427F
:1090B000E1D1A37801353B400F2BD5D9DBE7099AE5
:1090C00013702378E4184545EBD10120D4E7C0465E
:1090D000202200207F2370B58A7805000C00134001
:1090E0000F2B01D9002070BD054B2000997800F0AE
:1090F0008DFC0028F6D021002800FEF749FEF2E79B
:10910000202200207F2370B50B40134C5B00C9095F
:10911000E41864183034E578ED07ED0F04D1E378F6
:109120005B0703D5280070BD0025FBE701210B4E2E
:109130004942306803F048FAE378DB0707D4E37864
:109140005B0704D404220125E3781343E3703068FD
:1091500003F01AFAE6E7C04620220020742200201D
:1091600070B50D0001210F4C4942206803F02CFA24
:109170007F2129404B000C49ED09C91849193031AC
:10918000CB780025DB0707D4CB785B0704D5042216
:10919000CB7801359343CB70206803F0F5F92800B4
:1091A00070BDC046742200202022002070B57F24AC
:1091B0000C4065000E4C06006419C80924183034B0
:1091C000E5780020ED0700D570BD0125E078284343
:1091D000E0703000FEF7B2FE0028F5D10122E378FE
:1091E0009343E370E37803329343E370ECE7C046C4
:1091F0002022002070B50A4C0600082220000D0035
:10920000FEF728F800230021A360E36069563000D0
:10921000C943C90FC9010022FFF7C8FF70BDC0468E
:10922000C4210020F0B5C6469046294C082200B55E
:10923000060020000D001F00FEF70CF84346A36057
:109240000023E381EB79AA791B0213431A1CBB426A
:1092500000D93A1C97B2A281002B12D0002F1DD04A
:109260004346002B2ED03B1C402F1DD89FB22378A5
:109270007F2B1ED80021174A3B003000FFF796FFD6
:1092800009E0002169560023C943C90FC901002222
:109290003000FFF78BFF04BC9046F0BD23787F2B96
:1092A00012D800210022E7E740239FB223787F2BCA
:1092B000E0D9084C3A0041462000FDF7CBFF802161
:1092C0002200D9E70020E6E780210022D4E7C0464B
:1092D000C4210020E021002010B514220021024802
:1092E000FDF7B2FF10BDC046C4210020014B18613C
:1092F0007047C046C421002010B5054C010008226B
:109300002000FDF7A7FF0023A360E36010BDC04667
:10931000C4210020F8B53B4C1D0023780600DA0973
:10932000C9098A4212D00020002D0ED1364B002BE5
:1093300003D021003000FEF71DFD2369002B5AD019
:1093400022000221300098470120F8BDA7687F2B3A
:1093500008D80020002FF8D038002A002B49FDF74C
:1093600079FFA768E289E388521992B27F19E281F6
:10937000A760934201D03F2D13D82369002B05D05D
:10938000220001213000984700281DD0002161569D
:109390000023C943C90FC90100223000FFF706FFAF
:1093A000D3E7A089811A0D1C89B2402916D82378E9
:1093B000ADB27F2B14D8002182421ED0134A2B005D
:1093C0003000FFF7F3FEC0E700213000FEF7C8FDD4
:1093D00030008021FEF7C4FD0120B6E74025E6E716
:1093E00082420CD0094C2A0039002000FDF732FFE0
:1093F00080212200E3E70120A7E70022DFE78021A8
:109400000022DCE7C4210020757D0010E02100204F
:1094100010B50400FEF7D2FF002801D1002010BDD6
:10942000FEF7D4FF0028F9D1B6208000444303485A
:109430000019037901201840F1E7C046EC1E002016
:109440000300B6208000584310B5034B1030C018FD
:1094500000F06AFB10BDC046EC1E0020F0B5B6253A
:10946000AD0045432C00C646174E1034A41900B574
:1094700092B2200000F0D0FB0700200000F06EFB4D
:109480003F2803D8380004BC9046F0BD7319D97842
:1094900000209846FFF736FE0028F3D0200000F0A9
:1094A0005DFB3F2805D843460020D978FFF758FEDA
:1094B000E8E796239B00EA1843469219D9780020E2
:1094C0004023FFF773FEDDE7EC1E0020F0B5B62564
:1094D000AD0045432C00C6461F4E2C34A41900B5E0
:1094E00092B2200000F050FC0700200000F01CFBAE
:1094F0003F2803D8380004BC9046F0BDFEF75EFF5D
:109500000028F7D0FEF762FF0028F3D1200000F01A
:109510000BFB0028EED07319997800209846FFF7CE
:10952000F1FD0028E6D0A6239B009C466544AE19B9
:1095300031004022200000F06FFB4346997800285C
:1095400005D0030032000020FFF730FED2E70020F4
:10955000FFF706FECEE7C046EC1E0020F8B505007A
:10956000FEF72CFF002801D10020F8BDFEF72EFFEA
:109570000028F9D1B624A40065432E00144F2C36E0
:10958000F619300000F0D0FA0028EDD07C19A1784F
:109590000020FFF7B7FD0028E6D0A6239B009C46DD
:1095A0006544ED1929003000402200F035FBA17818
:1095B000061E08D003002A000020FFF7F7FD002850
:1095C000D2D03000D1E70020FFF7CAFDCCE7C0467B
:1095D000EC1E00200300B6208000584310B5034B5A
:1095E0002C30C01800F0BAFA10BDC046EC1E0020A6
:1095F000B622F0B51B4C83B0920000212000FDF78D
:1096000023FEFF236371184B80260025E38001278A
:10961000082321002000760023732781320048317F
:109620000095073B103000F043FA2100200049313B
:109630003200FF31009701232C3000F039FA9223D9
:109640009B00E6183000F9F783FC94239B00A66288
:10965000E61865623000F9F77BFC2664656403B0A8
:10966000F0BDC046EC1E002000C2FFFF10B5094C43
:10967000052200212000FDF7E7FD20002C341030EA
:1096800000F0F6FB200000F0F3FB0121200000F0C9
:1096900015FC10BDEC1E0020F0B54B7983B0060020
:1096A000022B03D00025280003B0F0BD8B79022BDC
:1096B000F8D12F4FBB78002BF4D18B7809253B7064
:1096C0000C780C196378242B0BD1082A02D81FE0E0
:1096D000AA421DD32378E418ED186378ADB2242B89
:1096E000F6D0052B2CD0042B12D163790A2B0FD185
:1096F000204B2778019301330093E11902230222C2
:109700003000FFF795FC0028CCD00E35ED19ADB236
:10971000194C200000F022FA3F28C4D92600103E40
:10972000F1780020FFF7EEFC0028BCD0200000F00C
:1097300015FA3F2812D8F1780020FFF711FDB2E7A3
:1097400021003000FFF7C6FC0028ABD0A3787B7067
:109750002378ED18E418ADB26378C4E792239B0038
:10976000E218F17840230020FFF720FD9BE7C04678
:10977000EC1E0020EE1E0020FC1E0020F8B5602329
:109780001400127813400022202B01D01000F8BDE5
:109790002E4D637927792E781B023B439E42F5D1EB
:1097A0006378212B43D009D9222B24D0232B14D129
:1097B000002945D0022912D00122E7E7202B0CD145
:1097C000002936D00229F7D1214B002BF4D0A91D56
:1097D0000020FDF7A3FF0122D8E70022D6E71D4BAA
:1097E000002BE9D0E178A37809021943002000E0BA
:1097F00000BF0122CAE7002922D00229DCD10126BC
:10980000A178E478280024020C4331002C71A14394
:109810002C3000F053FB104B002BCDD031006208F0
:1098200032402140002000E000BF0122AEE70029C5
:10983000C2D10A4A07232100FFF7F4FC0122A5E761
:109840002100FFF7D7FC0122A0E7C046EC1E002054
:109850001D7700100000000000000000F21E002034
:10986000F8B54746CE4680B55D4C1E00E37880468D
:109870000D008B4263D1962327009B001037E1181F
:10988000B2B2380000F080FA564B002B1CD063793E
:10989000FF2B19D0002E17D00022914605E001239E
:1098A0009C46E1444E450FD06379962292004A448B
:1098B000A25C9A42F3D1380000F048F90028EED1BA
:1098C000617900E000BFEAE7474B484C002B04D029
:1098D000200000F03BF900285BD0200000F03EF9AA
:1098E0003F2859D8103CA378AB4205D00124200072
:1098F0000CBC90469946F8BD3D4B002B02D0002091
:1099000000E000BFFEF75AFD00281DD1394C2000B1
:1099100000F00AF90028E9D1002EE7D0B306E5D11E
:109920002C3CA1784046FFF7EDFB2500041EDDD05E
:10993000A978002300224046FFF738FCD7E7A37838
:109940008B42D9D00024D2E7FEF740FD294C0028F5
:10995000DDD1200000F0E8F80028D8D025002C3D0B
:10996000A9780020FFF7CEFB0028D0D09B239B00D6
:10997000E71839004022200000F04EF9A9780028AD
:1099800029D003003A000020FFF710FC0028ADD1D9
:10999000BDE700E000BFA0E72700103FF9780020F6
:1099A000FFF7B0FB002801D1BB789DE7200000F055
:1099B000D5F83F2805D8F9780020FFF7D1FBBB7810
:1099C00092E792239B00E218F97840230020FFF7EA
:1099D000EDFBBB7888E70020FFF7C2FB97E7C046A6
:1099E000EC1E00200000000000000000FC1E002013
:1099F00000000000181F002010B50020FEF7F4FC46
:109A000010BDC04610B5FEF7E9FC10BD072310B528
:109A10004479027923401B021A43C3789B079B0FAA
:109A2000022B1BD00DD80020012B09D102394B424B
:109A30005941124B00209C46614491424041C0B2C2
:109A400010BD02394B425941F023002049429B008E
:109A50001940403191424041C0B2F1E7022905D09E
:109A60000020402393424041C0B2E9E7044B9C46AA
:109A7000624450425041C0B2E2E7C046FF030000DA
:109A800000FEFFFFF0B500247F27002A0FD04D789D
:109A9000052D06D13D008E7835406D00F60945193B
:109AA000AB550D786419A4B24919A242EFD8F0BDA4
:109AB000F8B54746CE4680B5984608AB1F78802358
:109AC0000400894615001B0200269A4227D84069E7
:109AD000002803D00121494202F076FDA069002848
:109AE00003D00121494202F06FFD4B4623604346FB
:109AF000A5806D00ADB2E3806B1EA3810023606979
:109B00006D42E381277265812382002801D002F033
:109B10003BFDA0690126002801D002F035FD300090
:109B20000CBC90469946F8BDC189028A89B292B2AE
:109B30008B1A9BB2914202D242899B1A9BB28288B5
:109B4000101C9A4200D9181C80B27047C389008A41
:109B5000181A43425841C0B27047C04610B5C48974
:109B6000018AA4B289B2631A82889BB28C4202D263
:109B700040891B1A9BB2D01A80B210BD70B5040088
:109B800080690D00002803D00121494202F01CFD2C
:109B9000E089218A80B289B2421A92B2884202D206
:109BA0006389D21A92B2A388934208D2C21A92B29F
:109BB00098422DD26089121A92B222821A00002A8B
:109BC00002D11EE0C91A89B28B42FBD92368E28810
:109BD0009C46514328006144FDF73CFB228A012545
:109BE00092B2531C9BB29A420ED9002362899B18F1
:109BF0009BB2A0692382002801D002F0C5FC280096
:109C000070BD0025238A9BB2A2899A42F1D2EDE76A
:109C1000A0899042D1D2CDE7F8B54746CE460400A0
:109C2000806980B50E001700002803D00121494249
:109C300002F0CAFCE289218A92B289B2551AADB209
:109C40008A4202D26389ED1AADB2A388AB420AD22E
:109C5000D11A89B29A424CD26289891A89B21D00FE
:109C60002182218A89B2002D47D03A1CAF423BD8CD
:109C700095B28B4203D8C91A89B28B42FBD95B1AC1
:109C80009FB2E3885943984623689C466144BD428D
:109C900024D94046784383B21A0030009946FDF734
:109CA000D9FA43463000EA1B5A43484492B221682D
:109CB000FDF7D0FA228A92B253199BB29A421ED96A
:109CC00062899B189BB2A0692382002801D002F010
:109CD0005BFC28000CBC90469946F8BD424630001B
:109CE0006A43FDF7B7FAE5E72A1C95B28B42C2D961
:109CF000C5E7A2898A42B2D2AEE7238A9BB2A28983
:109D00009A42E0D2DCE7C046F8B5040040690E0094
:109D1000002803D00121494202F056FCE589238A3C
:109D2000ADB29BB2EA1A92B2AB4202D96389D21A9F
:109D300092B2A388934222D028009D4203D3C01A36
:109D400080B28342FBD92368E2889C4650433100AD
:109D50006044FDF77FFA6B1C9BB29D420BD9628970
:109D60009B189BB26069E3810127002801D002F0B3
:109D70000BFC3800F8BDA2899A42F3D2EFE7277AAC
:109D8000002FD9D1F5E7C046F0B54F46D646464636
:109D90000500C0B514000F00002A05D120001CBC2E
:109DA00090469946A246F0BD4069002803D00121A3
:109DB000494202F009FCEA88EE899046298A2A7A0B
:109DC000B6B289B2AB88002A0ED1721A92B28E4214
:109DD00002D26989521A92B29A1A111C92B2A24204
:109DE00000D9211C8CB207E09C4205D34246E41AFC
:109DF00054430E003F191C0030009E4203D3C01A8A
:109E000080B29842FBD21B1A9BB2994643465843F4
:109E10002B689C4660444C4515D842463900624345
:109E2000FDF718FAA3199BB29E4202D8AA899A425A
:109E300002D26A899B189BB26869EB810028ADD079
:109E400002F0A2FBAAE74B46414659438BB21A00E7
:109E500039009A46FDF7FEF94B46E21A43463900AF
:109E60005A43514492B22868FDF7F4F9DAE7C04644
:109E700010B504004069002803D00121494202F0D6
:109E8000A3FBA069002803D00121494202F09CFBFA
:109E90000023E3812382A38860695B009BB25A1E82
:109EA0005B42A2816381002801D002F06DFBA069B2
:109EB000002801D002F068FB012010BD70B504003D
:109EC00040690D00002803D00121494202F07CFBCB
:109ED000A069002803D00121494202F075FB6069A6
:109EE0002572002801D002F04FFBA069002801D0A4
:109EF00002F04AFB012070BD10B5024800F0EAF8FC
:109F000010BDC04648280020013930B5002900D1D5
:109F1000B4E06F4B1A781211D5B22C003034092AF4
:109F200000DDAEE00470012900D1A6E00F221C780C
:109F3000224014003034092A00D9A4E044700229D8
:109F400000D19AE05A781211D5B22C003034092A87
:109F500000DD9BE08470032900D18EE00F225C7845
:109F6000224014003034092A00D991E0C470042939
:109F700000D182E09A781211D5B22C003034092A2F
:109F800000DD88E00471052977D00F229C782240FB
:109F900014003034092A00D97FE0447106296CD0BE
:109FA000DA781211D4B225003035092A00DD77E0C5
:109FB0008571072961D00F22DC78224014003034EB
:109FC000092A00D96FE0C471082956D01A791211F4
:109FD000D5B22C003034092A00DD07340472092977
:109FE0004BD00F221C79224014003034092A01D9A9
:109FF0003732140044720A293FD05A791211D4B270
:10A0000025003035092A01DD3734250085720B29FA
:10A0100033D00F225C79224014003034092A49D809
:10A02000C4720C2929D09A791211D5B22C0030347F
:10A03000092A42DC04730D291FD00F229C7922408B
:10A0400014003034092A3AD844730E2915D0DA792D
:10A050001211D5B22C003034092A33DC84730F2955
:10A060000BD0DA790F2313401A003732092B2BD982
:10A07000C273102901D0103000E040180023037093
:10A0800030BD07344EE73732140057E7073461E735
:10A09000373214006AE7073474E7373214007CE77C
:10A0A0003734250084E737321400C471082900D002
:10A0B0008CE7E2E737321400B2E70734BAE7373209
:10A0C0001400C1E70734C9E730331A00D0E7C046AF
:10A0D0004828002010B588B004000D2200216846F1
:10A0E000FDF7B2F80D22002104A8FDF7ADF84B23CF
:10A0F0006A4604A9137068460D2202F03DFA152144
:10A10000082269442000FDF7A5F808B010BDC0463C
:10A11000F0B546468046354BD64643445A1E9341D9
:10A120008022520294464F465B421340304A6344B9
:10A13000C0B513602F4A0D002F49136018008A68BC
:10A140009043FBD10620F9F719FC80268146E90DE2
:10A150006802AB0DAA020224760006E0914507D3FF
:10A1600012184B413C00B74202D0A71C002BF5D07F
:10A1700080272602361B7F0003E05746361B012F3F
:10A1800031D07B1E310048469A46FCF7E5F98542FE
:10A19000F3D23900534661431B02424614611268F0
:10A1A00040465340FF2212021340802252010243D4
:10A1B0001360036807205840CF23034013604246D2
:10A1C000802303209B0124321A4310604246171D4E
:10A1D0001F43022348463B60FCF7BEF91CBC904677
:10A1E0009946A246F0BD21000023D6E70040FCBFFF
:10A1F00000E0004000F0004000C000400020704738
:10A200007047C046F0B5CE46474680B583B06B4632
:10A21000591D13230B700D3B6B44994601244A468C
:10A22000002313702300C268D02793403F06BB6110
:10A230000C4B050001221800984602F0CDF96B4640
:10A24000DE1D320001234946404602F0CDF9EB689D
:10A250009C407C613078EB69C01A03B00CBC90461E
:10A260009946F0BD00C00340F0B5CE46474680B5E4
:10A2700085B06B46D9710368364A5B680400934227
:10A2800062D10921222369440B70183B6B44984624
:10A2900001274246002313703B00C268D02693403A
:10A2A0000F253606B36101226D442B4802F094F964
:10A2B00001232A004146284802F096F93B00E26853
:10A2C000934073612A789046FF2A3AD00B21802070
:10A2D0006A466944087003A88146D2790270B36166
:10A2E00001221D4802F078F901232A0049461A4844
:10A2F00002F07AF93B00E268934001227361012683
:10A300000E2742446F443A700D21D022A2206944A6
:10A3100012060870904693610F48012202F05CF922
:10A3200001232A0039000C4802F05EF90123E2689B
:10A33000934042465361300005B00CBC90469946AC
:10A34000F0BD00220026DBE769460122073198476D
:10A350000600F0E719A4001000C00340F0B5C6469F
:10A3600000B503682A4A1B6982B00400934249D1B0
:10A370006B46D91C13230B7001AB984601250023B3
:10A38000424613702B00C268D02793403F06BB6142
:10A390000122204802F020F96B46DE1D3200012325
:10A3A00041461C4802F020F9E3689D407D61307809
:10A3B000E369C01A002827D0E36906220133E3616C
:10A3C0006B460125591D00236A440B7013702B0046
:10A3D0009046E268D02793403F06BB6101220D48BA
:10A3E00002F0FAF86B46DE1D3200012341460948AF
:10A3F00002F0FAF8E3689D407D61307802B004BC59
:10A400009046F0BD9847D5E701204042F6E7C046A8
:10A4100005A2001000C00340F0B55746DE464E4688
:10A420004546E0B587B004AB0C00591C22230B70E5
:10A4300004AB9F1C012500233B702B008146C068A4
:10A44000D0268340360602929046B36101223748F7
:10A4500002F0C2F804AA9446072363449A463900DE
:10A4600001235246314802F0BFF84B46DB685146A3
:10A470009D40C446756109782A008C44604603906B
:10A48000FF2805D9FF20401A8446614402900391B9
:10A490000299002927D08C46A4446246019204AA5E
:10A4A000D71C802293467F3A904605AE2278D0256D
:10A4B0003270424659469A402D0639701B48AA61AF
:10A4C0003900012202F088F8012352463100174872
:10A4D00002F08AF84B464246DB6801999A40013403
:10A4E0006A618C42E2D104AB591DA223D0240B70C7
:10A4F00004AB9D1D039B24062B700C48A261012216
:10A5000002F06AF8524601232900084802F06CF86C
:10A510004B46DA68012393400298636107B03CBC64
:10A5200090469946A246AB46F0BDC04600C00340E7
:10A53000F0B5D6464F464646C0B50368454A1B6946
:10A5400084B00400934200D07FE06B46D91D1323F2
:10A550000B7002AB984601250023424613702B0076
:10A56000C268D02793400F263F06BB6101226E448C
:10A57000394802F031F8012332004146364802F0F2
:10A5800033F8E3689D407D613078E369C01A0028A4
:10A590005DD00D210D2369440B7001336B44994646
:10A5A0000023984601264B4642461A703300E26863
:10A5B000D02593400F272D066F44AB61012226481A
:10A5C00002F00AF8494601233A00234802F00CF849
:10A5D0003300E2680B2193406B613A7869449246FC
:10A5E000424640460A7003AA91461070AB610122B0
:10A5F000194801F0F1FF494601233A00164801F0DD
:10A60000F3FF3300E268092193406B613A786944B3
:10A6100090468D220A70833A6A44504691461070E3
:10A62000AB6101220C4801F0D7FF01233A004946F3
:10A63000094801F0D9FFE36840469E406E6104B0CE
:10A640001CBC90469946A246F0BD98479FE7012062
:10A650004042F4E705A2001000C00340F0B54546B3
:10A66000DE464E465746E0B50126050089B0C06873
:10A670008846F7F7ABFD3300EA68D0249340286999
:10A68000240663626361431C0FD0F7F79FFD33001C
:10A690002A690A2093406362A361F8F709FA2B69DB
:10A6A0000A209E406661F8F703FAC849C848FFF7D8
:10A6B0002FFD01211020F7F771FD01211220F7F77E
:10A6C0006DFD01211320F7F769FD0820F7F77EFDE6
:10A6D000D024802324065B00636263616B46D91C2F
:10A6E000422301260B70002301AF3B703300EA6860
:10A6F000B74893400122A36101F06EFF1F2201239E
:10A700006A443900B24801F06FFF3300EA6800275D
:10A7100093406A466361D27F122A07D0380009B09D
:10A720003CBC90469946A246AB46F0BD11216F3223
:10A7300069440A7091466F3A6A44924680225046B4
:10A740000270A3617F3AA24801F046FF1F225146E2
:10A7500001236A449E4801F047FF3300EA689340B2
:10A760009A4663614346D917AB61C9045B0B194331
:10A770004346984AD8040023FBF730FF172186236D
:10A78000694480460B7006AB9B4643465A461B0CF9
:10A79000137053460122A3618D4801F01DFF1F2253
:10A7A00001236A4459468A4801F01EFF3300EA68D3
:10A7B000152193408722694463610A70713A6A44A3
:10A7C000924642465046120A0270A3610122804816
:10A7D00001F002FF1F22514601236A447C4801F028
:10A7E00003FF3300EA6813219340882240466944FE
:10A7F00063610A7005AA10709246A3610122744831
:10A8000001F0EAFE1F22514601236A44704801F01C
:10A81000EBFE3300EA680F2193408E2269446361A6
:10A820000A7004AA17709046A3610122684801F0DB
:10A83000D3FE1F22414601236A44654801F0D4FE3D
:10A840003300EA680D2193408F226944636190468A
:10A850000A70813A6A4417709246A36101225C48EB
:10A8600001F0BAFE1F22514601236A44584801F004
:10A87000BBFE3300EA680B2193400C2269446361FC
:10A880000A7003AA17709246A3610122504801F092
:10A89000A3FE1F2201236A4451464D4801F0A4FE45
:10A8A0003200EB6809219A408C206B466944626152
:10A8B00008700320DB7F0A3703436F443B70444832
:10A8C000A261012201F088FE1F22390001236A449F
:10A8D0003F4801F089FE3300EA6802AF93406A46C0
:10A8E000D11DA62263610A70A23A3A703848A3616A
:10A8F000033A01F071FE1F22390001236A443448F3
:10A9000001F072FE3300EA681B219340CD226944B6
:10A91000636107AF0A70493A3A702D48A361833AE0
:10A9200001F05AFE1F22390001236A44284801F031
:10A930005BFE3300EA68192193401A278B22694491
:10A9400063616F440A70603A3A702148A3612A3A01
:10A9500001F042FE1F22390001236A441C4801F025
:10A9600043FE3300EA681D219340892269441E2773
:10A9700063610A7042466F443A701548A3618E3A8B
:10A9800001F02AFE1F22390001236A44104801F019
:10A990002BFE3300EA680E4893406A46511D4A4632
:10A9A00063610A706A46971D4A463A70A361803A0D
:10A9B00001F012FE1F22012339006A44044801F00D
:10A9C00013FEEB6801279E406661A7E6D4300000C5
:10A9D00000C003400048E801F0B5CE46474680B5C8
:10A9E00087B06B4601258946D91C002301AF3B7017
:10A9F00098462B00C268D026934036060D7004009E
:10AA0000B3610122794801F0E7FD172201236A446E
:10AA10003900764801F0E8FD2A00E36800209A40FA
:10AA20006B467261DB7DDB439B0700D19FE06B4689
:10AA3000591D12230B706B469F1D43466B483B709C
:10AA4000B261012201F0C8FD172201236A443900D6
:10AA5000664801F0C9FD2B00E26893406A467361C5
:10AA6000D17D08220A4200D086E009210A25D0269D
:10AA7000812269446D4436060A702A705B48B361CE
:10AA8000803A01F0A9FD17222900012501236A441B
:10AA9000564801F0A9FD2B00E26893404A467361D5
:10AAA000002A00D07FE0112122621D226944122772
:10AAB0000A704A466F443A704C48B361012201F073
:10AAC0008BFD1722390001236A44484801F08CFDB0
:10AAD0002A00E3680F219A406B469D207261DB7D5E
:10AAE0006944087004AFAB433B704048B261012237
:10AAF00001F072FD1722390001236A443B4801F03E
:10AB000073FDE36815219D408D2375616944162707
:10AB1000D0260B70002336066F443B700122B561CE
:10AB20003248984601F058FD1722012539000123CB
:10AB30006A442E4801F058FD2B00E268132193402F
:10AB4000A222694473610A70424605AF3A702748F1
:10AB5000B361013201F040FD172201236A4439003C
:10AB6000224801F041FDE36801209D40756107B076
:10AB70000CBC90469946F0BD69469220073102AF61
:10AB800008703A701948B361073A01F025FD1722A1
:10AB900001236A443900154801F026FD2B00E268C4
:10ABA0009340736161E70D211D2269440E270A70ED
:10ABB00000226F443A7025620132B3610B4801F004
:10ABC0000BFD1722390001236A44084801F00CFDEF
:10ABD0002A00E3680B219A409D206B46694472610C
:10ABE00008700120DB7D03AF03437DE700C0034015
:10ABF000F0B50124D6464F4646462300C0B5C2688C
:10AC000084B00500934000293DD00F226A4490464D
:10AC1000826A002A17D06A46D026D11DC02202AF10
:10AC20000A703606803A3A704448B3613F3A01F000
:10AC3000D3FC012342463900404801F0D5FC2300F3
:10AC4000EA6893407361092181220A26D02469446D
:10AC50000A706E440232240632703848A361823A88
:10AC600001F0BAFC012342463100344801F0BCFC3B
:10AC70000123EA6893406361012004B01CBC904644
:10AC80009946A246F0BD092181220A27D0266944AF
:10AC90000A706F44360602323A702848B361823A2D
:10ACA00001F09AFC0F236B44984639000123424679
:10ACB000224801F099FCEB6812229C400B27924637
:10ACC000113A74616F4403AE914603E00020F7F738
:10ACD000EFFEEB6852463A70002232704A46D024AA
:10ACE0009A402406A26139000122144801F074FC44
:10ACF000012342463100114801F076FC4B46EA68D8
:10AD0000934042466361117808220A42DED00D2149
:10AD10000E26922069446E44087032700748A36181
:10AD2000012201F059FC012342463100034801F0A1
:10AD30005BFC4A46EB689A4062619DE700C00340B5
:10AD4000F0B5DE4657464E464546E0B58BB06B46FD
:10AD50008A46D91D12230B7002AB984600239946F0
:10AD6000012643464A461A703300C268D0279340F2
:10AD700027243F060500BB6101226C44B74801F05F
:10AD80002BFC012322004146B44801F02DFC330086
:10AD9000EA6893407B61227890465246002A00DCA4
:10ADA00037E10D211D2269440A700F3A6A44484672
:10ADB000934610702E620122BB61A84801F00CFC82
:10ADC000012322005946A54801F00EFC3200EB6831
:10ADD0000B219A409D2069447A61087003A881463E
:10ADE00001202378034348460370BA619B4801223F
:10ADF00001F0F2FB494601232200984801F0F4FBE0
:10AE00003300EA6809219340A22269447B610A70F9
:10AE1000983A6A44504691461070BB6101228F48AF
:10AE200001F0DAFB4946012322008C4801F0DCFBEB
:10AE3000EB6815219E4092237E61D02742466944EB
:10AE40000B7099467C3B6B443F069A461A70BE6174
:10AE500001260122814801F0BFFB01232200514657
:10AE60007E4801F0C1FB3300EA68132193404A4653
:10AE700069447B6140460A7005AA91461070BB6127
:10AE80000122764801F0A8FB0123220049467348BD
:10AE900001F0AAFB3200EB6841469A4060237A61D8
:10AEA0000B40402B00D073E000202B6AE861002BA0
:10AEB00066D1192113206944087007306844804620
:10AEC0000370BA616548012201F086FB4146012307
:10AED0002200624801F088FB3300EA681F2193409A
:10AEE0007B612278694490461022D0270A700022A4
:10AEF0003F0608AE32705948BB61013201F06CFB6D
:10AF00003100012601232200544801F06DFB33007B
:10AF1000EA681D2193408D2069447B6108706F3879
:10AF20006844814622780270BB6101224B4801F0DF
:10AF300053FB494601232200484801F055FB3300EA
:10AF4000EA681B21934007A88122814669447B61FE
:10AF50000A700270BB61803A404801F03DFB01235A
:10AF6000220049463D4801F03FFBEB689E407E6170
:10AF700040460BB03CBC90469946A246AB46F0BD5D
:10AF80001721222369440B7006AB9846187098E786
:10AF900022236B44984621210023404669440370D4
:10AFA0000E702E48BA61012201F016FB41460123C2
:10AFB00022002A4801F018FB3300EA680021934080
:10AFC0007B6122788846862AD2D08D222531694439
:10AFD0000A70673A6A44404691461070BB6101228C
:10AFE0001E4801F0F9FA4946012322001B4801F0EE
:10AFF000FBFA3300EA6823219340812269447B6194
:10B000000A7009AA9146862248460270BB61853AB9
:10B01000A2E74A4611212A621D2269440A700B3AAE
:10B020006A44484692461070BB6101220B4801F009
:10B03000D3FA012322005146084801F0D5FA320024
:10B04000EB680F219A409D207A612378694408704B
:10B05000B34304A803708146BA61DFE600C0034031
:10B06000F0B5C64600B582B06B46591D1A230B7069
:10B07000143B6B449846012442460023137023007E
:10B08000C268D02793403F060500BB6101221148EA
:10B0900001F0A2FA6B46DE1D3200414601230D4845
:10B0A00001F0A2FAEB689C407C61A869FBF738FDCF
:10B0B0008022094BD205FBF705FD431E9841434210
:10B0C0000720347818409D30201A02B004BC904606
:10B0D000F0BDC04600C00340DD4ABF41F0B5CE46DA
:10B0E000474680B585B06B468946591CC02301246C
:10B0F00000270B70BE3B6B441F7098462300C2684C
:10B10000D02593402D060600AB6101224E4801F088
:10B1100063FA0F2201236A4441464B4801F064FA66
:10B120002300F26893404A466B61002A67DD6A4655
:10B13000D11D1D220A7002AA177034629046AB61BD
:10B140000122414801F048FA0F2201236A44414696
:10B150003D4801F049FA2200F36869469A409D2073
:10B1600005316A61087068466B46871D0120DB7BEC
:10B1700003433B703448AA61012201F02DFA0F22EB
:10B18000390001236A44304801F02EFA2300F268A6
:10B1900001AF93406A46D11CA2226B610A704A46F5
:10B1A0003A70AB610122284801F016FA0F223900EB
:10B1B0006A440123244801F017FAF3680D219C40EA
:10B1C0000E276C618123D02569440B706F440433D2
:10B1D0002D063B700122AC611B4801F0FDF90F22E6
:10B1E00001236A443900184801F0FEF90123F2688E
:10B1F00093406B6105B00CBC90469946F0BD0B21A5
:10B200001D2269440A7003AA177037629046AB6129
:10B2100001220D4801F0E0F90F2201236A44414662
:10B22000094801F0E1F92200F36809219A406B46D0
:10B230000A279D206A61DB7B69446F44A343087041
:10B240003B70AA61AEE7C04600C00340F0B5CE46F1
:10B2500047460500012080B5EB6885B09840002A7C
:10B2600025D10B000E2900DDA5E06A46D11C8922FC
:10B270000A70DA43D2171340D026702201AC134370
:10B28000360623700122B0614E4801F0A5F90F2265
:10B2900001236A4421004B4801F0A6F90123EA6822
:10B2A0009340736105B00CBC90469946F0BD1129DE
:10B2B00029DD142900DD80E06B46CC1ED91DCD238D
:10B2C00002AE0B70463B3370D0230F271B069861EC
:10B2D00001223C48984601F07FF9310001266F4475
:10B2E00001233A00374801F07FF93300EA689340C0
:10B2F000424653616A46511D8B220A70853A6A4460
:10B300009146312227E00C00022958DB0B21CD2386
:10B3100069440B7003AE493B3370D0230F271B06E3
:10B32000986101222748984601F056F9310001261C
:10B330006F4401233A00234801F056F93300EA68CC
:10B3400009219340424653618B2269440A70813A35
:10B350006A4491462B22484602704246194893613E
:10B36000012201F039F901233A004946154801F05C
:10B370003BF93300EA680D2193404246536189222C
:10B380000E2669440A700A3AFF3A023C14436E449E
:10B390003470D0242406A36181320A4801F01CF9DC
:10B3A00001233A003100074801F01EF90123EA6841
:10B3B0009340636176E70E2357E714217CE702246C
:10B3C000A4E7C04600C00340F0B54546DE465746F8
:10B3D0004E46E0B5050087B0052900DC0AE10C29DE
:10B3E00000DDFCE0062900D104E109014BB29846DA
:10B3F0000921B12369440B70A73B6B449946012690
:10B400004A46C32313703300EA68D02793401724B9
:10B410003F06BB6101226C44944801F0DDF84946C7
:10B4200001232200914801F0DFF83300EA689340DD
:10B430006A46D11DB7227B610A7002AA91460A2290
:10B4400048460270BB61093A884801F0C5F80123FB
:10B4500022004946854801F0C7F83300EA68934066
:10B460007B610D211E2269440E26D0270A7000221E
:10B470003F066E4432709146BB6101327B4801F059
:10B48000ABF83100012601232200784801F0ACF826
:10B490003200EB680B219A409E2369447A610B705D
:10B4A00003AB9A460F23207803404046184303001D
:10B4B00050460370BA616D48012201F08DF80123F6
:10B4C00022005146694801F08FF83300EA680F21E5
:10B4D00093401D2269447B6148460A7004AA904645
:10B4E0001070BB610122614801F076F8012322004F
:10B4F00041465E4801F078F83200EB689A407A6184
:10B5000023781B11092B6EDC59499B005B58994627
:10B5100013211E236944D0270B7000233F0605AE7C
:10B5200033705248BA6101229B4601F055F8310050
:10B530000126012322004D4801F056F83300EA6845
:10B54000112193407B6122786944924626220A7039
:10B55000143A6A44584690461070BB610122434831
:10B5600001F03AF8414601232200404801F03CF83E
:10B570003300EA68310093407B61984653461B11C3
:10B5800099404846FAF7C0FF0100FA20800027786A
:10B59000FAF7BAFF10282ADC08239F431521A623B7
:10B5A00069440B70903B6B44D0261F70994643460C
:10B5B0003606B36101222D4801F00EF82200012366
:10B5C00049462A4801F010F80123EA689340736164
:10B5D00007B03CBC90469946A246AB46F0BD40231E
:10B5E0005B42984604E701235B42994690E70823B3
:10B5F0001F43D3E76B46591DB1230B70AB3B6B4424
:10B60000984601264246C52313703300EA68D027C6
:10B61000934017243F06BB6101226C44134800F09D
:10B62000DBFF414601232200104800F0DDFF33001C
:10B63000EA6893406A46D11CB7227B610A7001AA6E
:10B6400090460C2240460270BB610B3A074800F05E
:10B65000C3FF012322004146044800F0C5FF330028
:10B66000EA68934060227B619046FAE600C003409E
:10B67000CCCD0010F0B5DE46454657464E46E0B507
:10B68000050085B00800FBF74BFA974B0022060037
:10B690000F00FBF71DFA00239846002855D1934B65
:10B6A000002230003900FBF713FA102398460028D7
:10B6B0004BD18F4B002230003900FBF709FA2023D1
:10B6C0009846002841D18B4B002230003900FBF70F
:10B6D000FFF930239846002837D1874B00223000ED
:10B6E0003900FBF7F5F94023984600282DD1834B0C
:10B6F000002230003900FBF7EBF950239846002870
:10B7000023D17F4B002230003900FBF7E1F96023A1
:10B710009846002819D17B4B002230003900FBF7F6
:10B72000D7F97023984600280FD1774B00223000BC
:10B730003900FBF7CDF9431E98410F227023404298
:10B7400090435B4280469C46E0446B46591D1D2356
:10B750000B709A46173B6B449B4600239946012683
:10B760005B464A461A703300EA68D02793400F249C
:10B770003F066C44BB610122644800F02DFF59462E
:10B7800001232200614800F02FFF3200EB689A404D
:10B790006B46D91C9D237A610B7001AB9B460F232E
:10B7A0002078034040461843030058460370BA61AE
:10B7B0005648012200F010FF594601232200534849
:10B7C00000F012FF3300EA68484693406A46D11DF4
:10B7D00052467B610A7002AA90461070BB6101223A
:10B7E0004A4800F0F9FE012322004146474800F094
:10B7F000FBFE3200EB689A407A6123781B11092B1B
:10B800006ADC43499B005B5899460B211E2369441F
:10B81000D0270B7000233F0603AE33703B48BA615C
:10B8200001229B4600F0D8FE3100012601232200B0
:10B83000364800F0D9FE3300EA68092193407B6165
:10B8400022786944924626220A701C3A6A44584675
:10B8500090461070BB6101222C4800F0BDFE4146AD
:10B8600001232200294800F0BFFE3300EA683100BE
:10B8700093407B61984653461B1199404846FAF71E
:10B8800043FE0100FA2080002778FAF73DFE1028D9
:10B8900026DC08239F430D21A62369440B70983BA7
:10B8A0006B44D0261F70994643463606B361012289
:10B8B000164800F091FE220001234946134800F08B
:10B8C00093FE0123EA689340736105B03CBC904647
:10B8D0009946A246AB46F0BD01235B42994694E7E8
:10B8E00008231F43D7E7C0460078BE400050C4403D
:10B8F0000078CE400050D4408084DE40805CE4403C
:10B900008084EE408084FE4080840E4100C003406D
:10B91000CCCD0010F0B5CE46474680B5050083B0CB
:10B920000C00082900DD08246B46591D1D230B70EF
:10B93000173B6B44994600234A461370EA6801336B
:10B94000D027984693403F06BB610122194800F07A
:10B9500043FE6B46DE1D320001234946154800F0C8
:10B9600043FE4346EA68694693409D207B6103316C
:10B970003278087001AF052C00DA05240E20043C53
:10B980008243640014433C70D0242406A361012246
:10B99000084800F021FE320001233900054800F07C
:10B9A00023FE0123EA689340636103B00CBC904618
:10B9B0009946F0BD00C00340F0B5CE46474680B57D
:10B9C00083B06B468946591DA0230B709A3B6B448C
:10B9D00098464B46424601241B1213702300C2684E
:10B9E000D0259340174E2D060700AB610122300091
:10B9F00000F0F2FD6A46414601230732300000F0B4
:10BA0000F3FD2300FA68484693406A46D11CA12200
:10BA10006B610A7001AA10709046AB610122300080
:10BA200000F0DAFD6A46012307324146300000F09B
:10BA3000DBFDFB689C406C6103B00CBC90469946F2
:10BA4000F0BDC04600C00340F0B5CE46474680B5C5
:10BA500083B06B46591D1E230B70183B6B449946EF
:10BA600001244A46002313702300C268D025934066
:10BA7000194E2D060700AB610122300000F0ACFD2D
:10BA800007236B449846494642460123300000F0A4
:10BA9000ABFD2200FB6869469A409E200331434675
:10BAA0006A61087001A8814604201B780343484658
:10BAB0000370AA613000012200F08EFD012342468E
:10BAC0004946300000F090FDFB689C406C6103B07B
:10BAD0000CBC90469946F0BD00C0034009490A4B92
:10BAE000083119600949002299600821D9600331A1
:10BAF000196101395A6059619A61DA611A625A62B0
:10BB00009A627047F4CD0010B01E002000C00340C0
:10BB100010B5062000F06AFB0120F7F78FFDC04644
:10BB2000F0B557464546DE464E46E0B50D000B35AE
:10BB300083B00700162D28D8102900D9C1E000F0E5
:10BB4000A7FA102518230220CE4EF3181A005C68BD
:10BB5000083A944200D160E1032362689A431300DB
:10BB6000E268A168CA6091600122E3185968380050
:10BB70000A435A6000F08EFA2000083003B03CBC43
:10BB800090469946A246AB46F0BD07239D4300D59B
:10BB900097E0A94200D994E000F07AFAF823FF3345
:10BBA0009D4200D85EE1680A00D18EE0042800D9E9
:10BBB00039E138239846A80980443930C100B14E94
:10BBC00071180839CC68A14218D0032362689A43DF
:10BBD0001300521B0F2A00DD1DE1002AC0DA0323E7
:10BBE0009C4608E06246636893435A1B0F2A00DDB7
:10BBF00011E1002AB4DAE468A142F3D132003469D9
:10BC00000832944267D00323616899438A460B0047
:10BC1000491B0F2900DD12E1726132610029A3DAAC
:10BC2000994A924500D948E1DB08FF3A9910FF3A5A
:10BC30008A40DB0071689B190A4399687260E3606F
:10BC4000A1609C60CC60012183109940914248D84A
:10BC50000A4205D103239843490004300A42FBD02D
:10BC600003239846C3009946B144CC4682466346B6
:10BC7000DC68A44507D1F9E0002A00DB0EE1E468A6
:10BC8000A44500D1F2E04246636893435A1B0F2A51
:10BC9000F2DD01208046611905436560A068E56812
:10BCA0000836C560A8604046F160B1601043486046
:10BCB000CE608E603800E25000F0ECF920000830D1
:10BCC0005CE70C2300203B6058E780213F2389007C
:10BCD0004020984673E70121726883109940914291
:10BCE000B6D90323B46862689A439046AA4203D344
:10BCF000531B0F2B00DD80E0644B654A9A46934648
:10BD00001B681268EB18013200D138E1614A944691
:10BD100063441B0B1B0300930099380000F0BCF92F
:10BD200003008146013300D1F6E04346E218824227
:10BD300000D9EFE051464968009B8C465146634468
:10BD40004B60824200D14BE159460968013100D174
:10BD50005DE149468A1AD3185246536007234A4682
:10BD60001A40019200D120E108214B4689469B1AD6
:10BD700099440099484B49449B1A5B1A1B051B0DBB
:10BD80000091380019009B4600F086F9431C00D151
:10BD90005AE1534652465B6849465B4453604A4603
:10BDA000B260801A0122584410434860B44211D056
:10BDB00041460F2900D827E107200C3981436068EC
:10BDC000024005200A4362606218506090600F29AB
:10BDD00000D941E15246D26A934201D95246D36218
:10BDE0000322B468616891430A005146096B8B4293
:10BDF00000D895E051460B6392E0012229001343DD
:10BE00001143651961603800B5606B6000F042F95C
:10BE100020000830B2E64046F0E6DC680230A3427B
:10BE200000D1EBE698E614286ED9542800D9A9E091
:10BE30006E239846280B80446F30C100BFE6012373
:10BE400060191D43656070613061C26082601A00D4
:10BE500053460A4342603800E15000F01BF92000CD
:10BE600008308BE62B00E80808336DE608239B4674
:10BE7000073BDC449B46DA4443465246134200D01B
:10BE8000F5E667E028190020FF0100007C1E002075
:10BE9000201900200F100000081000000122E318F4
:10BEA000596838000A435A60E368A268D3609A6010
:10BEB00000F0F0F82000083060E65A0A042A3AD967
:10BEC000142A00D983E05B23984690445C32D20068
:10BED00008235B429C46B218944463469968032346
:10BEE00099468C4559D04B464A689A43524502D9E7
:10BEF00089688C45F7D1CB6872689C466346A1601F
:10BF0000E3609C60CC609EE65B23984680445C3096
:10BF1000C10054E6B4427ED00323B46862689A43F9
:10BF2000531B954202D80F2B00DD66E7380000F066
:10BF3000B1F8002022E69A09382398469044393215
:10BF4000D200C5E74B461A68083B013891469A4231
:10BF500000D098E043460342F4D173688B4373608A
:10BF60004900994200D9BCE6002904D1B9E604226F
:10BF700094464900E2440B42F9D0504672E6103331
:10BF80000093C9E6AA235B00984233D8DD3B98466C
:10BF9000E80B80447830C10011E6434601229B1033
:10BFA0009A4073681A437260A8E7009B38004B44BC
:10BFB00000931B055B421B0D19009B4600F06CF8BB
:10BFC000431C00D0E5E6002300989B46E1E6542A96
:10BFD00029D81A0B6E23984690446F32D20077E727
:10BFE000110500D0B0E60120009AB1684244024336
:10BFF0004A60EFE6254B984220D87C239846A80C4F
:10C0000080447D30C100DAE54B465A608EE75B46DE
:10C010004A461A60A2E651464968009B8C46514642
:10C0200063444B6090E6AA2149008A421CD8DA0B8F
:10C030007723984690447832D20049E7FE217E2348
:10C0400089007F209846BAE5009B01989C46002312
:10C05000083860449B469CE621003800083100F017
:10C060008FF953465B68B5E608498A4206D89A0CB0
:10C070007C23984690447D32D20029E7FE227E231D
:10C080009200984624E773686AE7C04654050000AA
:10C090007047C0467047C046002370B5064C050087
:10C0A00008002360F7F7CCFA431C00D070BD23686A
:10C0B000002BFBD02B60F9E74C2D002010B5802120
:10C0C0000400FFF72DFDB7239B00E050002807D0A8
:10C0D00002000023803208C09042FCD1002010BD35
:10C0E00001204042FBE7C046B7239B00C25810B571
:10C0F0000023002A01D0180010BDFFF7DFFF030066
:10C10000F9E7C046F8B505000C0016001F2909D84C
:10C11000B727BF00C359002B09D0A4001C19206801
:10C120002660F8BD1623036001204042F9E7FFF7BF
:10C13000C5FF002801D1EB59EFE701204042F0E7AD
:10C1400070B505000C001F2922D8B7239B00C358E7
:10C15000002B0ED08A009B181A68002A09D0012AE9
:10C1600010D0511C10D000212000196090470020F1
:10C1700070BD280000F07EF822000100280000F0C9
:10C1800065F8F5E70020F3E7162303600120EFE7E9
:10C190001623036001204042EAE7C04670B505005F
:10C1A0000C001F291DD8B726B6008359002B10D0CC
:10C1B000A2009B181A68002A09D0511C0FD0012A2E
:10C1C00012D00021200019609047002070BD01208E
:10C1D000FCE7FFF773FF002803D1AB59E8E7022023
:10C1E000F4E701204042F1E70320EFE710B5034BED
:10C1F00001001868FFF7A4FF10BDC046F01400202E
:10C2000010B5044B0A001B6801001800FFF77AFF05
:10C2100010BDC046F0140020B722064B92001B68E8
:10C2200010B59A580020002A00D010BD1800FFF762
:10C2300045FFFAE7F014002010B5034B0100186821
:10C24000FFF7ACFF10BDC046F0140020002370B50E
:10C25000074C050008001100236000F083F9431C1F
:10C2600000D070BD2368002BFBD02B60F9E7C046DF
:10C270004C2D002010B500F06DF910BD10B5040074
:10C2800083070AD00378002B23D0032202E003782F
:10C29000002B1CD001301042F9D102680E4B0F491F
:10C2A000D31893430B420FD1043002680A4BD318C2
:10C2B00093430B4208D104300268074BD3189343D1
:10C2C0000B42F1D000E001300378002BFBD1001BC2
:10C2D00010BD0020FCE7C046FFFEFEFE808080808F
:10C2E000F8B50C000600FFF7D3FE204FBB685D6871
:10C2F00003239D431E4B2C1B9C466444240B1D4B67
:10C30000013C24039C4207DD00213000FFF7C4FEFE
:10C31000BB685B19984204D03000FFF7BBFE0020D9
:10C32000F8BD61423000FFF7B7FE431C0DD001227B
:10C33000BB682D1B15435D600F4B30001A68141B42
:10C340001C60FFF7A7FE0120EAE700213000FFF79D
:10C35000A3FEBA68831A0F2BDEDD08490968401A6C
:10C360000549086001210B435360D5E728190020D7
:10C37000EF0F0000FF0F0000801E0020201900209A
:10C38000F8B5CE464746050080B50C1E55D0FFF7E0
:10C390007FFE210008394F68012438000323A043A1
:10C3A0000A1856689E43B146644EB368934229D03A
:10C3B0004B465360D3189C463C4242D10F68C91B80
:10C3C0008B68C019984663465F6808239C46B4444E
:10C3D0002740E0456AD04346CC68DC60A360002F6C
:10C3E00032D1012448440443A0469368544C0F18AA
:10C3F000A34200D17FE0D268DA60936043464B608D
:10C40000386025E003004B443C4206D10A68891A93
:10C4100088689B18CA68C260906001221A434A600B
:10C42000484AB16012689A4204D8474B28001968FC
:10C43000FFF756FF2800FFF72DFE0CBC90469946EB
:10C44000F8BD5F682740CCD0012303434B60085000
:10C450003E4B98421AD9430A042B33D88209140060
:10C4600039323834D200B218083A936803279A4216
:10C4700039D05C68BC43844233D99B689A42F8D176
:10C48000D368CB608A609960D160D3E7C008FF3B76
:10C490008210FF3B93407268C0001343736086199B
:10C4A000B368CE608B60B160D960C3E7002F41D123
:10C4B000030090684B44D2681C43C26090604C609B
:10C4C000CB50B7E7142B07D9542B1CD8020B140000
:10C4D0006F326E34D200C6E71C005C335B34DA0086
:10C4E000C1E71A00CCE70123A410A34070680343FE
:10C4F00073601300C5E7D9609960CB608B604346D9
:10C500004B60386096E7AA225200934205D8C20BCE
:10C51000140078327734D200A5E70D4A934205D84B
:10C52000820C14007D327C34D2009CE7FE227E24F3
:10C53000920098E704434C6010607BE728190020C4
:10C5400030190020241900207C1E0020FF0100006B
:10C550005405000058220120014B40421A607047E8
:10C560004C2D002058220120014B40421A60704798
:10C570004C2D0020F8B5C04601B40248844601BCE9
:10C58000604700BF8D02002001B40248844601BC10
:10C59000604700BFE901002001B40248844601BCA5
:10C5A000604700BFDD03002001B40248844601BC9F
:10C5B000604700BFDD03002001B40248844601BC8F
:10C5C000604700BF0901002001B40248844601BC55
:10C5D000604700BF5101002001B40248844601BCFD
:10C5E000604700BF9103002001B40248844601BCAB
:10C5F000604700BF3903002001B40248844601BCF3
:10C60000604700BFC100002001B40248844601BC5D
:08C61000604700BFC9120020C1
:10C618008A2100109C1300108A2100108A21001022
:10C628008A2100108A210010400F00108A21001072
:10C638008A2100108A2100108A2100108A21001006
:10C648008A2100108A2100108A2100108A210010F6
:10C658008A2100108A2100108A2100108A210010E6
:10C668008A2100108A2100108A2100108A210010D6
:10C678008A2100108A2100108A2100108A210010C6
:10C688008A2100108A2100103E0E0010F80E0010BA
:10C69800A60E00108E0E0010BE0E0010760E0010B2
:10C6A800D60E0010540E001030303030300000002C
:10C6B8004C6F52612073657474696E67733A000039
:10C6C8006C6F72614672657175656E6379202020A2
:10C6D800202020203D2025750A0000006C6F726123
:10C6E800537072656164696E67466163746F722026
:10C6F8003D2025690A0000006C6F72615072656107
:10C708006D626C6520202020202020203D20256996
:10C718000A0000006C6F7261436F64696E67526152
:10C7280074652020202020203D2025690A00000073
:10C738006C6F72615478506F7765722020202020CA
:10C74800202020203D2025690A0000004C6F5261FE
:10C75800506153656C6563742020202020202020C0
:10C768003D2025690A0000006C6F726142616E64A9
:10C778007769647468202020202020203D202575BA
:10C788000A0000005374617274696E67204C6F521E
:10C798006120726164696F0020205B204641494C2A
:10C7A8004544205D0000000020205B20444F4E459A
:10C7B800205D0000415052532073657474696E67A0
:10C7C800733A00004D792063616C6C3A2025730A36
:10C7D800000000005365727665722063616C6C3AE4
:10C7E8002025730A00000000536F7572636520618D
:10C7F8006464726573733A2025730A4469676970C3
:10C8080065617465727320282575293A202573207F
:10C8180025732025732025730A446174613A202505
:10C82800730A00004D6573736167652066726F6DEA
:10C83800207365727665723A2025732028636F6DC0
:10C848006D616E64202575290A00000041636B6ED6
:10C858006F776C6564676520726571756573743A86
:10C868002025730A000000004572726F722064650B
:10C87800636F64696E672041505253206672616D20
:10C88800652E000052656365697665642070616392
:10C898006B6574202852535349203D202569644212
:10C8A8006D290A004552524F523A204E6F206F723E
:10C8B80020636F7272757074656420415052532002
:10C8C8006672616D652E00004E6F207370696E6C24
:10C8D8006F636B732061726520617661696C616258
:10C8E8006C650000486172647761726520616C61F3
:10C8F800726D20256420616C726561647920636CB7
:10C9080061696D6564000000486172642061737339
:10C91800657274000A2A2A2A2050414E4943202A67
:10C928002A2A0A005A5300101253001012530010FA
:10C9380052530010125300101253001012530010DB
:10C94800125300101253001012530010125300100B
:10C9580042530010125300104A5300101253001093
:10C9680012530010FC520010A4530010E25A001099
:10C9780098530010E25A001084530010E25A001035
:10C98800E25A0010E25A0010E25A0010E25A00106F
:10C99800E25A0010E25A001068530010E25A0010E0
:10C9A800E25A0010E25A0010E25A0010E25A00104F
:10C9B80068530010F0530010A2520010A252001049
:10C9C800A2520010A2520010A2520010A25200104F
:10C9D800A2520010A2520010A2520010A25200103F
:10C9E800A2520010A2520010A2520010A25200102F
:10C9F800A2520010A2520010A2520010A25200101F
:10CA0800A2520010A2520010A2520010A25200100E
:10CA1800A2520010A2520010A2520010A2520010FE
:10CA2800A2520010A2520010A2520010A2520010EE
:10CA3800A25200100A570010B65300100A570010EF
:10CA4800A2520010A2520010A2520010A2520010CE
:10CA5800A2520010A2520010A2520010A2520010BE
:10CA6800A2520010A2520010A2520010A2520010AE
:10CA7800A2520010A2520010A2520010A25200109E
:10CA880098550010A2520010A2520010A252001095
:10CA9800A2520010A2520010A2520010A25200107E
:10CAA800A2520010A2520010985500102C550010E8
:10CAB800985500100A570010B65300100A57001076
:10CAC800A252001098550010A2520010A252001055
:10CAD800A2520010A2520010A25200109855001045
:10CAE800BC540010A2520010A252001000540010B2
:10CAF800A252001098550010A2520010A252001025
:10CB0800985500106E616E00666E692D0000000079
:10CB1800666E692B00000000666E69000000000068
:10CB2800000000000000F03F00000000000024406A
:10CB380000000000000059400000000000408F4045
:10CB4800000000000088C34000000000006AF840B0
:10CB58000000000080842E4100000000D0126341D4
:10CB68000000000084D797410000000065CDCD414A
:10CB780006005250BBFF3CB6BCCB0010060052501A
:10CB8800E182887FA4CB001006005250D3F0754292
:10CB98009CCB001052656C6561736500626F6F74A1
:10CBA800325F77323571303830000000312E332E45
:10CBB800300000007069636F000000006D61696EED
:10CBC80000000000417072203239203230323200C9
:10CBD8000D0A000071760010757600108576001039
:10CBE800AD7600108176001000000000060052505B
:10CBF80053B4F4A100CC00105553422073746469F7
:10CC08006E202F207374646F757400005261737006
:10CC18006265727279205069000000005069636F84
:10CC280000000000426F617264204344430000002A
:10CC38005265736574000000090254000301008006
:10CC48007D080B0002020200000904000001020234
:10CC58000004052400200105240100010424020227
:10CC680005240600010705810308001009040100D6
:10CC7800020A0000000705020240000007058202C0
:10CC88004000000904020000FF0001051201000233
:10CC9800EF0201408A2E0A00000101020301000090
:10CCA8000000000014CC001024CC0010702A0020D2
:10CCB8002CCC001038CC0010556E68616E646C6521
:10CCC800642049525120307825780A006570202563
:10CCD800642025732077617320616C7265616479C3
:10CCE80020617661696C61626C65000043616E2742
:10CCF8007420636F6E74696E75652078666572203E
:10CD08006F6E20696E616374697665206570202591
:10CD180064202573000000006F757400696E0000C0
:10CD2800E484001058870010CA860010748600102A
:10CD3800568600103E8600108E8500103285001041
:10CD480026850010328A0010188A00107288001098
:10CD5800528A001072880010008A0010EC890010B6
:10CD680072880010D8890010AE89001072880010EF
:10CD7800E28A0010B68A0010AA8A00107288001091
:10CD8800728800108C8A0010B68A00107288001011
:10CD98007288001072880010728800107288001063
:10CDA80072880010728800106C8A0010F1950010CB
:10CDB8006D960010999600107D97001061980010EC
:10CDC80000000000781E0000A0280000F03C0000D1
:10CDD80040510000127A0000E4A2000024F4000090
:10CDE80048E8010090D0030020A1070000000000DF
:10CDF8000000000069A2001019A40010FDA1001095
:10CE080001A2001005A200105DA3001031A50010BA
:10CE1800080052500A38A5040900525000010000C9
:0CCE28002CCE0010535049204353000052
:10CE3400A0B20181ABF080010000000080140181E8
:10CE4400B0B0ABF00000000080020181B0B0AB30A4
:10CE54000000000080040181B0B0AB30000000008D
:10CE640080010181B0B0AB10000000008006018198
:10CE7400B0B0ABF00000000080030181B0B0AB7033
:10CE84000000000080080181B0B0ABF00000000099
:10CE940080060181B0B0AB30000000008003018146
:10CEA400B0B0AB7000000000800A0181B0B0ABF0FC
:10CEB4000000000080010181B0B0AB100000000050
:10CEC40080040181B0B0AB30000000008004018117
:10CED400B0B0AB300000000080060181B0B0ABF010
:10CEE4000000000080040181B0B0ABF0000000003D
:10CEF40080020181B0B0AB300000000080020181EB
:10CF0400B0B0AB300000000080020181B0B0AB30A3
:10CF14000000000074B20181B0AB3080000000005A
:10CF2400800A0181B0B0ABF0000000003F02018133
:10CF3400B0AB30800000000080060181B0B0ABF0DF
:04CF440000000000E9
:10CF48001434FF7FB0B0A8803C34FF7FAB70808082
:10CF58004035FF7FAB1080800039FF7FD0FEFF7F18
:10CF6800343DFF7F01000000443DFF7FCCFEFF7F82
:10CF78002452FF7F0100000084D2FF7FC8FEFF7F9C
:10CF8800E0D2FF7FCCFEFF7FCCD3FF7FD0FEFF7FB8
:10CF980080D4FF7FD4FEFF7F90D5FF7FD8FEFF7F30
:10CFA800B4D6FF7FDCFEFF7F28DAFF7FE0FEFF7F3D
:10CFB80038DCFF7FE4FEFF7F80DDFF7FE8FEFF7F38
:10CFC80098E0FF7FECFEFF7F0CE1FF7FF0FEFF7F24
:10CFD80074E2FF7FF4FEFF7FE8E3FF7FF8FEFF7F48
:10CFE8008CE6FF7FFCFEFF7F24E9FF7F00FFFF7FC9
:10CFF800C0E9FF7F04FFFF7F48EAFF7F08FFFF7F4C
:10D00800D4EAFF7F010000008434FF0FB0A902803A
:10D018001835FF0FB0B0A8806435FF0F010000007D
:10D028007035FF0FB0B0AA80A435FF0FE4FEFF7F74
:10D038006436FF0F010000006036FF0FAA3F3980F9
:10D04800AC36FF0FB0B0A880B836FF0FB0B0AA80DA
:10D05800F836FF0FB0B0A8800C37FF0F01000000B2
:10D068000837FF0FB0B0A8801037FF0F010000008D
:10D078009837FF0FAA0FB2800038FF0FA0FEFF7F7E
:10D08800D83AFF0FB0B0A880F43AFF0F9CFEFF7F9C
:10D09800503DFF0F01000000C03EFF0F00840480D8
:10D0A800D03EFF0FB0B0A880D03EFF0F88FEFF7FB4
:10D0B800B841FF0F00840480D841FF0FB0B0A880AA
:08D0C800F041FF0F0100000020
:10D0D000B4020010A80200109C02001078CB0010CF
:10D0E0009002001084CB001090CB001018CE0010DE
:08D0F00020CE0010F4CB00106B
:10D0F800D02330B500251B065D57002406E00368E1
:10D10800BFF35F8F1C6081F3108820BF0268EFF3C4
:10D11800108172B61368002BFCD0BFF35F8F0379C0
:10D128007F2BECD905710368BFF35F8F00221A606B
:10D1380081F3108830BDC046030010B50068EFF3D6
:10D14800108472B60268002AFCD0BFF35F8F0422F5
:10D158009A56002A0BDB00290FD000200A601B68B2
:10D16800BFF35F8F00221A6084F3108810BDD022AD
:10D178001206126801201A71F1E70020EFE7C04695
:10D18800F0B5C64600B50C00070001F01DF9FA22FB
:10D1980005000E00920020000023002101F01CF978
:10D1A8002C002A00350024184D41AE422FD9012405
:10D1B8006442E517D0231B061B68002698460BE03F
:10D1C8003B68BFF35F8F1E6081F310882000290041
:10D1D80001F0EAF8002818D13A68EFF3108172B626
:10D1E8001368002BFCD0BFF35F8F3B797F2BE7D907
:10D1F80043463B713B68BFF35F8F00221A6081F39F
:10D208001088012004BC9046F0BD0020FAE7AE4229
:10D21800D0D1A242CBD8CDE70268EFF3108172B625
:10D228001368002BFCD0BFF35F8FFF2303710368E3
:10D23800BFF35F8F00221A6081F3108840BF7047E8
:10D2480030B5094C2378002B0DD1802307480849B5
:10D258005B05F0221D6812069A18043385508B422C
:10D26800F7D10123237030BD842A00208C220020AE
:10D278000001001010B5024B0133984710BDC0469D
:10D288008C220020054B1A6880239B005340C02243
:10D2980092001340024A13607047C0460C80014058
:10D2A8000C900140034B1A68C0239B009343024A29
:10D2B800136070470C8001400C900140F0B5D646D1
:10D2C8004F4646461423C0B51827984681460D0098
:10D2D800188822493B8814009847434682462049CB
:10D2E80018883B88984743461E49060018883B889B
:10D2F80098478046FFF7A4FFD047B047FFF7C2FF23
:10D30800C020220008264005163F230013431BD0E7
:10D318003100836A19401F420BD0002C09D0131B1F
:10D328000D2B06D84B461B78013C036601239C460F
:10D33800E1440029E9D0002AE7D0036E013A2B70B6
:10D34800230001351343E3D1FFF7ACFFC047FFF7D4
:10D3580091FF1CBC90469946A246F0BD4946000084
:10D368004558000046430000F0B5C6468C461D00EF
:10D378001C000221042700B526002E431BD0002DD7
:10D388000DD0C66831420AD02E000836A64206D90A
:10D3980066463678013D86600126B046C444002CB6
:10D3A800EAD0C6683742E7D08668013C1670260086
:10D3B80001322E43E3D1180004BC9046F0BDC046AC
:10D3C80030B50300002A09D002258818DC682542F8
:10D3D800FCD00C7801319C608842F7D1D9684907A4
:10D3E80004D504249968D9680C42FBD11024D96863
:10D3F8000C42FCD1D968490704D504249968D96836
:10D408000C42FBD101211000196230BD7047C046A3
:10D4180003685A0003D45B005B08C0187047802279
:10D4280012061343F9E7C046F0B557464E46DE46A6
:10D438004546E0B5814683B09246002925D04B1E6B
:10D448009B46002701935B46FB18DC0FE4184B460C
:10D458006410E5005E193000FFF7DAFF019B804693
:10D46800A3420BD0280008304844FFF7D1FFD0452D
:10D4780006D80138504509D2671CE4E7504505D95C
:10D48800A74202D0631E9B46DDE70026300003B0AA
:10D498003CBC90469946A246AB46F0BD012809D04F
:10D4A800022805D0002801D0002070470248FCE778
:10D4B8000248FAE70248F8E7610B0020790B0020E0
:10D4C8006D0B002030B5234B83B005008C1E002B5C
:10D4D80026D001A9200000E000BF00281CD0019937
:10D4E8002200FFF7A1FF041E16D0FFF791FF636823
:10D4F800A864012B2AD0201D002B23DBFFF788FF0F
:10D508000023E8642B650368002B0FDBFFF780FF1F
:10D518002861002003B030BD002309202B61F9E702
:10D528000D480E49091AC9100191D9E71801000FD1
:10D53800FFF7B4FF2861431E9841082340429843EF
:10D548000930E7E70123E8642B65DCE700230520C1
:10D558002B61DFE70000000048CF0010D0D000109A
:10D56800036810B50400DA0705D448309B070ED5C8
:10D5780000F06CFC23685A070ED51A0713D5DB0692
:10D5880004D42000D130FF3000F06CFC10BD00F056
:10D5980059FC23685A07F0D42000D03000F05AFC18
:10D5A80023681A07EBD420005130FF3000F056FCF6
:10D5B8002368E4E70368002B00D01B1818007047A5
:10D5C800092070477047C04670B504000D0008E098
:10D5D8002B6C2A00636121000120236998470828E1
:10D5E80007D1296C2000FFF76DFF0028F0D000F06C
:10D5F800E3FE0728FBD10020296CFFF7E3FF281D75
:10D6080000F00AFCF0B5CE46474680B5C3682E4CFC
:10D618009846A5448369060014000431402205A8F1
:10D62800994600F0B9FE002304AD049323E0F022EC
:10D638002B6C5200736129007CA800F0ADFE7CAA17
:10D6480031003369200098478A9B07006B64039375
:10D658004B46009501933200330021000120C0475A
:10D6680000281FD1F0227CA95200280000F094FE67
:10D678000024082F1FD1296C3000FFF723FF611EFB
:10D688008C41070009340028D1D0AB6B10216B64A2
:10D698004B46214301930095330032000120C047D7
:10D6A800002800D009273800F5239B009D440CBCB6
:10D6B80090469946F0BD072FF4D12000296CFFF75A
:10D6C80081FF05A800F0A8FB2CFCFFFF406C704709
:10D6D80070B5CB6BFAB00B6404000E004022043125
:10D6E80003A800F059FE01235B42029306E002AA58
:10D6F800210023699847050008280AD1129B2000B9
:10D7080019000193FFF7DEFE0028F0D009207AB057
:10D7180070BD02A8FFF724FF062DF7D131002000C5
:10D72800FFF752FF10B58261DA6BC1601A64190005
:10D738000022FFF767FF10BD436970B50B64C3682B
:10D7480004000D00002B15D10A00236901000220F6
:10D758009847072807D0082803D129002000FFF799
:10D7680033FF00F029FE0020296CFFF72BFF281D4E
:10D7780000F052FB0122FFF745FF00F01DFEC046F6
:10D78800C36810B5002B05D0CB6B00220B64FFF7E4
:10D7980039FF10BDFFF79CFFFBE7C0467047C04646
:10D7A800836810B5002B02D001000120984710BDF6
:10D7B800012906D0002906D003390220012900D901
:10D7C80070470120FCE7002B08D10F2A06D89200E9
:10D7D80082185268009B00201A60F1E70220EFE7E8
:10D7E80000B585B003AB0A00009300210023FFF7C2
:10D7F800DFFF039805B000BD012906D0002906D037
:10D8080003390220012900D970470120FCE7002BC9
:10D8180008D10F2A06D8009B92001B688218536013
:10D828000020F1E70220EFE700B585B003AB0392D3
:10D8380000930A0000230021FFF7DEFF05B000BDBA
:10D8480070B51A4CD36BA544136406000D0019A8D3
:10D85800111D402200F0A0FD01235B42189314E043
:10D868000C2118A802AAFFF7DFFF290018A8B04763
:10D87800002812D1069B18AA02A9083001939847DC
:10D88800040005280AD0092807D0289B02A81900F7
:10D898000193FFF717FE0028E2D0092418A8FFF724
:10D8A8005FFE200090239B009D4470BDC0FDFFFFDC
:10D8B800F0B5DE4657464E464546E0B5160003220B
:10D8C8000D0011008BB01F000193EB6C01401C1D73
:10D8D800009107A91B688B460894002F6BD01A0C7F
:10D8E8001B045946079302230B72FD3313409B0018
:10D8F8004A72E418009B022B00D1AC6B2B6DDB073E
:10D9080047D4002305930833034002932768002F68
:10D9180000D112E1019B022B49D0638827889846E1
:10D928000434012340469A469843AB6C0F2199462C
:10D9380081443000FFF754FF0021814506D83900A3
:10D9480053469943494488428941494243465A00CB
:10D9580002231340012217403B43012B3AD0002BEE
:10D9680030D0022B1BD12368009A5F007F08002A61
:10D9780067D1002906D0029A002A00D17CE0002F46
:10D9880000D1A9E0002B00DA04340137BF00E41904
:10D99800BCE75946300000F00BFB002810D00920E6
:10D9A8000BB03CBC90469946A246AB46F0BD6368B6
:10D9B80008349846B5E71B0207935B461A8199E736
:10D9C8000820EDE7009B002B02D0002900D08DE055
:10D9D80004349BE7009B002B1AD1002916D023683A
:10D9E800DF0F63689A1CDAD02A0058320692013396
:10D9F80000D1BDE0201DFFF7DDFD06AB01003A00B8
:10DA0800280000E000BF002800D082E008347DE74D
:10DA18000D2130002F6AFFF7E3FE8742F6D1AB6A8B
:10DA28009C42F3D12000FFF7F3FC0F2102003000E5
:10DA3800FFF7FAFE30002A000021FFF7F5FE072065
:10DA4800AEE72B6A0D2130009846FFF7C9FE8045E6
:10DA580001D0236896E7AB6A9C42FAD10023EB62B7
:10DA680004332B63231DAF626B632368002B00DA3A
:10DA780086E00123059388E7002F2DD058239C4684
:10DA8800AC4463460393231D99460023984606AB8E
:10DA9800220004933B004C464746B24698462E0067
:10DAA800914603E004342F00454542D0039B2000F3
:10DAB8000693FFF77FFD049B0100002230007D1CC8
:10DAC80000E000BF0028EDD04346B84635004C467C
:10DAD80056461F009845BCD10D213000FFF780FE47
:10DAE800069B28626B62AC62062059E72000FFF7AC
:10DAF8008FFC04340700AC63280000E000BF002856
:10DB080000D14CE730003A000F21FFF78DFE0720C7
:10DB180046E707000D213000FFF762FE2862022F5A
:10DB28002BD1069BEB622B002C336B62AC62062078
:10DB380036E735004C465646CEE75946300000F0E9
:10DB480037FA002800D02AE7059B002B00D137E7D9
:10DB58000F213000FFF744FE0E2102003000FFF7CE
:10DB680063FE3000094A0F21FFF75EFE072017E722
:10DB78000D213000FFF734FE2862069B6B62D5E763
:10DB880038000130800020184DE7C0460000000032
:10DB980010B50023FFF78CFE10BDC04610B5012359
:10DBA800FFF786FE10BDC04610B50223FFF780FEC2
:10DBB80010BDC046F0B5CE46474680B50500C3B097
:10DBC80014001E00012955D000294BD0032922D06A
:10DBD800042949D1002B47D1102A45D810220368BF
:10DBE8001A4200D0F1E020AF380000F03DF90023E0
:10DBF8000120A96B02009A40144203D00E689A00D3
:10DC0800BE5004310133042BF4D13800A96300F06D
:10DC180029F9002029E0032B26D11404230C160C23
:10DC28009846F318102B1FD8082203681A4200D010
:10DC380098E020AF380000F013F94246AB6BF600CD
:10DC48001C00002A08D0D400F21A1C19BA18196846
:10DC5800D15004339C42FAD1AC63380000F0FEF88E
:10DC6800002002E0002B24D0022043B00CBC9046D8
:10DC78009946F0BD130C14049846240C012E2ED09E
:10DC8800052EF1D11B19202BEED842460F2A70D948
:10DC9800A146002C7ED1AA6B4346AA630F2B00D85D
:10DCA8009AE04B46002BDBD0684600F0D3F8002002
:10DCB800DBE700231004A96B000C013632009A4000
:10DCC800104204D00F689A00AA1857600431013333
:10DCD800102BF3D10020A304C7D4A963C5E71B19EF
:10DCE800102BC1D843460F2BBED82B681E4206D036
:10DCF8000322280093432B60483000F0A5F820AF9A
:10DD0800380000F0A1F8AA6B002C24D04346DB00B1
:10DD1800FF180023994664000023A400D158F95045
:10DD280004339C42FAD14B4612196F46002B0FD090
:10DD38004046102800D210204B46D9000023103846
:10DD4800C0003818D458C45004339942FAD1521834
:10DD5800012EA1D120AF04323800AA6300F072F876
:10DD6800002082E7934303605130FF3000F078F8D9
:10DD78005FE7102B3BD910225242914699442B68F9
:10DD8800194208D0022228008B4313432B604830E5
:10DD980000F05EF82B6804221A4221D143460F2B6B
:10DDA80003D820AF380000F053F86F46380000F071
:10DDB80053F810244346AA6BE41A002CB8DD4346F6
:10DDC80020AFDB006400FF18A6E793430360D1305F
:10DDD800FF3000F049F806E720A800F037F860E7C0
:10DDE800280093432B60D03000F036F8D6E72B6834
:10DDF8000B4207D0022228008B4313432B60483084
:10DE080000F026F820AF380000F022F8A146AA6BEF
:10DE1800002C00D07AE73FE7011C343138C9043BB5
:10DE28009C461D60A646011C20313CC99046994677
:10DE3800A246AB46011C0831FCC941680068E546AA
:10DE480000BDC0467047C0467047C0467047C046D0
:10DE58007047C0467047C0467047C0467047C046C6
:10DE68007047C0467047C0467047C04601B401A815
:10DE780001B585B0FFB408A841464A4653465C46FA
:10DE880065463EC001A83EC80F98009000230CB418
:10DE980001A9FFF71DFC109B12B0184701B401A897
:10DEA80001B585B0FFB408A841464A4653465C46CA
:10DEB80065463EC001A83EC80F98009000230CB4E8
:10DEC80001A9FFF739FC109B12B0184701B401A84B
:10DED80001B585B0FFB408A841464A4653465C469A
:10DEE80065463EC001A83EC80F98009000230CB4B8
:10DEF80001A9FFF745FC109B12B0184701B401A80F
:10DF080001B585B0FFB408A841464A4653465C4669
:10DF180065463EC001A83EC80F98009000230CB487
:10DF280001ABFFF7FFFB109B12B0184701B401A823
:10DF380001B585B0FFB408A841464A4653465C4639
:10DF480065463EC001A83EC80F98009000230CB457
:10DF580001AAFFF775FC109B12B01847027A03005C
:10DF6800002A0BD1427A002A0FD0013A4272426845
:10DF7800111D416003211268017202E0013A027228
:10DF88000268100E12021A607047B020FCE7C04603
:10DF980000B585B003AB00930C2200230021FFF7E6
:10DFA80007FC039805B000BD10B5FFF7F1FF10BDE1
:10DFB800F0B557464E464546DE460023E0B587B0E5
:10DFC80003930F339846083B994680231B030600AA
:10DFD8000F009A463800FFF7C1FF0400B02800D1AF
:10DFE800C3E003062AD5030042469343DBB2802BE5
:10DFF80000D171E0902B3DD0A02B00D185E0B02B53
:10E0080050D0C02B00D196E003004A469343DBB2C0
:10E01800D02B0AD15346024001321A43052301216D
:10E028003000FFF7C7FD0028D4D00924200007B02E
:10E038003CBC90469946A246AB46F0BDFF23820001
:10E0480013401D1D05AB9B4600930D2200230021A4
:10E058003000FFF7ADFB630620D4059B9C46654462
:10E0680005955B460D220093002100233000FFF741
:10E07800C3FBAFE7833B03400D2BD6D005AD024071
:10E088000095002300213000FFF792FB0095002344
:10E098000D2200213000FFF7AFFB9BE7059B5D1BBE
:10E0A8000595DEE7B12874D0B22800D1CFE0B328B7
:10E0B80000D184E0FC230340B42BB6D04A46534633
:10E0C800024001321A43012101233000FFF772FD9B
:10E0D800002800D17EE7A8E704023800FFF73EFFDA
:10E0E800802520432D02A8429FD004010005020C80
:10E0F800002300213000FFF75DFD002895D12C4258
:10E1080000D167E70123039364E7FF234A461B0115
:10E118001900824311410A001A40030702D58023DF
:10E12800DB011A43002300213000FFF743FD0028DC
:10E1380000D14FE779E7C6284CD0C7285ED0030046
:10E148004A469343DBB2C02B6DD0C82872D0C92889
:10E1580000D06AE73800FFF701FFF02302031B0332
:10E16800134042460240013257E7039B0024002B2C
:10E1780000D05BE705AD00950E2200213000FFF7C7
:10E1880017FB009500230F2200213000FFF734FB16
:10E198004CE73800FFF7E2FE002800D145E703000E
:10E1A80042469343DBB2002B00D03EE70200002139
:10E1B8003000FFF7FFFC002800D10BE735E73800F7
:10E1C800FFF7CCFEF02302031B0313404246024034
:10E1D800013277E73800FFF7C1FEF02302031B0383
:10E1E80013404246024001321A4303230321300000
:10E1F800FFF7E0FC002800D1ECE616E73800FFF74F
:10E20800ADFE021E00D110E7030041468B43DBB28E
:10E21800002B00D009E704213000FFF7CBFC0028D1
:10E2280000D1D7E601E74346A0221C40013412037F
:10E238002243DAE73800FFF791FE434602009A438B
:10E24800D2B210321840120301300243E6E605ABA1
:10E2580000939B460D22002300213000FFF7A8FA07
:10E268003800FFF77BFE030618D57F25B03C059BD9
:10E278002840A0409C466044059038000734FFF7CA
:10E288006DFE0306F3D481217F23890003408C4669
:10E29800A340059A62449B180593E2E60224F2E73C
:10E2A800030000B5DB6C85B05A68080012020192C1
:10E2B8001A0001A908324A6003220A72DB794B72FC
:10E2C800FFF776FE05B000BD10B5FFF76DFE806C58
:10E2D80010BDC04610B5FFF767FEC26CD3799B002E
:10E2E8000833D01810BDC04610B500F065F8C04618
:10E2F80010B5FFF7F9FFC046F0B588420AD98B1868
:10E30800984207D2531E002A03D0CA5CC254013B6C
:10E31800FBD2F0BD0F2A09D80500002AF9D0002346
:10E32800CC5CEC5401339342FAD1F2E70D0005437B
:10E338000C000300AD0729D11500103D2D092F0150
:10E348003F18103726681E6066685E60A6689E6083
:10E35800E6681034DE601033BB42F3D10F24013578
:10E368002D01491914404519032C11D90023CE5801
:10E37800EE500433E61A032EF9D80323043CA4080C
:10E388000134A4002D1909191A40C6E70500C6E78B
:10E398002200C2E70000000001B40248844601BC24
:10E3A800604700BF5572001001B40248844601BCA2
:10E3B800604700BFE92A001001B40248844601BC46
:10E3C800604700BF11BB001001B40248844601BC7D
:10E3D800604700BF652D001001B40248844601BCA7
:10E3E800604700BF717100105045315258462D35B5
:10E3F80000005045315258462D33000041505A4DC7
:10E40800444D0000000000494445312D3100000012
:10E4180000494445322D3200000056312C436F6EBE
:10E4280074726F6C6C65722030310000000000005F
:10E438000100000048E801000500000098E1DA1931
:10E44800080000000C00000011000000100000008F
:10E458003814002000000000581D0020B8230020B8
:10E468000000000000000000C82300200000000099
:10E478000000000010000000000000000000010083
:10E488000000000000000000000002000000000082
:10E498000000000000000300000000000000000071
:10E4A8000000FF000000000000B5486801318E46FA
:10E4B8000047704609380149884700BDE13B001014
:10E4C800503300004C330000543300005233000036
:10E4D8004D5300004D430000533400004334000006
:10E4E800E9770010000000005177001000000000DC
:10E4F8000001000020CD001024CD00108C2C00203D
:10E5080010000C000000E0FF1F00000000000000E9
:10E5180000000000000000000000000000000000F3
:10E52800F81400200000000000000000E41700209C
:10E538004C180020B4180020000000000000000063
:10E5480000000000000000000000000000000000C3
:10E5580000000000000000000000000000000000B3
:10E5680000000000000000000000000000000000A3
:10E578000000000000000000000000000000000093
:10E588000000000000000000000000000000000083
:10E598000000000000000000000000000000000073
:10E5A8000000000000000000000000000000000063
:10E5B8000000000000000000000000000000000053
:10E5C8000000000000000000000000000000000043
:10E5D80001000000000000000E33CDAB34126DE6E0
:10E5E800ECDE05000B000000000000000000000049
:10E5F8000000000000000000000000000000000013
:10E608000000000000000000000000000000000002
:10E6180000000000000000000000000000000000F2
:10E6280000000000000000000000000000000000E2
:10E95800FFFFFFFF000002000000000000000000B1
:10E96800281900202819002030190020301900200B
:10E9780038190020381900204019002040190020BB
:10E98800481900204819002050190020501900206B
:10E99800581900205819002060190020601900201B
:10E9A80068190020681900207019002070190020CB
:10E9B800781900207819002080190020801900207B
:10E9C800881900208819002090190020901900202B
:10E9D8009819002098190020A0190020A0190020DB
:10E9E800A8190020A8190020B0190020B01900208B
:10E9F800B8190020B8190020C0190020C01900203B
:10EA0800C8190020C8190020D0190020D0190020EA
:10EA1800D8190020D8190020E0190020E01900209A
:10EA2800E8190020E8190020F0190020F01900204A
:10EA3800F8190020F8190020001A0020001A0020F8
:10EA4800081A0020081A0020101A0020101A0020A6
:10EA5800181A0020181A0020201A0020201A002056
:10EA6800281A0020281A0020301A0020301A002006
:10EA7800381A0020381A0020401A0020401A0020B6
:10EA8800481A0020481A0020501A0020501A002066
:10EA9800581A0020581A0020601A0020601A002016
:10EAA800681A0020681A0020701A0020701A0020C6
:10EAB800781A0020781A0020801A0020801A002076
:10EAC800881A0020881A0020901A0020901A002026
:10EAD800981A0020981A0020A01A0020A01A0020D6
:10EAE800A81A0020A81A0020B01A0020B01A002086
:10EAF800B81A0020B81A0020C01A0020C01A002036
:10EB0800C81A0020C81A0020D01A0020D01A0020E5
:10EB1800D81A0020D81A0020E01A0020E01A002095
:10EB2800E81A0020E81A0020F01A0020F01A002045
:10EB3800F81A0020F81A0020001B0020001B0020F3
:10EB4800081B0020081B0020101B0020101B0020A1
:10EB5800181B0020181B0020201B0020201B002051
:10EB6800281B0020281B0020301B0020301B002001
:10EB7800381B0020381B0020401B0020401B0020B1
:10EB8800481B0020481B0020501B0020501B002061
:10EB9800581B0020581B0020601B0020601B002011
:10EBA800681B0020681B0020701B0020701B0020C1
:10EBB800781B0020781B0020801B0020801B002071
:10EBC800881B0020881B0020901B0020901B002021
:10EBD800981B0020981B0020A01B0020A01B0020D1
:10EBE800A81B0020A81B0020B01B0020B01B002081
:10EBF800B81B0020B81B0020C01B0020C01B002031
:10EC0800C81B0020C81B0020D01B0020D01B0020E0
:10EC1800D81B0020D81B0020E01B0020E01B002090
:10EC2800E81B0020E81B0020F01B0020F01B002040
:10EC3800F81B0020F81B0020001C0020001C0020EE
:10EC4800081C0020081C0020101C0020101C00209C
:10EC5800181C0020181C0020201C0020201C00204C
:10EC6800281C0020281C0020301C0020301C0020FC
:10EC7800381C0020381C0020401C0020401C0020AC
:10EC8800481C0020481C0020501C0020501C00205C
:10EC9800581C0020581C0020601C0020601C00200C
:10ECA800681C0020681C0020701C0020701C0020BC
:10ECB800781C0020781C0020801C0020801C00206C
:10ECC800881C0020881C0020901C0020901C00201C
:10ECD800981C0020981C0020A01C0020A01C0020CC
:10ECE800A81C0020A81C0020B01C0020B01C00207C
:10ECF800B81C0020B81C0020C01C0020C01C00202C
:10ED0800C81C0020C81C0020D01C0020D01C0020DB
:10ED1800D81C0020D81C0020E01C0020E01C00208B
:10ED2800E81C0020E81C0020F01C0020F01C00203B
:10ED3800F81C0020F81C0020001D0020001D0020E9
:10ED4800081D0020081D0020101D0020101D002097
:10ED5800181D0020181D0020201D0020201D002047
:10ED68000000000000000000397200109D640010CF
:10ED7800B16B0010A5710010390300109D0C001034
:08ED8800F99E0010DDBA001035
:04000005100001E9FD
:00000001FF
